Component: ARM Compiler 5.06 update 1 (build 61) Tool: armlink [4d35a8]

==============================================================================

Section Cross References

    main.o(i.ENS210_set_mode) refers to main.o(i.nrf_drv_twi_tx) for nrf_drv_twi_tx
    main.o(i.ENS210_set_mode) refers to app_error.o(i.app_error_handler_bare) for app_error_handler_bare
    main.o(i.ENS210_set_mode) refers to main.o(i.nrf_drv_twi_rx) for nrf_drv_twi_rx
    main.o(i.ENS210_set_mode) refers to main.o(.data) for .data
    main.o(i.ENS210_set_mode) refers to main.o(.constdata) for .constdata
    main.o(i.assert_nrf_callback) refers to app_error_handler_keil.o(.emb_text) for app_error_handler
    main.o(i.ble_evt_handler) refers to nrf_log_frontend.o(i.nrf_log_frontend_std_0) for nrf_log_frontend_std_0
    main.o(i.ble_evt_handler) refers to bsp.o(i.bsp_indication_set) for bsp_indication_set
    main.o(i.ble_evt_handler) refers to app_error.o(i.app_error_handler_bare) for app_error_handler_bare
    main.o(i.ble_evt_handler) refers to main.o(.data) for .data
    main.o(i.ble_evt_handler) refers to nrf_log_frontend.o(log_const_data) for m_nrf_log_app_logs_data_const
    main.o(i.bsp_event_handler) refers to main.o(i.sleep_mode_enter) for sleep_mode_enter
    main.o(i.bsp_event_handler) refers to app_error.o(i.app_error_handler_bare) for app_error_handler_bare
    main.o(i.bsp_event_handler) refers to ble_advertising.o(i.ble_advertising_restart_without_whitelist) for ble_advertising_restart_without_whitelist
    main.o(i.bsp_event_handler) refers to main.o(.data) for .data
    main.o(i.bsp_event_handler) refers to main.o(.bss) for .bss
    main.o(i.buttons_leds_init) refers to main.o(i.nrf_gpio_cfg_output) for nrf_gpio_cfg_output
    main.o(i.buttons_leds_init) refers to main.o(i.nrf_gpio_pin_clear) for nrf_gpio_pin_clear
    main.o(i.buttons_leds_init) refers to main.o(i.nrf_delay_ms) for nrf_delay_ms
    main.o(i.buttons_leds_init) refers to main.o(i.nrf_gpio_pin_set) for nrf_gpio_pin_set
    main.o(i.conn_params_error_handler) refers to app_error.o(i.app_error_handler_bare) for app_error_handler_bare
    main.o(i.gatt_evt_handler) refers to nrf_log_frontend.o(i.nrf_log_frontend_std_2) for nrf_log_frontend_std_2
    main.o(i.gatt_evt_handler) refers to main.o(.data) for .data
    main.o(i.gatt_evt_handler) refers to nrf_log_frontend.o(log_const_data) for m_nrf_log_app_logs_data_const
    main.o(i.gatt_init) refers to nrf_ble_gatt.o(i.nrf_ble_gatt_init) for nrf_ble_gatt_init
    main.o(i.gatt_init) refers to app_error.o(i.app_error_handler_bare) for app_error_handler_bare
    main.o(i.gatt_init) refers to nrf_ble_gatt.o(i.nrf_ble_gatt_att_mtu_periph_set) for nrf_ble_gatt_att_mtu_periph_set
    main.o(i.gatt_init) refers to main.o(i.gatt_evt_handler) for gatt_evt_handler
    main.o(i.gatt_init) refers to main.o(.bss) for .bss
    main.o(i.heart_rate_meas_timeout_handler) refers to malloc.o(i.malloc) for malloc
    main.o(i.heart_rate_meas_timeout_handler) refers to main.o(i.read_ENS210_sensor_data) for read_ENS210_sensor_data
    main.o(i.heart_rate_meas_timeout_handler) refers to ble_nus.o(i.ble_nus_data_send) for ble_nus_data_send
    main.o(i.heart_rate_meas_timeout_handler) refers to malloc.o(i.free) for free
    main.o(i.heart_rate_meas_timeout_handler) refers to main.o(.data) for .data
    main.o(i.main) refers to memcpya.o(.text) for __aeabi_memcpy4
    main.o(i.main) refers to app_uart_fifo.o(i.app_uart_init) for app_uart_init
    main.o(i.main) refers to app_error.o(i.app_error_handler_bare) for app_error_handler_bare
    main.o(i.main) refers to nrf_log_frontend.o(i.nrf_log_init) for nrf_log_init
    main.o(i.main) refers to nrf_log_default_backends.o(i.nrf_log_default_backends_init) for nrf_log_default_backends_init
    main.o(i.main) refers to app_timer.o(i.app_timer_init) for app_timer_init
    main.o(i.main) refers to app_timer.o(i.app_timer_create) for app_timer_create
    main.o(i.main) refers to main.o(i.buttons_leds_init) for buttons_leds_init
    main.o(i.main) refers to nrf_pwr_mgmt.o(i.nrf_pwr_mgmt_init) for nrf_pwr_mgmt_init
    main.o(i.main) refers to nrf_sdh.o(i.nrf_sdh_enable_request) for nrf_sdh_enable_request
    main.o(i.main) refers to nrf_sdh_ble.o(i.nrf_sdh_ble_default_cfg_set) for nrf_sdh_ble_default_cfg_set
    main.o(i.main) refers to nrf_sdh_ble.o(i.nrf_sdh_ble_enable) for nrf_sdh_ble_enable
    main.o(i.main) refers to main.o(i.gatt_init) for gatt_init
    main.o(i.main) refers to nrf_ble_qwr.o(i.nrf_ble_qwr_init) for nrf_ble_qwr_init
    main.o(i.main) refers to ble_nus.o(i.ble_nus_init) for ble_nus_init
    main.o(i.main) refers to memseta.o(.text) for __aeabi_memclr4
    main.o(i.main) refers to ble_advertising.o(i.ble_advertising_init) for ble_advertising_init
    main.o(i.main) refers to ble_advertising.o(i.ble_advertising_conn_cfg_tag_set) for ble_advertising_conn_cfg_tag_set
    main.o(i.main) refers to ble_conn_params.o(i.ble_conn_params_init) for ble_conn_params_init
    main.o(i.main) refers to main.o(i.twi_init) for twi_init
    main.o(i.main) refers to main.o(i.ENS210_set_mode) for ENS210_set_mode
    main.o(i.main) refers to app_timer.o(i.app_timer_start) for app_timer_start
    main.o(i.main) refers to nrf_log_frontend.o(i.nrf_log_frontend_std_0) for nrf_log_frontend_std_0
    main.o(i.main) refers to ble_advertising.o(i.ble_advertising_start) for ble_advertising_start
    main.o(i.main) refers to nrf_log_frontend.o(i.nrf_log_frontend_dequeue) for nrf_log_frontend_dequeue
    main.o(i.main) refers to nrf_pwr_mgmt.o(i.nrf_pwr_mgmt_run) for nrf_pwr_mgmt_run
    main.o(i.main) refers to main.o(.constdata) for .constdata
    main.o(i.main) refers to main.o(.bss) for .bss
    main.o(i.main) refers to main.o(i.uart_event_handle) for uart_event_handle
    main.o(i.main) refers to main.o(i.heart_rate_meas_timeout_handler) for heart_rate_meas_timeout_handler
    main.o(i.main) refers to main.o(i.nrf_qwr_error_handler) for nrf_qwr_error_handler
    main.o(i.main) refers to main.o(i.nus_data_handler) for nus_data_handler
    main.o(i.main) refers to main.o(.data) for .data
    main.o(i.main) refers to main.o(i.on_adv_evt) for on_adv_evt
    main.o(i.main) refers to main.o(i.on_conn_params_evt) for on_conn_params_evt
    main.o(i.main) refers to main.o(i.conn_params_error_handler) for conn_params_error_handler
    main.o(i.main) refers to nrf_log_frontend.o(log_const_data) for m_nrf_log_app_logs_data_const
    main.o(i.nrf_delay_ms) refers to main.o(.constdata) for .constdata
    main.o(i.nrf_drv_twi_rx) refers to nrfx_twim.o(i.nrfx_twim_rx) for nrfx_twim_rx
    main.o(i.nrf_drv_twi_tx) refers to nrfx_twim.o(i.nrfx_twim_tx) for nrfx_twim_tx
    main.o(i.nrf_qwr_error_handler) refers to app_error.o(i.app_error_handler_bare) for app_error_handler_bare
    main.o(i.nus_data_handler) refers to nrf_log_frontend.o(i.nrf_log_frontend_std_0) for nrf_log_frontend_std_0
    main.o(i.nus_data_handler) refers to nrf_log_frontend.o(log_const_data) for m_nrf_log_app_logs_data_const
    main.o(i.on_adv_evt) refers to bsp.o(i.bsp_indication_set) for bsp_indication_set
    main.o(i.on_adv_evt) refers to app_error.o(i.app_error_handler_bare) for app_error_handler_bare
    main.o(i.on_adv_evt) refers to main.o(i.sleep_mode_enter) for sleep_mode_enter
    main.o(i.on_conn_params_evt) refers to app_error.o(i.app_error_handler_bare) for app_error_handler_bare
    main.o(i.on_conn_params_evt) refers to main.o(.data) for .data
    main.o(i.read_ENS210_sensor_data) refers to main.o(i.nrf_drv_twi_tx) for nrf_drv_twi_tx
    main.o(i.read_ENS210_sensor_data) refers to app_error.o(i.app_error_handler_bare) for app_error_handler_bare
    main.o(i.read_ENS210_sensor_data) refers to main.o(i.nrf_drv_twi_rx) for nrf_drv_twi_rx
    main.o(i.read_ENS210_sensor_data) refers to main.o(.data) for .data
    main.o(i.read_ENS210_sensor_data) refers to main.o(.constdata) for .constdata
    main.o(i.sleep_mode_enter) refers to bsp.o(i.bsp_indication_set) for bsp_indication_set
    main.o(i.sleep_mode_enter) refers to app_error.o(i.app_error_handler_bare) for app_error_handler_bare
    main.o(i.sleep_mode_enter) refers to bsp_btn_ble.o(i.bsp_btn_ble_sleep_mode_prepare) for bsp_btn_ble_sleep_mode_prepare
    main.o(i.twi_handler) refers to ffltui.o(.text) for __aeabi_ui2f
    main.o(i.twi_handler) refers to fscalb.o(.text) for __ARM_scalbnf
    main.o(i.twi_handler) refers to fadd.o(.text) for __aeabi_fsub
    main.o(i.twi_handler) refers to ffixui.o(.text) for __aeabi_f2uiz
    main.o(i.twi_handler) refers to nrf_log_frontend.o(i.nrf_log_frontend_std_1) for nrf_log_frontend_std_1
    main.o(i.twi_handler) refers to nrf_log_frontend.o(i.nrf_log_frontend_std_0) for nrf_log_frontend_std_0
    main.o(i.twi_handler) refers to main.o(.data) for .data
    main.o(i.twi_handler) refers to nrf_log_frontend.o(log_const_data) for m_nrf_log_app_logs_data_const
    main.o(i.twi_init) refers to nrf_drv_twi.o(i.nrf_drv_twi_init) for nrf_drv_twi_init
    main.o(i.twi_init) refers to app_error.o(i.app_error_handler_bare) for app_error_handler_bare
    main.o(i.twi_init) refers to nrfx_twim.o(i.nrfx_twim_enable) for nrfx_twim_enable
    main.o(i.twi_init) refers to main.o(.constdata) for .constdata
    main.o(i.twi_init) refers to main.o(i.twi_handler) for twi_handler
    main.o(i.uart_event_handle) refers to app_uart_fifo.o(i.app_uart_get) for app_uart_get
    main.o(i.uart_event_handle) refers to ble_nus.o(i.ble_nus_data_send) for ble_nus_data_send
    main.o(i.uart_event_handle) refers to app_error.o(i.app_error_handler_bare) for app_error_handler_bare
    main.o(i.uart_event_handle) refers to main.o(.bss) for .bss
    main.o(i.uart_event_handle) refers to main.o(.data) for .data
    main.o(.constdata) refers to main.o(.bss) for m_heart_rate_timer_id_data
    main.o(.data) refers to main.o(.data) for m_nus_link_ctx_storage_ctx_data_pool
    main.o(.data) refers to main.o(.data) for m_nus_link_ctx_storage
    main.o(sdh_ble_observers1) refers to nrf_ble_gatt.o(i.nrf_ble_gatt_on_ble_evt) for nrf_ble_gatt_on_ble_evt
    main.o(sdh_ble_observers1) refers to main.o(.bss) for m_gatt
    main.o(sdh_ble_observers1) refers to ble_advertising.o(i.ble_advertising_on_ble_evt) for ble_advertising_on_ble_evt
    main.o(sdh_ble_observers2) refers to ble_nus.o(i.ble_nus_on_ble_evt) for ble_nus_on_ble_evt
    main.o(sdh_ble_observers2) refers to main.o(.data) for m_nus
    main.o(sdh_ble_observers2) refers to nrf_ble_qwr.o(i.nrf_ble_qwr_on_ble_evt) for nrf_ble_qwr_on_ble_evt
    main.o(sdh_ble_observers2) refers to main.o(.bss) for m_qwr
    main.o(sdh_ble_observers3) refers to main.o(i.ble_evt_handler) for ble_evt_handler
    main.o(sdh_soc_observers1) refers to ble_advertising.o(i.ble_advertising_on_sys_evt) for ble_advertising_on_sys_evt
    main.o(sdh_soc_observers1) refers to main.o(.bss) for m_advertising
    boards.o(i.bsp_board_button_idx_to_pin) refers to boards.o(.constdata) for .constdata
    boards.o(i.bsp_board_button_state_get) refers to boards.o(.constdata) for .constdata
    boards.o(i.bsp_board_init) refers to boards.o(i.nrf_gpio_cfg) for nrf_gpio_cfg
    boards.o(i.bsp_board_init) refers to boards.o(i.bsp_board_leds_off) for bsp_board_leds_off
    boards.o(i.bsp_board_init) refers to boards.o(.constdata) for .constdata
    boards.o(i.bsp_board_led_idx_to_pin) refers to boards.o(.constdata) for .constdata
    boards.o(i.bsp_board_led_invert) refers to boards.o(.constdata) for .constdata
    boards.o(i.bsp_board_led_off) refers to boards.o(i.nrf_gpio_pin_write) for nrf_gpio_pin_write
    boards.o(i.bsp_board_led_off) refers to boards.o(.constdata) for .constdata
    boards.o(i.bsp_board_led_on) refers to boards.o(i.nrf_gpio_pin_write) for nrf_gpio_pin_write
    boards.o(i.bsp_board_led_on) refers to boards.o(.constdata) for .constdata
    boards.o(i.bsp_board_led_state_get) refers to boards.o(.constdata) for .constdata
    boards.o(i.bsp_board_leds_off) refers to boards.o(i.bsp_board_led_off) for bsp_board_led_off
    boards.o(i.bsp_board_leds_on) refers to boards.o(i.bsp_board_led_on) for bsp_board_led_on
    boards.o(i.bsp_board_pin_to_button_idx) refers to boards.o(.constdata) for .constdata
    boards.o(i.bsp_board_pin_to_led_idx) refers to boards.o(.constdata) for .constdata
    bsp.o(i.alert_timer_handler) refers to boards.o(i.bsp_board_led_invert) for bsp_board_led_invert
    bsp.o(i.bsp_button_event_handler) refers to boards.o(i.bsp_board_pin_to_button_idx) for bsp_board_pin_to_button_idx
    bsp.o(i.bsp_button_event_handler) refers to app_timer.o(i.app_timer_start) for app_timer_start
    bsp.o(i.bsp_button_event_handler) refers to app_timer.o(i.app_timer_stop) for app_timer_stop
    bsp.o(i.bsp_button_event_handler) refers to bsp.o(.constdata) for .constdata
    bsp.o(i.bsp_button_event_handler) refers to bsp.o(.data) for .data
    bsp.o(i.bsp_button_event_handler) refers to bsp.o(.bss) for .bss
    bsp.o(i.bsp_button_is_pressed) refers to boards.o(i.bsp_board_button_state_get) for bsp_board_button_state_get
    bsp.o(i.bsp_buttons_disable) refers to app_button.o(i.app_button_disable) for app_button_disable
    bsp.o(i.bsp_buttons_enable) refers to app_button.o(i.app_button_enable) for app_button_enable
    bsp.o(i.bsp_event_to_button_action_assign) refers to bsp.o(.bss) for .bss
    bsp.o(i.bsp_indication_set) refers to bsp.o(i.bsp_led_indication) for bsp_led_indication
    bsp.o(i.bsp_indication_set) refers to bsp.o(.data) for .data
    bsp.o(i.bsp_init) refers to bsp.o(i.bsp_event_to_button_action_assign) for bsp_event_to_button_action_assign
    bsp.o(i.bsp_init) refers to app_button.o(i.app_button_init) for app_button_init
    bsp.o(i.bsp_init) refers to app_button.o(i.app_button_enable) for app_button_enable
    bsp.o(i.bsp_init) refers to app_timer.o(i.app_timer_create) for app_timer_create
    bsp.o(i.bsp_init) refers to boards.o(i.bsp_board_init) for bsp_board_init
    bsp.o(i.bsp_init) refers to bsp.o(.data) for .data
    bsp.o(i.bsp_init) refers to bsp.o(.constdata) for .constdata
    bsp.o(i.bsp_init) refers to bsp.o(i.button_timer_handler) for button_timer_handler
    bsp.o(i.bsp_init) refers to bsp.o(i.leds_timer_handler) for leds_timer_handler
    bsp.o(i.bsp_init) refers to bsp.o(i.alert_timer_handler) for alert_timer_handler
    bsp.o(i.bsp_led_indication) refers to bsp.o(i.leds_off) for leds_off
    bsp.o(i.bsp_led_indication) refers to app_timer.o(i.app_timer_stop) for app_timer_stop
    bsp.o(i.bsp_led_indication) refers to boards.o(i.bsp_board_led_state_get) for bsp_board_led_state_get
    bsp.o(i.bsp_led_indication) refers to boards.o(i.bsp_board_led_off) for bsp_board_led_off
    bsp.o(i.bsp_led_indication) refers to boards.o(i.bsp_board_led_on) for bsp_board_led_on
    bsp.o(i.bsp_led_indication) refers to uldiv.o(.text) for __aeabi_uldivmod
    bsp.o(i.bsp_led_indication) refers to app_timer.o(i.app_timer_start) for app_timer_start
    bsp.o(i.bsp_led_indication) refers to boards.o(i.bsp_board_led_invert) for bsp_board_led_invert
    bsp.o(i.bsp_led_indication) refers to boards.o(i.bsp_board_leds_on) for bsp_board_leds_on
    bsp.o(i.bsp_led_indication) refers to bsp.o(.data) for .data
    bsp.o(i.bsp_led_indication) refers to bsp.o(.constdata) for .constdata
    bsp.o(i.bsp_wakeup_button_disable) refers to bsp.o(i.wakeup_button_cfg) for wakeup_button_cfg
    bsp.o(i.bsp_wakeup_button_enable) refers to bsp.o(i.wakeup_button_cfg) for wakeup_button_cfg
    bsp.o(i.button_timer_handler) refers to bsp.o(i.bsp_button_event_handler) for bsp_button_event_handler
    bsp.o(i.leds_off) refers to boards.o(i.bsp_board_led_off) for bsp_board_led_off
    bsp.o(i.leds_off) refers to boards.o(i.bsp_board_leds_off) for bsp_board_leds_off
    bsp.o(i.leds_off) refers to bsp.o(.data) for .data
    bsp.o(i.leds_timer_handler) refers to bsp.o(i.bsp_led_indication) for bsp_led_indication
    bsp.o(i.leds_timer_handler) refers to bsp.o(.data) for .data
    bsp.o(i.wakeup_button_cfg) refers to boards.o(i.bsp_board_button_idx_to_pin) for bsp_board_button_idx_to_pin
    bsp.o(.constdata) refers to bsp.o(.bss) for m_bsp_leds_tmr_data
    bsp.o(.constdata) refers to bsp.o(.bss) for m_bsp_alert_tmr_data
    bsp.o(.constdata) refers to bsp.o(.bss) for m_bsp_button_tmr_data
    bsp.o(.constdata) refers to bsp.o(i.bsp_button_event_handler) for bsp_button_event_handler
    bsp_btn_ble.o(i.advertising_buttons_configure) refers to bsp.o(i.bsp_event_to_button_action_assign) for bsp_event_to_button_action_assign
    bsp_btn_ble.o(i.ble_evt_handler) refers to bsp_btn_ble.o(i.advertising_buttons_configure) for advertising_buttons_configure
    bsp_btn_ble.o(i.ble_evt_handler) refers to bsp.o(i.bsp_event_to_button_action_assign) for bsp_event_to_button_action_assign
    bsp_btn_ble.o(i.ble_evt_handler) refers to bsp_btn_ble.o(.data) for .data
    bsp_btn_ble.o(i.bsp_btn_ble_init) refers to bsp.o(i.bsp_button_is_pressed) for bsp_button_is_pressed
    bsp_btn_ble.o(i.bsp_btn_ble_init) refers to bsp_btn_ble.o(i.advertising_buttons_configure) for advertising_buttons_configure
    bsp_btn_ble.o(i.bsp_btn_ble_init) refers to bsp_btn_ble.o(.data) for .data
    bsp_btn_ble.o(i.bsp_btn_ble_sleep_mode_prepare) refers to bsp.o(i.bsp_wakeup_button_enable) for bsp_wakeup_button_enable
    bsp_btn_ble.o(sdh_ble_observers1) refers to bsp_btn_ble.o(i.ble_evt_handler) for ble_evt_handler
    utf.o(i.utf16RuneCount) refers to utf.o(i.utf16DecodeRune) for utf16DecodeRune
    utf.o(i.utf16UTF8Count) refers to utf.o(i.utf16DecodeRune) for utf16DecodeRune
    utf.o(i.utf16UTF8Count) refers to utf.o(i.utf8EncodeRune) for utf8EncodeRune
    utf.o(i.utf8RuneCount) refers to utf.o(i.utf8DecodeRune) for utf8DecodeRune
    utf.o(i.utf8UTF16Count) refers to utf.o(i.utf8DecodeRune) for utf8DecodeRune
    utf.o(i.utf8UTF16Count) refers to utf.o(i.utf16EncodeRune) for utf16EncodeRune
    ble_advdata.o(i.ble_advdata_appearance_find) refers to ble_advdata.o(i.ble_advdata_search) for ble_advdata_search
    ble_advdata.o(i.ble_advdata_encode) refers to ble_advdata.o(i.ble_device_addr_encode) for ble_device_addr_encode
    ble_advdata.o(i.ble_advdata_encode) refers to ble_advdata.o(i.uint16_encode) for uint16_encode
    ble_advdata.o(i.ble_advdata_encode) refers to ble_advdata.o(i.uuid_list_encode) for uuid_list_encode
    ble_advdata.o(i.ble_advdata_encode) refers to ble_advdata.o(i.conn_int_encode) for conn_int_encode
    ble_advdata.o(i.ble_advdata_encode) refers to ble_advdata.o(i.manuf_specific_data_encode) for manuf_specific_data_encode
    ble_advdata.o(i.ble_advdata_encode) refers to ble_advdata.o(i.service_data_encode) for service_data_encode
    ble_advdata.o(i.ble_advdata_encode) refers to ble_advdata.o(i.name_encode) for name_encode
    ble_advdata.o(i.ble_advdata_name_find) refers to ble_advdata.o(i.ble_advdata_search) for ble_advdata_search
    ble_advdata.o(i.ble_advdata_name_find) refers to strlen.o(.text) for strlen
    ble_advdata.o(i.ble_advdata_name_find) refers to memcmp.o(.text) for memcmp
    ble_advdata.o(i.ble_advdata_parse) refers to ble_advdata.o(i.ble_advdata_search) for ble_advdata_search
    ble_advdata.o(i.ble_advdata_short_name_find) refers to ble_advdata.o(i.ble_advdata_search) for ble_advdata_search
    ble_advdata.o(i.ble_advdata_short_name_find) refers to strlen.o(.text) for strlen
    ble_advdata.o(i.ble_advdata_short_name_find) refers to memcmp.o(.text) for memcmp
    ble_advdata.o(i.ble_advdata_uuid_find) refers to ble_advdata.o(i.ble_advdata_search) for ble_advdata_search
    ble_advdata.o(i.ble_advdata_uuid_find) refers to memcmp.o(.text) for memcmp
    ble_advdata.o(i.conn_int_encode) refers to ble_advdata.o(i.uint16_encode) for uint16_encode
    ble_advdata.o(i.manuf_specific_data_encode) refers to ble_advdata.o(i.uint16_encode) for uint16_encode
    ble_advdata.o(i.manuf_specific_data_encode) refers to memcpya.o(.text) for __aeabi_memcpy
    ble_advdata.o(i.service_data_encode) refers to ble_advdata.o(i.uint16_encode) for uint16_encode
    ble_advdata.o(i.service_data_encode) refers to memcpya.o(.text) for __aeabi_memcpy
    ble_advdata.o(i.uuid_list_encode) refers to ble_advdata.o(i.uuid_list_sized_encode) for uuid_list_sized_encode
    ble_advertising.o(i.ble_advertising_init) refers to memcpya.o(.text) for __aeabi_memcpy4
    ble_advertising.o(i.ble_advertising_init) refers to ble_advdata.o(i.ble_advdata_encode) for ble_advdata_encode
    ble_advertising.o(i.ble_advertising_modes_config_set) refers to memcpya.o(.text) for __aeabi_memcpy4
    ble_advertising.o(i.ble_advertising_on_ble_evt) refers to ble_advertising.o(i.ble_advertising_start) for ble_advertising_start
    ble_advertising.o(i.ble_advertising_restart_without_whitelist) refers to ble_advertising.o(i.flags_set) for flags_set
    ble_advertising.o(i.ble_advertising_restart_without_whitelist) refers to ble_advertising.o(i.ble_advertising_start) for ble_advertising_start
    ble_advertising.o(i.ble_advertising_start) refers to memseta.o(.text) for __aeabi_memclr4
    ble_advertising.o(i.ble_advertising_start) refers to ble_advertising.o(i.phy_is_valid) for phy_is_valid
    ble_advertising.o(i.ble_advertising_start) refers to ble_advertising.o(i.use_whitelist) for use_whitelist
    ble_advertising.o(i.ble_advertising_start) refers to ble_advertising.o(i.flags_set) for flags_set
    ble_advertising.o(i.flags_set) refers to ble_advdata.o(i.ble_advdata_parse) for ble_advdata_parse
    ble_conn_params.o(i.ble_conn_params_change_conn_params) refers to ble_conn_params.o(i.instance_get) for instance_get
    ble_conn_params.o(i.ble_conn_params_change_conn_params) refers to ble_conn_params.o(.data) for .data
    ble_conn_params.o(i.ble_conn_params_init) refers to memcpya.o(.text) for __aeabi_memcpy4
    ble_conn_params.o(i.ble_conn_params_init) refers to app_timer.o(i.app_timer_create) for app_timer_create
    ble_conn_params.o(i.ble_conn_params_init) refers to ble_conn_params.o(.bss) for .bss
    ble_conn_params.o(i.ble_conn_params_init) refers to ble_conn_params.o(.data) for .data
    ble_conn_params.o(i.ble_conn_params_init) refers to ble_conn_params.o(i.update_timeout_handler) for update_timeout_handler
    ble_conn_params.o(i.ble_conn_params_stop) refers to app_timer.o(i.app_timer_stop) for app_timer_stop
    ble_conn_params.o(i.ble_conn_params_stop) refers to ble_conn_params.o(.bss) for .bss
    ble_conn_params.o(i.ble_evt_handler) refers to ble_conn_params.o(i.instance_get) for instance_get
    ble_conn_params.o(i.ble_evt_handler) refers to ble_srv_common.o(i.ble_srv_is_notification_enabled) for ble_srv_is_notification_enabled
    ble_conn_params.o(i.ble_evt_handler) refers to ble_conn_params.o(i.is_conn_params_ok) for is_conn_params_ok
    ble_conn_params.o(i.ble_evt_handler) refers to app_timer.o(i.app_timer_stop) for app_timer_stop
    ble_conn_params.o(i.ble_evt_handler) refers to ble_conn_params.o(i.send_error_evt) for send_error_evt
    ble_conn_params.o(i.ble_evt_handler) refers to ble_conn_params.o(i.conn_params_negotiation) for conn_params_negotiation
    ble_conn_params.o(i.ble_evt_handler) refers to ble_conn_params.o(.bss) for .bss
    ble_conn_params.o(i.ble_evt_handler) refers to ble_conn_params.o(.data) for .data
    ble_conn_params.o(i.conn_params_negotiation) refers to app_timer.o(i.app_timer_start) for app_timer_start
    ble_conn_params.o(i.conn_params_negotiation) refers to ble_conn_params.o(i.send_error_evt) for send_error_evt
    ble_conn_params.o(i.conn_params_negotiation) refers to ble_conn_params.o(.bss) for .bss
    ble_conn_params.o(i.instance_get) refers to ble_conn_params.o(.bss) for .bss
    ble_conn_params.o(i.send_error_evt) refers to ble_conn_params.o(.bss) for .bss
    ble_conn_params.o(i.update_timeout_handler) refers to ble_conn_params.o(i.instance_get) for instance_get
    ble_conn_params.o(i.update_timeout_handler) refers to ble_conn_params.o(i.send_error_evt) for send_error_evt
    ble_conn_params.o(i.update_timeout_handler) refers to ble_conn_params.o(.bss) for .bss
    ble_conn_params.o(sdh_ble_observers1) refers to ble_conn_params.o(i.ble_evt_handler) for ble_evt_handler
    ble_conn_state.o(i.active_flag_count) refers to nrf_atflags.o(i.nrf_atflags_get) for nrf_atflags_get
    ble_conn_state.o(i.bcs_internal_state_reset) refers to memseta.o(.text) for __aeabi_memclr4
    ble_conn_state.o(i.bcs_internal_state_reset) refers to ble_conn_state.o(.bss) for .bss
    ble_conn_state.o(i.ble_conn_state_central_conn_count) refers to nrf_atomic.o(i.nrf_atomic_u32_and) for nrf_atomic_u32_and
    ble_conn_state.o(i.ble_conn_state_central_conn_count) refers to ble_conn_state.o(i.active_flag_count) for active_flag_count
    ble_conn_state.o(i.ble_conn_state_central_conn_count) refers to ble_conn_state.o(.bss) for .bss
    ble_conn_state.o(i.ble_conn_state_central_handles) refers to nrf_atomic.o(i.nrf_atomic_u32_and) for nrf_atomic_u32_and
    ble_conn_state.o(i.ble_conn_state_central_handles) refers to ble_conn_state.o(i.conn_handle_list_get) for conn_handle_list_get
    ble_conn_state.o(i.ble_conn_state_central_handles) refers to ble_conn_state.o(.bss) for .bss
    ble_conn_state.o(i.ble_conn_state_conn_count) refers to ble_conn_state.o(i.active_flag_count) for active_flag_count
    ble_conn_state.o(i.ble_conn_state_conn_count) refers to ble_conn_state.o(.bss) for .bss
    ble_conn_state.o(i.ble_conn_state_conn_handles) refers to ble_conn_state.o(i.conn_handle_list_get) for conn_handle_list_get
    ble_conn_state.o(i.ble_conn_state_conn_handles) refers to ble_conn_state.o(.bss) for .bss
    ble_conn_state.o(i.ble_conn_state_conn_idx) refers to ble_conn_state.o(i.ble_conn_state_valid) for ble_conn_state_valid
    ble_conn_state.o(i.ble_conn_state_encrypted) refers to ble_conn_state.o(i.ble_conn_state_valid) for ble_conn_state_valid
    ble_conn_state.o(i.ble_conn_state_encrypted) refers to nrf_atflags.o(i.nrf_atflags_get) for nrf_atflags_get
    ble_conn_state.o(i.ble_conn_state_encrypted) refers to ble_conn_state.o(.bss) for .bss
    ble_conn_state.o(i.ble_conn_state_for_each_connected) refers to ble_conn_state.o(i.for_each_set_flag) for for_each_set_flag
    ble_conn_state.o(i.ble_conn_state_for_each_connected) refers to ble_conn_state.o(.bss) for .bss
    ble_conn_state.o(i.ble_conn_state_for_each_set_user_flag) refers to ble_conn_state.o(i.user_flag_is_acquired) for user_flag_is_acquired
    ble_conn_state.o(i.ble_conn_state_for_each_set_user_flag) refers to ble_conn_state.o(i.for_each_set_flag) for for_each_set_flag
    ble_conn_state.o(i.ble_conn_state_for_each_set_user_flag) refers to ble_conn_state.o(.bss) for .bss
    ble_conn_state.o(i.ble_conn_state_init) refers to ble_conn_state.o(i.bcs_internal_state_reset) for bcs_internal_state_reset
    ble_conn_state.o(i.ble_conn_state_mitm_protected) refers to ble_conn_state.o(i.ble_conn_state_valid) for ble_conn_state_valid
    ble_conn_state.o(i.ble_conn_state_mitm_protected) refers to nrf_atflags.o(i.nrf_atflags_get) for nrf_atflags_get
    ble_conn_state.o(i.ble_conn_state_mitm_protected) refers to ble_conn_state.o(.bss) for .bss
    ble_conn_state.o(i.ble_conn_state_periph_handles) refers to nrf_atomic.o(i.nrf_atomic_u32_and) for nrf_atomic_u32_and
    ble_conn_state.o(i.ble_conn_state_periph_handles) refers to ble_conn_state.o(i.conn_handle_list_get) for conn_handle_list_get
    ble_conn_state.o(i.ble_conn_state_periph_handles) refers to ble_conn_state.o(.bss) for .bss
    ble_conn_state.o(i.ble_conn_state_peripheral_conn_count) refers to nrf_atomic.o(i.nrf_atomic_u32_and) for nrf_atomic_u32_and
    ble_conn_state.o(i.ble_conn_state_peripheral_conn_count) refers to ble_conn_state.o(i.active_flag_count) for active_flag_count
    ble_conn_state.o(i.ble_conn_state_peripheral_conn_count) refers to ble_conn_state.o(.bss) for .bss
    ble_conn_state.o(i.ble_conn_state_role) refers to ble_conn_state.o(i.ble_conn_state_valid) for ble_conn_state_valid
    ble_conn_state.o(i.ble_conn_state_status) refers to ble_conn_state.o(i.ble_conn_state_valid) for ble_conn_state_valid
    ble_conn_state.o(i.ble_conn_state_status) refers to nrf_atflags.o(i.nrf_atflags_get) for nrf_atflags_get
    ble_conn_state.o(i.ble_conn_state_status) refers to ble_conn_state.o(.bss) for .bss
    ble_conn_state.o(i.ble_conn_state_user_flag_acquire) refers to nrf_atflags.o(i.nrf_atflags_find_and_set_flag) for nrf_atflags_find_and_set_flag
    ble_conn_state.o(i.ble_conn_state_user_flag_acquire) refers to ble_conn_state.o(.bss) for .bss
    ble_conn_state.o(i.ble_conn_state_user_flag_get) refers to ble_conn_state.o(i.user_flag_is_acquired) for user_flag_is_acquired
    ble_conn_state.o(i.ble_conn_state_user_flag_get) refers to ble_conn_state.o(i.ble_conn_state_valid) for ble_conn_state_valid
    ble_conn_state.o(i.ble_conn_state_user_flag_get) refers to nrf_atflags.o(i.nrf_atflags_get) for nrf_atflags_get
    ble_conn_state.o(i.ble_conn_state_user_flag_get) refers to ble_conn_state.o(.bss) for .bss
    ble_conn_state.o(i.ble_conn_state_user_flag_set) refers to ble_conn_state.o(i.user_flag_is_acquired) for user_flag_is_acquired
    ble_conn_state.o(i.ble_conn_state_user_flag_set) refers to ble_conn_state.o(i.ble_conn_state_valid) for ble_conn_state_valid
    ble_conn_state.o(i.ble_conn_state_user_flag_set) refers to nrf_atflags.o(i.nrf_atflags_set) for nrf_atflags_set
    ble_conn_state.o(i.ble_conn_state_user_flag_set) refers to nrf_atflags.o(i.nrf_atflags_clear) for nrf_atflags_clear
    ble_conn_state.o(i.ble_conn_state_user_flag_set) refers to ble_conn_state.o(.bss) for .bss
    ble_conn_state.o(i.ble_conn_state_valid) refers to nrf_atflags.o(i.nrf_atflags_get) for nrf_atflags_get
    ble_conn_state.o(i.ble_conn_state_valid) refers to ble_conn_state.o(.bss) for .bss
    ble_conn_state.o(i.ble_evt_handler) refers to nrf_atomic.o(i.nrf_atomic_u32_and) for nrf_atomic_u32_and
    ble_conn_state.o(i.ble_evt_handler) refers to ble_conn_state.o(i.conn_handle_list_get) for conn_handle_list_get
    ble_conn_state.o(i.ble_evt_handler) refers to memcpya.o(.text) for __aeabi_memcpy4
    ble_conn_state.o(i.ble_evt_handler) refers to nrf_atflags.o(i.nrf_atflags_clear) for nrf_atflags_clear
    ble_conn_state.o(i.ble_evt_handler) refers to app_error.o(i.app_error_handler_bare) for app_error_handler_bare
    ble_conn_state.o(i.ble_evt_handler) refers to nrf_atflags.o(i.nrf_atflags_set) for nrf_atflags_set
    ble_conn_state.o(i.ble_evt_handler) refers to ble_conn_state.o(.bss) for .bss
    ble_conn_state.o(i.conn_handle_list_get) refers to nrf_atflags.o(i.nrf_atflags_get) for nrf_atflags_get
    ble_conn_state.o(i.conn_handle_list_get) refers to memcpya.o(.text) for __aeabi_memcpy4
    ble_conn_state.o(i.for_each_set_flag) refers to nrf_atflags.o(i.nrf_atflags_get) for nrf_atflags_get
    ble_conn_state.o(i.user_flag_is_acquired) refers to nrf_atflags.o(i.nrf_atflags_get) for nrf_atflags_get
    ble_conn_state.o(i.user_flag_is_acquired) refers to ble_conn_state.o(.bss) for .bss
    ble_conn_state.o(sdh_ble_observers0) refers to ble_conn_state.o(i.ble_evt_handler) for ble_evt_handler
    ble_link_ctx_manager.o(i.blcm_link_ctx_get) refers to ble_conn_state.o(i.ble_conn_state_conn_idx) for ble_conn_state_conn_idx
    ble_srv_common.o(i.ble_srv_ascii_to_utf8) refers to strlen.o(.text) for strlen
    ble_srv_common.o(i.characteristic_add) refers to ble_srv_common.o(i.set_security_req) for set_security_req
    ble_srv_common.o(i.characteristic_add) refers to memseta.o(.text) for __aeabi_memclr4
    ble_srv_common.o(i.descriptor_add) refers to memseta.o(.text) for __aeabi_memclr4
    ble_srv_common.o(i.descriptor_add) refers to ble_srv_common.o(i.set_security_req) for set_security_req
    nrf_ble_gatt.o(i.nrf_ble_gatt_init) refers to nrf_ble_gatt.o(i.link_init) for link_init
    nrf_ble_gatt.o(i.nrf_ble_gatt_on_ble_evt) refers to nrf_ble_gatt.o(i.on_connected_evt) for on_connected_evt
    nrf_ble_gatt.o(i.nrf_ble_gatt_on_ble_evt) refers to nrf_ble_gatt.o(i.link_init) for link_init
    nrf_ble_gatt.o(i.nrf_ble_gatt_on_ble_evt) refers to nrf_ble_gatt.o(i.on_exchange_mtu_request_evt) for on_exchange_mtu_request_evt
    nrf_ble_gatt.o(i.nrf_ble_gatt_on_ble_evt) refers to nrf_strerror.o(i.nrf_strerror_get) for nrf_strerror_get
    nrf_ble_gatt.o(i.nrf_ble_gatt_on_ble_evt) refers to nrf_log_frontend.o(i.nrf_log_frontend_std_1) for nrf_log_frontend_std_1
    nrf_ble_gatt.o(i.nrf_ble_gatt_on_ble_evt) refers to nrf_ble_gatt.o(.constdata) for .constdata
    nrf_ble_gatt.o(i.nrf_ble_gatt_on_ble_evt) refers to nrf_ble_gatt.o(log_const_data) for log_const_data
    nrf_ble_gatt.o(i.on_connected_evt) refers to nrf_strerror.o(i.nrf_strerror_get) for nrf_strerror_get
    nrf_ble_gatt.o(i.on_connected_evt) refers to nrf_log_frontend.o(i.nrf_log_frontend_std_1) for nrf_log_frontend_std_1
    nrf_ble_gatt.o(i.on_connected_evt) refers to nrf_ble_gatt.o(log_const_data) for log_const_data
    nrf_ble_gatt.o(i.on_exchange_mtu_request_evt) refers to nrf_strerror.o(i.nrf_strerror_get) for nrf_strerror_get
    nrf_ble_gatt.o(i.on_exchange_mtu_request_evt) refers to nrf_log_frontend.o(i.nrf_log_frontend_std_1) for nrf_log_frontend_std_1
    nrf_ble_gatt.o(i.on_exchange_mtu_request_evt) refers to nrf_ble_gatt.o(log_const_data) for log_const_data
    nrf_ble_gatt.o(i.on_exchange_mtu_request_evt) refers to nrf_ble_gatt.o(.constdata) for .constdata
    nrf_ble_gatt.o(log_const_data) refers to nrf_ble_gatt.o(.conststrlit) for .conststrlit
    nrf_ble_qwr.o(i.nrf_ble_qwr_on_ble_evt) refers to nrf_ble_qwr.o(i.user_mem_reply) for user_mem_reply
    ble_nus.o(i.ble_nus_data_send) refers to ble_link_ctx_manager.o(i.blcm_link_ctx_get) for blcm_link_ctx_get
    ble_nus.o(i.ble_nus_init) refers to memseta.o(.text) for __aeabi_memclr4
    ble_nus.o(i.ble_nus_init) refers to ble_srv_common.o(i.characteristic_add) for characteristic_add
    ble_nus.o(i.ble_nus_init) refers to ble_nus.o(.constdata) for .constdata
    ble_nus.o(i.ble_nus_on_ble_evt) refers to ble_link_ctx_manager.o(i.blcm_link_ctx_get) for blcm_link_ctx_get
    ble_nus.o(i.ble_nus_on_ble_evt) refers to memseta.o(.text) for __aeabi_memclr4
    ble_nus.o(i.ble_nus_on_ble_evt) refers to ble_nus.o(i.on_connect) for on_connect
    ble_nus.o(i.ble_nus_on_ble_evt) refers to ble_nus.o(i.on_write) for on_write
    ble_nus.o(i.on_connect) refers to ble_link_ctx_manager.o(i.blcm_link_ctx_get) for blcm_link_ctx_get
    ble_nus.o(i.on_connect) refers to ble_srv_common.o(i.ble_srv_is_notification_enabled) for ble_srv_is_notification_enabled
    ble_nus.o(i.on_connect) refers to memseta.o(.text) for __aeabi_memclr4
    ble_nus.o(i.on_write) refers to ble_link_ctx_manager.o(i.blcm_link_ctx_get) for blcm_link_ctx_get
    ble_nus.o(i.on_write) refers to memseta.o(.text) for __aeabi_memclr4
    ble_nus.o(i.on_write) refers to ble_srv_common.o(i.ble_srv_is_notification_enabled) for ble_srv_is_notification_enabled
    ble_nus.o(log_const_data) refers to ble_nus.o(.conststrlit) for .conststrlit
    nrf_drv_clock.o(i.clock_clk_started_notify) refers to nrf_drv_clock.o(.bss) for .bss
    nrf_drv_clock.o(i.clock_irq_handler) refers to nrf_drv_clock.o(i.clock_clk_started_notify) for clock_clk_started_notify
    nrf_drv_clock.o(i.clock_irq_handler) refers to nrf_drv_clock.o(.bss) for .bss
    nrf_drv_clock.o(i.nrf_drv_clock_hfclk_is_running) refers to nrf_sdh.o(i.nrf_sdh_is_enabled) for nrf_sdh_is_enabled
    nrf_drv_clock.o(i.nrf_drv_clock_hfclk_release) refers to app_util_platform.o(i.app_util_critical_region_enter) for app_util_critical_region_enter
    nrf_drv_clock.o(i.nrf_drv_clock_hfclk_release) refers to nrf_sdh.o(i.nrf_sdh_is_enabled) for nrf_sdh_is_enabled
    nrf_drv_clock.o(i.nrf_drv_clock_hfclk_release) refers to nrfx_clock.o(i.nrfx_clock_hfclk_stop) for nrfx_clock_hfclk_stop
    nrf_drv_clock.o(i.nrf_drv_clock_hfclk_release) refers to app_util_platform.o(i.app_util_critical_region_exit) for app_util_critical_region_exit
    nrf_drv_clock.o(i.nrf_drv_clock_hfclk_release) refers to nrf_drv_clock.o(.bss) for .bss
    nrf_drv_clock.o(i.nrf_drv_clock_hfclk_request) refers to app_util_platform.o(i.app_util_critical_region_enter) for app_util_critical_region_enter
    nrf_drv_clock.o(i.nrf_drv_clock_hfclk_request) refers to nrf_drv_clock.o(i.item_enqueue) for item_enqueue
    nrf_drv_clock.o(i.nrf_drv_clock_hfclk_request) refers to nrf_sdh.o(i.nrf_sdh_is_enabled) for nrf_sdh_is_enabled
    nrf_drv_clock.o(i.nrf_drv_clock_hfclk_request) refers to nrfx_clock.o(i.nrfx_clock_hfclk_start) for nrfx_clock_hfclk_start
    nrf_drv_clock.o(i.nrf_drv_clock_hfclk_request) refers to app_util_platform.o(i.app_util_critical_region_exit) for app_util_critical_region_exit
    nrf_drv_clock.o(i.nrf_drv_clock_hfclk_request) refers to nrf_drv_clock.o(.bss) for .bss
    nrf_drv_clock.o(i.nrf_drv_clock_init) refers to nrfx_clock.o(i.nrfx_clock_init) for nrfx_clock_init
    nrf_drv_clock.o(i.nrf_drv_clock_init) refers to nrf_sdh.o(i.nrf_sdh_is_enabled) for nrf_sdh_is_enabled
    nrf_drv_clock.o(i.nrf_drv_clock_init) refers to nrfx_clock.o(i.nrfx_clock_enable) for nrfx_clock_enable
    nrf_drv_clock.o(i.nrf_drv_clock_init) refers to nrf_drv_clock.o(.bss) for .bss
    nrf_drv_clock.o(i.nrf_drv_clock_init) refers to nrf_drv_clock.o(i.clock_irq_handler) for clock_irq_handler
    nrf_drv_clock.o(i.nrf_drv_clock_init_check) refers to nrf_drv_clock.o(.bss) for .bss
    nrf_drv_clock.o(i.nrf_drv_clock_lfclk_is_running) refers to nrf_sdh.o(i.nrf_sdh_is_enabled) for nrf_sdh_is_enabled
    nrf_drv_clock.o(i.nrf_drv_clock_lfclk_release) refers to app_util_platform.o(i.app_util_critical_region_enter) for app_util_critical_region_enter
    nrf_drv_clock.o(i.nrf_drv_clock_lfclk_release) refers to nrfx_clock.o(i.nrfx_clock_lfclk_stop) for nrfx_clock_lfclk_stop
    nrf_drv_clock.o(i.nrf_drv_clock_lfclk_release) refers to app_util_platform.o(i.app_util_critical_region_exit) for app_util_critical_region_exit
    nrf_drv_clock.o(i.nrf_drv_clock_lfclk_release) refers to nrf_drv_clock.o(.bss) for .bss
    nrf_drv_clock.o(i.nrf_drv_clock_lfclk_request) refers to app_util_platform.o(i.app_util_critical_region_enter) for app_util_critical_region_enter
    nrf_drv_clock.o(i.nrf_drv_clock_lfclk_request) refers to nrf_drv_clock.o(i.item_enqueue) for item_enqueue
    nrf_drv_clock.o(i.nrf_drv_clock_lfclk_request) refers to nrfx_clock.o(i.nrfx_clock_lfclk_start) for nrfx_clock_lfclk_start
    nrf_drv_clock.o(i.nrf_drv_clock_lfclk_request) refers to app_util_platform.o(i.app_util_critical_region_exit) for app_util_critical_region_exit
    nrf_drv_clock.o(i.nrf_drv_clock_lfclk_request) refers to nrf_drv_clock.o(.bss) for .bss
    nrf_drv_clock.o(i.nrf_drv_clock_uninit) refers to nrfx_clock.o(i.nrfx_clock_disable) for nrfx_clock_disable
    nrf_drv_clock.o(i.nrf_drv_clock_uninit) refers to nrfx_clock.o(i.nrfx_clock_uninit) for nrfx_clock_uninit
    nrf_drv_clock.o(i.nrf_drv_clock_uninit) refers to nrf_drv_clock.o(.bss) for .bss
    nrf_drv_clock.o(i.sd_state_evt_handler) refers to nrfx_clock.o(i.nrfx_clock_enable) for nrfx_clock_enable
    nrf_drv_clock.o(i.sd_state_evt_handler) refers to nrf_drv_clock.o(i.nrf_drv_clock_lfclk_release) for nrf_drv_clock_lfclk_release
    nrf_drv_clock.o(i.sd_state_evt_handler) refers to app_util_platform.o(i.app_util_critical_region_enter) for app_util_critical_region_enter
    nrf_drv_clock.o(i.sd_state_evt_handler) refers to nrf_drv_clock.o(i.nrf_drv_clock_init) for nrf_drv_clock_init
    nrf_drv_clock.o(i.sd_state_evt_handler) refers to app_util_platform.o(i.app_util_critical_region_exit) for app_util_critical_region_exit
    nrf_drv_clock.o(i.sd_state_evt_handler) refers to nrf_drv_clock.o(.bss) for .bss
    nrf_drv_clock.o(i.soc_evt_handler) refers to nrf_drv_clock.o(i.clock_clk_started_notify) for clock_clk_started_notify
    nrf_drv_clock.o(i.soc_evt_handler) refers to nrf_drv_clock.o(.bss) for .bss
    nrf_drv_clock.o(log_const_data) refers to nrf_drv_clock.o(.conststrlit) for .conststrlit
    nrf_drv_clock.o(sdh_soc_observers0) refers to nrf_drv_clock.o(i.soc_evt_handler) for soc_evt_handler
    nrf_drv_clock.o(sdh_state_observers0) refers to nrf_drv_clock.o(i.sd_state_evt_handler) for sd_state_evt_handler
    nrf_drv_uart.o(i.nrf_drv_uart_init) refers to memcpya.o(.text) for __aeabi_memcpy4
    nrf_drv_uart.o(i.nrf_drv_uart_init) refers to nrfx_uarte.o(i.nrfx_uarte_init) for nrfx_uarte_init
    nrf_drv_uart.o(i.nrf_drv_uart_init) refers to nrf_drv_uart.o(.data) for .data
    nrf_drv_uart.o(i.nrf_drv_uart_init) refers to nrf_drv_uart.o(i.uarte_evt_handler) for uarte_evt_handler
    nrf_drv_uart.o(i.uarte_evt_handler) refers to nrf_drv_uart.o(.data) for .data
    nrfx_clock.o(i.POWER_CLOCK_IRQHandler) refers to nrfx_clock.o(i.nrf_clock_event_check) for nrf_clock_event_check
    nrfx_clock.o(i.POWER_CLOCK_IRQHandler) refers to nrfx_clock.o(i.nrf_clock_event_clear) for nrf_clock_event_clear
    nrfx_clock.o(i.POWER_CLOCK_IRQHandler) refers to nrfx_clock.o(.data) for .data
    nrfx_clock.o(i.nrfx_clock_calibration_timer_start) refers to nrfx_clock.o(i.nrf_clock_event_clear) for nrf_clock_event_clear
    nrfx_clock.o(i.nrfx_clock_hfclk_start) refers to nrfx_clock.o(i.nrf_clock_event_clear) for nrf_clock_event_clear
    nrfx_clock.o(i.nrfx_clock_hfclk_stop) refers to nrfx_clock.o(.data) for .data
    nrfx_clock.o(i.nrfx_clock_init) refers to nrfx_clock.o(.data) for .data
    nrfx_clock.o(i.nrfx_clock_lfclk_start) refers to nrfx_clock.o(i.nrf_clock_event_clear) for nrf_clock_event_clear
    nrfx_clock.o(i.nrfx_clock_uninit) refers to nrfx_clock.o(i.nrfx_clock_lfclk_stop) for nrfx_clock_lfclk_stop
    nrfx_clock.o(i.nrfx_clock_uninit) refers to nrfx_clock.o(i.nrfx_clock_hfclk_stop) for nrfx_clock_hfclk_stop
    nrfx_clock.o(i.nrfx_clock_uninit) refers to nrfx_clock.o(.data) for .data
    nrfx_clock.o(log_const_data) refers to nrfx_clock.o(.conststrlit) for .conststrlit
    nrfx_gpiote.o(i.GPIOTE_IRQHandler) refers to nrfx_gpiote.o(i.nrf_gpiote_event_is_set) for nrf_gpiote_event_is_set
    nrfx_gpiote.o(i.GPIOTE_IRQHandler) refers to nrfx_gpiote.o(i.nrf_gpiote_event_clear) for nrf_gpiote_event_clear
    nrfx_gpiote.o(i.GPIOTE_IRQHandler) refers to nrfx_gpiote.o(i.nrf_gpio_ports_read) for nrf_gpio_ports_read
    nrfx_gpiote.o(i.GPIOTE_IRQHandler) refers to nrfx_gpiote.o(i.nrf_bitmask_bit_is_set) for nrf_bitmask_bit_is_set
    nrfx_gpiote.o(i.GPIOTE_IRQHandler) refers to nrfx_gpiote.o(i.channel_port_get) for channel_port_get
    nrfx_gpiote.o(i.GPIOTE_IRQHandler) refers to nrfx_gpiote.o(i.nrf_bitmask_bit_set) for nrf_bitmask_bit_set
    nrfx_gpiote.o(i.GPIOTE_IRQHandler) refers to nrfx_gpiote.o(i.nrf_gpio_cfg_sense_set) for nrf_gpio_cfg_sense_set
    nrfx_gpiote.o(i.GPIOTE_IRQHandler) refers to nrfx_gpiote.o(.bss) for .bss
    nrfx_gpiote.o(i.channel_free) refers to nrfx_gpiote.o(.bss) for .bss
    nrfx_gpiote.o(i.channel_port_alloc) refers to nrfx_gpiote.o(.bss) for .bss
    nrfx_gpiote.o(i.channel_port_get) refers to nrfx_gpiote.o(.bss) for .bss
    nrfx_gpiote.o(i.nrf_gpio_cfg_default) refers to nrfx_gpiote.o(i.nrf_gpio_cfg) for nrf_gpio_cfg
    nrfx_gpiote.o(i.nrf_gpio_ports_read) refers to nrfx_gpiote.o(.constdata) for .constdata
    nrfx_gpiote.o(i.nrfx_gpiote_clr_task_addr_get) refers to nrfx_gpiote.o(i.channel_port_get) for channel_port_get
    nrfx_gpiote.o(i.nrfx_gpiote_clr_task_trigger) refers to nrfx_gpiote.o(i.channel_port_get) for channel_port_get
    nrfx_gpiote.o(i.nrfx_gpiote_in_event_addr_get) refers to nrfx_gpiote.o(i.pin_in_use_by_te) for pin_in_use_by_te
    nrfx_gpiote.o(i.nrfx_gpiote_in_event_addr_get) refers to nrfx_gpiote.o(i.channel_port_get) for channel_port_get
    nrfx_gpiote.o(i.nrfx_gpiote_in_event_disable) refers to nrfx_gpiote.o(i.pin_in_use_by_port) for pin_in_use_by_port
    nrfx_gpiote.o(i.nrfx_gpiote_in_event_disable) refers to nrfx_gpiote.o(i.nrf_gpio_cfg_sense_set) for nrf_gpio_cfg_sense_set
    nrfx_gpiote.o(i.nrfx_gpiote_in_event_disable) refers to nrfx_gpiote.o(i.pin_in_use_by_te) for pin_in_use_by_te
    nrfx_gpiote.o(i.nrfx_gpiote_in_event_disable) refers to nrfx_gpiote.o(i.channel_port_get) for channel_port_get
    nrfx_gpiote.o(i.nrfx_gpiote_in_event_enable) refers to nrfx_gpiote.o(i.pin_in_use_by_port) for pin_in_use_by_port
    nrfx_gpiote.o(i.nrfx_gpiote_in_event_enable) refers to nrfx_gpiote.o(i.channel_port_get) for channel_port_get
    nrfx_gpiote.o(i.nrfx_gpiote_in_event_enable) refers to nrfx_gpiote.o(i.nrf_gpio_cfg_sense_set) for nrf_gpio_cfg_sense_set
    nrfx_gpiote.o(i.nrfx_gpiote_in_event_enable) refers to nrfx_gpiote.o(i.pin_in_use_by_te) for pin_in_use_by_te
    nrfx_gpiote.o(i.nrfx_gpiote_in_event_enable) refers to nrfx_gpiote.o(i.nrf_gpiote_event_clear) for nrf_gpiote_event_clear
    nrfx_gpiote.o(i.nrfx_gpiote_in_event_enable) refers to nrfx_gpiote.o(.bss) for .bss
    nrfx_gpiote.o(i.nrfx_gpiote_in_init) refers to nrfx_gpiote.o(i.channel_port_alloc) for channel_port_alloc
    nrfx_gpiote.o(i.nrfx_gpiote_in_init) refers to nrfx_gpiote.o(i.nrf_gpio_cfg) for nrf_gpio_cfg
    nrfx_gpiote.o(i.nrfx_gpiote_in_init) refers to nrfx_gpiote.o(i.nrf_bitmask_bit_set) for nrf_bitmask_bit_set
    nrfx_gpiote.o(i.nrfx_gpiote_in_init) refers to nrfx_gpiote.o(.bss) for .bss
    nrfx_gpiote.o(i.nrfx_gpiote_in_uninit) refers to nrfx_gpiote.o(i.nrfx_gpiote_in_event_disable) for nrfx_gpiote_in_event_disable
    nrfx_gpiote.o(i.nrfx_gpiote_in_uninit) refers to nrfx_gpiote.o(i.pin_in_use_by_te) for pin_in_use_by_te
    nrfx_gpiote.o(i.nrfx_gpiote_in_uninit) refers to nrfx_gpiote.o(i.channel_port_get) for channel_port_get
    nrfx_gpiote.o(i.nrfx_gpiote_in_uninit) refers to nrfx_gpiote.o(i.pin_configured_check) for pin_configured_check
    nrfx_gpiote.o(i.nrfx_gpiote_in_uninit) refers to nrfx_gpiote.o(i.nrf_gpio_cfg_default) for nrf_gpio_cfg_default
    nrfx_gpiote.o(i.nrfx_gpiote_in_uninit) refers to nrfx_gpiote.o(i.pin_configured_clear) for pin_configured_clear
    nrfx_gpiote.o(i.nrfx_gpiote_in_uninit) refers to nrfx_gpiote.o(i.channel_free) for channel_free
    nrfx_gpiote.o(i.nrfx_gpiote_in_uninit) refers to nrfx_gpiote.o(.bss) for .bss
    nrfx_gpiote.o(i.nrfx_gpiote_init) refers to nrfx_gpiote.o(i.channel_free) for channel_free
    nrfx_gpiote.o(i.nrfx_gpiote_init) refers to nrfx_gpiote.o(i.nrf_gpiote_event_clear) for nrf_gpiote_event_clear
    nrfx_gpiote.o(i.nrfx_gpiote_init) refers to nrfx_gpiote.o(.bss) for .bss
    nrfx_gpiote.o(i.nrfx_gpiote_is_init) refers to nrfx_gpiote.o(.bss) for .bss
    nrfx_gpiote.o(i.nrfx_gpiote_out_init) refers to nrfx_gpiote.o(i.channel_port_alloc) for channel_port_alloc
    nrfx_gpiote.o(i.nrfx_gpiote_out_init) refers to nrfx_gpiote.o(i.nrf_gpio_cfg) for nrf_gpio_cfg
    nrfx_gpiote.o(i.nrfx_gpiote_out_init) refers to nrfx_gpiote.o(i.nrf_bitmask_bit_set) for nrf_bitmask_bit_set
    nrfx_gpiote.o(i.nrfx_gpiote_out_init) refers to nrfx_gpiote.o(.bss) for .bss
    nrfx_gpiote.o(i.nrfx_gpiote_out_task_addr_get) refers to nrfx_gpiote.o(i.channel_port_get) for channel_port_get
    nrfx_gpiote.o(i.nrfx_gpiote_out_task_disable) refers to nrfx_gpiote.o(.bss) for .bss
    nrfx_gpiote.o(i.nrfx_gpiote_out_task_enable) refers to nrfx_gpiote.o(.bss) for .bss
    nrfx_gpiote.o(i.nrfx_gpiote_out_task_force) refers to nrfx_gpiote.o(.bss) for .bss
    nrfx_gpiote.o(i.nrfx_gpiote_out_task_trigger) refers to nrfx_gpiote.o(i.channel_port_get) for channel_port_get
    nrfx_gpiote.o(i.nrfx_gpiote_out_uninit) refers to nrfx_gpiote.o(i.pin_in_use_by_te) for pin_in_use_by_te
    nrfx_gpiote.o(i.nrfx_gpiote_out_uninit) refers to nrfx_gpiote.o(i.channel_port_get) for channel_port_get
    nrfx_gpiote.o(i.nrfx_gpiote_out_uninit) refers to nrfx_gpiote.o(i.channel_free) for channel_free
    nrfx_gpiote.o(i.nrfx_gpiote_out_uninit) refers to nrfx_gpiote.o(i.pin_configured_check) for pin_configured_check
    nrfx_gpiote.o(i.nrfx_gpiote_out_uninit) refers to nrfx_gpiote.o(i.nrf_gpio_cfg_default) for nrf_gpio_cfg_default
    nrfx_gpiote.o(i.nrfx_gpiote_out_uninit) refers to nrfx_gpiote.o(i.pin_configured_clear) for pin_configured_clear
    nrfx_gpiote.o(i.nrfx_gpiote_out_uninit) refers to nrfx_gpiote.o(.bss) for .bss
    nrfx_gpiote.o(i.nrfx_gpiote_set_task_addr_get) refers to nrfx_gpiote.o(i.channel_port_get) for channel_port_get
    nrfx_gpiote.o(i.nrfx_gpiote_set_task_trigger) refers to nrfx_gpiote.o(i.channel_port_get) for channel_port_get
    nrfx_gpiote.o(i.nrfx_gpiote_uninit) refers to nrfx_gpiote.o(i.nrfx_gpiote_in_uninit) for nrfx_gpiote_in_uninit
    nrfx_gpiote.o(i.nrfx_gpiote_uninit) refers to nrfx_gpiote.o(i.nrfx_gpiote_out_uninit) for nrfx_gpiote_out_uninit
    nrfx_gpiote.o(i.nrfx_gpiote_uninit) refers to nrfx_gpiote.o(.bss) for .bss
    nrfx_gpiote.o(i.pin_configured_check) refers to nrfx_gpiote.o(i.nrf_bitmask_bit_is_set) for nrf_bitmask_bit_is_set
    nrfx_gpiote.o(i.pin_configured_check) refers to nrfx_gpiote.o(.bss) for .bss
    nrfx_gpiote.o(i.pin_configured_clear) refers to nrfx_gpiote.o(.bss) for .bss
    nrfx_gpiote.o(i.pin_in_use_by_port) refers to nrfx_gpiote.o(.bss) for .bss
    nrfx_gpiote.o(i.pin_in_use_by_te) refers to nrfx_gpiote.o(.bss) for .bss
    nrfx_gpiote.o(log_const_data) refers to nrfx_gpiote.o(.conststrlit) for .conststrlit
    nrfx_prs.o(log_const_data) refers to nrfx_prs.o(.conststrlit) for .conststrlit
    nrfx_uarte.o(i.UARTE0_IRQHandler) refers to nrfx_uarte.o(i.uarte_irq_handler) for uarte_irq_handler
    nrfx_uarte.o(i.UARTE0_IRQHandler) refers to nrfx_uarte.o(.bss) for .bss
    nrfx_uarte.o(i.apply_config) refers to nrfx_uarte.o(i.nrf_gpio_cfg_output) for nrf_gpio_cfg_output
    nrfx_uarte.o(i.apply_config) refers to nrfx_uarte.o(i.nrf_gpio_cfg_input) for nrf_gpio_cfg_input
    nrfx_uarte.o(i.interrupts_enable) refers to nrfx_uarte.o(i.nrf_uarte_event_clear) for nrf_uarte_event_clear
    nrfx_uarte.o(i.nrf_gpio_cfg_default) refers to nrfx_uarte.o(i.nrf_gpio_cfg) for nrf_gpio_cfg
    nrfx_uarte.o(i.nrf_gpio_cfg_input) refers to nrfx_uarte.o(i.nrf_gpio_cfg) for nrf_gpio_cfg
    nrfx_uarte.o(i.nrf_gpio_cfg_output) refers to nrfx_uarte.o(i.nrf_gpio_cfg) for nrf_gpio_cfg
    nrfx_uarte.o(i.nrfx_uarte_errorsrc_get) refers to nrfx_uarte.o(i.nrf_uarte_event_clear) for nrf_uarte_event_clear
    nrfx_uarte.o(i.nrfx_uarte_init) refers to nrfx_prs.o(i.nrfx_prs_acquire) for nrfx_prs_acquire
    nrfx_uarte.o(i.nrfx_uarte_init) refers to nrfx_uarte.o(i.apply_config) for apply_config
    nrfx_uarte.o(i.nrfx_uarte_init) refers to nrfx_uarte.o(i.interrupts_enable) for interrupts_enable
    nrfx_uarte.o(i.nrfx_uarte_init) refers to nrfx_uarte.o(.bss) for .bss
    nrfx_uarte.o(i.nrfx_uarte_init) refers to nrfx_uarte.o(.constdata) for .constdata
    nrfx_uarte.o(i.nrfx_uarte_rx) refers to nrfx_uarte.o(i.nrfx_is_in_ram) for nrfx_is_in_ram
    nrfx_uarte.o(i.nrfx_uarte_rx) refers to nrfx_uarte.o(i.nrf_uarte_event_clear) for nrf_uarte_event_clear
    nrfx_uarte.o(i.nrfx_uarte_rx) refers to nrfx_uarte.o(i.nrf_uarte_event_check) for nrf_uarte_event_check
    nrfx_uarte.o(i.nrfx_uarte_rx) refers to nrfx_uarte.o(.bss) for .bss
    nrfx_uarte.o(i.nrfx_uarte_tx) refers to nrfx_uarte.o(i.nrfx_is_in_ram) for nrfx_is_in_ram
    nrfx_uarte.o(i.nrfx_uarte_tx) refers to nrfx_uarte.o(i.nrfx_uarte_tx_in_progress) for nrfx_uarte_tx_in_progress
    nrfx_uarte.o(i.nrfx_uarte_tx) refers to nrfx_uarte.o(i.nrf_uarte_event_clear) for nrf_uarte_event_clear
    nrfx_uarte.o(i.nrfx_uarte_tx) refers to nrfx_uarte.o(i.nrf_uarte_event_check) for nrf_uarte_event_check
    nrfx_uarte.o(i.nrfx_uarte_tx) refers to nrfx_uarte.o(.bss) for .bss
    nrfx_uarte.o(i.nrfx_uarte_tx_abort) refers to nrfx_uarte.o(i.nrf_uarte_event_clear) for nrf_uarte_event_clear
    nrfx_uarte.o(i.nrfx_uarte_tx_abort) refers to nrfx_uarte.o(i.nrf_uarte_event_check) for nrf_uarte_event_check
    nrfx_uarte.o(i.nrfx_uarte_tx_abort) refers to nrfx_uarte.o(.bss) for .bss
    nrfx_uarte.o(i.nrfx_uarte_tx_in_progress) refers to nrfx_uarte.o(.bss) for .bss
    nrfx_uarte.o(i.nrfx_uarte_uninit) refers to nrfx_uarte.o(i.nrf_gpio_cfg_default) for nrf_gpio_cfg_default
    nrfx_uarte.o(i.nrfx_uarte_uninit) refers to nrfx_prs.o(i.nrfx_prs_release) for nrfx_prs_release
    nrfx_uarte.o(i.nrfx_uarte_uninit) refers to nrfx_uarte.o(.bss) for .bss
    nrfx_uarte.o(i.uarte_irq_handler) refers to nrfx_uarte.o(i.nrf_uarte_event_check) for nrf_uarte_event_check
    nrfx_uarte.o(i.uarte_irq_handler) refers to nrfx_uarte.o(i.nrf_uarte_event_clear) for nrf_uarte_event_clear
    nrfx_uarte.o(i.uarte_irq_handler) refers to nrfx_uarte.o(i.rx_done_event) for rx_done_event
    nrfx_uarte.o(.constdata) refers to nrfx_uarte.o(i.UARTE0_IRQHandler) for UARTE0_IRQHandler
    nrfx_uarte.o(log_const_data) refers to nrfx_uarte.o(.conststrlit) for .conststrlit
    nrfx_twim.o(i.TWIM0_TWIS0_IRQHandler) refers to nrfx_twim.o(i.twim_irq_handler) for twim_irq_handler
    nrfx_twim.o(i.TWIM0_TWIS0_IRQHandler) refers to nrfx_twim.o(.bss) for .bss
    nrfx_twim.o(i.nrf_gpio_cfg_default) refers to nrfx_twim.o(i.nrf_gpio_cfg) for nrf_gpio_cfg
    nrfx_twim.o(i.nrfx_twim_disable) refers to nrfx_twim.o(.bss) for .bss
    nrfx_twim.o(i.nrfx_twim_enable) refers to nrfx_twim.o(.bss) for .bss
    nrfx_twim.o(i.nrfx_twim_init) refers to nrfx_prs.o(i.nrfx_prs_acquire) for nrfx_prs_acquire
    nrfx_twim.o(i.nrfx_twim_init) refers to nrfx_twim.o(i.nrf_gpio_cfg) for nrf_gpio_cfg
    nrfx_twim.o(i.nrfx_twim_init) refers to nrfx_twim.o(.bss) for .bss
    nrfx_twim.o(i.nrfx_twim_init) refers to nrfx_twim.o(.constdata) for .constdata
    nrfx_twim.o(i.nrfx_twim_is_busy) refers to nrfx_twim.o(.bss) for .bss
    nrfx_twim.o(i.nrfx_twim_rx) refers to memcpya.o(.text) for __aeabi_memcpy4
    nrfx_twim.o(i.nrfx_twim_rx) refers to nrfx_twim.o(i.nrfx_twim_xfer) for nrfx_twim_xfer
    nrfx_twim.o(i.nrfx_twim_rx) refers to nrfx_twim.o(.constdata) for .constdata
    nrfx_twim.o(i.nrfx_twim_tx) refers to memseta.o(.text) for __aeabi_memclr4
    nrfx_twim.o(i.nrfx_twim_tx) refers to nrfx_twim.o(i.nrfx_twim_xfer) for nrfx_twim_xfer
    nrfx_twim.o(i.nrfx_twim_uninit) refers to nrfx_twim.o(i.nrfx_twim_disable) for nrfx_twim_disable
    nrfx_twim.o(i.nrfx_twim_uninit) refers to nrfx_prs.o(i.nrfx_prs_release) for nrfx_prs_release
    nrfx_twim.o(i.nrfx_twim_uninit) refers to nrfx_twim.o(i.nrf_gpio_cfg_default) for nrf_gpio_cfg_default
    nrfx_twim.o(i.nrfx_twim_uninit) refers to nrfx_twim.o(.bss) for .bss
    nrfx_twim.o(i.nrfx_twim_xfer) refers to nrfx_twim.o(i.twim_xfer) for twim_xfer
    nrfx_twim.o(i.nrfx_twim_xfer) refers to nrfx_twim.o(.bss) for .bss
    nrfx_twim.o(i.twim_irq_handler) refers to nrfx_twim.o(i.nrf_twim_event_check) for nrf_twim_event_check
    nrfx_twim.o(i.twim_irq_handler) refers to nrfx_twim.o(i.nrf_twim_event_clear) for nrf_twim_event_clear
    nrfx_twim.o(i.twim_irq_handler) refers to memcpya.o(.text) for __aeabi_memcpy4
    nrfx_twim.o(i.twim_xfer) refers to nrfx_twim.o(i.nrfx_is_in_ram) for nrfx_is_in_ram
    nrfx_twim.o(i.twim_xfer) refers to memcpya.o(.text) for __aeabi_memcpy4
    nrfx_twim.o(i.twim_xfer) refers to nrfx_twim.o(i.nrf_twim_event_clear) for nrf_twim_event_clear
    nrfx_twim.o(i.twim_xfer) refers to nrfx_twim.o(i.nrf_twim_event_check) for nrf_twim_event_check
    nrfx_twim.o(.constdata) refers to nrfx_twim.o(i.TWIM0_TWIS0_IRQHandler) for TWIM0_TWIS0_IRQHandler
    nrfx_twim.o(log_const_data) refers to nrfx_twim.o(.conststrlit) for .conststrlit
    nrf_drv_twi.o(i.nrf_drv_twi_init) refers to nrf_drv_twi.o(i.twi_clear_bus) for twi_clear_bus
    nrf_drv_twi.o(i.nrf_drv_twi_init) refers to nrfx_twim.o(i.nrfx_twim_init) for nrfx_twim_init
    nrf_drv_twi.o(i.nrf_drv_twi_init) refers to nrf_drv_twi.o(.data) for .data
    nrf_drv_twi.o(i.nrf_drv_twi_init) refers to nrf_drv_twi.o(i.twim_evt_handler) for twim_evt_handler
    nrf_drv_twi.o(i.nrfx_coredep_delay_us) refers to nrf_drv_twi.o(.constdata) for .constdata
    nrf_drv_twi.o(i.twi_clear_bus) refers to nrf_drv_twi.o(i.nrf_gpio_pin_set) for nrf_gpio_pin_set
    nrf_drv_twi.o(i.twi_clear_bus) refers to nrf_drv_twi.o(i.nrfx_coredep_delay_us) for nrfx_coredep_delay_us
    nrf_drv_twi.o(i.twim_evt_handler) refers to nrf_drv_twi.o(.data) for .data
    app_button.o(i.app_button_disable) refers to nrfx_gpiote.o(i.nrfx_gpiote_in_event_disable) for nrfx_gpiote_in_event_disable
    app_button.o(i.app_button_disable) refers to app_timer.o(i.app_timer_stop) for app_timer_stop
    app_button.o(i.app_button_disable) refers to app_button.o(.data) for .data
    app_button.o(i.app_button_disable) refers to app_button.o(.constdata) for .constdata
    app_button.o(i.app_button_enable) refers to nrfx_gpiote.o(i.nrfx_gpiote_in_event_enable) for nrfx_gpiote_in_event_enable
    app_button.o(i.app_button_enable) refers to app_button.o(.data) for .data
    app_button.o(i.app_button_init) refers to nrfx_gpiote.o(i.nrfx_gpiote_is_init) for nrfx_gpiote_is_init
    app_button.o(i.app_button_init) refers to nrfx_gpiote.o(i.nrfx_gpiote_init) for nrfx_gpiote_init
    app_button.o(i.app_button_init) refers to nrfx_gpiote.o(i.nrfx_gpiote_in_init) for nrfx_gpiote_in_init
    app_button.o(i.app_button_init) refers to app_timer.o(i.app_timer_create) for app_timer_create
    app_button.o(i.app_button_init) refers to app_button.o(.data) for .data
    app_button.o(i.app_button_init) refers to app_button.o(.constdata) for .constdata
    app_button.o(i.app_button_init) refers to app_button.o(i.gpiote_event_handler) for gpiote_event_handler
    app_button.o(i.app_button_init) refers to app_button.o(i.detection_delay_timeout_handler) for detection_delay_timeout_handler
    app_button.o(i.app_button_is_pushed) refers to nrfx_gpiote.o(i.nrfx_gpiote_in_is_set) for nrfx_gpiote_in_is_set
    app_button.o(i.app_button_is_pushed) refers to app_button.o(.data) for .data
    app_button.o(i.detection_delay_timeout_handler) refers to llshl.o(.text) for __aeabi_llsl
    app_button.o(i.detection_delay_timeout_handler) refers to nrfx_gpiote.o(i.nrfx_gpiote_in_is_set) for nrfx_gpiote_in_is_set
    app_button.o(i.detection_delay_timeout_handler) refers to app_button.o(.data) for .data
    app_button.o(i.gpiote_event_handler) refers to llshl.o(.text) for __aeabi_llsl
    app_button.o(i.gpiote_event_handler) refers to app_timer.o(i.app_timer_stop) for app_timer_stop
    app_button.o(i.gpiote_event_handler) refers to nrfx_gpiote.o(i.nrfx_gpiote_in_is_set) for nrfx_gpiote_in_is_set
    app_button.o(i.gpiote_event_handler) refers to app_timer.o(i.app_timer_start) for app_timer_start
    app_button.o(i.gpiote_event_handler) refers to app_button.o(.constdata) for .constdata
    app_button.o(i.gpiote_event_handler) refers to app_button.o(.data) for .data
    app_button.o(.constdata) refers to app_button.o(.bss) for m_detection_delay_timer_id_data
    app_error.o(i.app_error_handler_bare) refers to app_error_weak.o(i.app_error_fault_handler) for app_error_fault_handler
    app_error.o(i.app_error_save_and_stop) refers to app_error.o(.bss) for .bss
    app_error_handler_keil.o(.emb_text) refers to app_error_weak.o(i.app_error_fault_handler) for app_error_fault_handler
    app_error_weak.o(i.app_error_fault_handler) refers to nrf_log_frontend.o(i.nrf_log_panic) for nrf_log_panic
    app_error_weak.o(i.app_error_fault_handler) refers to nrf_log_frontend.o(i.nrf_log_frontend_dequeue) for nrf_log_frontend_dequeue
    app_error_weak.o(i.app_error_fault_handler) refers to nrf_log_frontend.o(i.nrf_log_frontend_std_0) for nrf_log_frontend_std_0
    app_error_weak.o(i.app_error_fault_handler) refers to nrf_log_frontend.o(log_const_data) for m_nrf_log_app_logs_data_const
    app_fifo.o(i.app_fifo_get) refers to app_fifo.o(i.fifo_get) for fifo_get
    app_fifo.o(i.app_fifo_put) refers to app_fifo.o(i.fifo_put) for fifo_put
    app_fifo.o(i.app_fifo_read) refers to app_fifo.o(i.fifo_get) for fifo_get
    app_fifo.o(i.app_fifo_write) refers to app_fifo.o(i.fifo_put) for fifo_put
    app_scheduler.o(i.app_sched_event_put) refers to app_util_platform.o(i.app_util_critical_region_enter) for app_util_critical_region_enter
    app_scheduler.o(i.app_sched_event_put) refers to app_util_platform.o(i.app_util_critical_region_exit) for app_util_critical_region_exit
    app_scheduler.o(i.app_sched_event_put) refers to memcpya.o(.text) for __aeabi_memcpy
    app_scheduler.o(i.app_sched_event_put) refers to app_scheduler.o(.data) for .data
    app_scheduler.o(i.app_sched_execute) refers to app_scheduler.o(.data) for .data
    app_scheduler.o(i.app_sched_init) refers to app_scheduler.o(.data) for .data
    app_scheduler.o(i.app_sched_queue_space_get) refers to app_scheduler.o(.data) for .data
    app_timer.o(i.RTC1_IRQHandler) refers to app_timer.o(i.timer_timeouts_check) for timer_timeouts_check
    app_timer.o(i.SWI0_EGU0_IRQHandler) refers to app_timer.o(i.timer_list_handler) for timer_list_handler
    app_timer.o(i.app_timer_create) refers to app_timer.o(.bss) for .bss
    app_timer.o(i.app_timer_init) refers to app_timer.o(i.rtc1_stop) for rtc1_stop
    app_timer.o(i.app_timer_init) refers to app_timer.o(i.NVIC_ClearPendingIRQ) for NVIC_ClearPendingIRQ
    app_timer.o(i.app_timer_init) refers to app_timer.o(i.NVIC_SetPriority) for NVIC_SetPriority
    app_timer.o(i.app_timer_init) refers to app_timer.o(i.NVIC_EnableIRQ) for NVIC_EnableIRQ
    app_timer.o(i.app_timer_init) refers to app_timer.o(.bss) for .bss
    app_timer.o(i.app_timer_init) refers to app_timer.o(.data) for .data
    app_timer.o(i.app_timer_start) refers to app_util_platform.o(i.app_util_critical_region_enter) for app_util_critical_region_enter
    app_timer.o(i.app_timer_start) refers to app_timer.o(i.user_op_alloc) for user_op_alloc
    app_timer.o(i.app_timer_start) refers to app_util_platform.o(i.app_util_critical_region_exit) for app_util_critical_region_exit
    app_timer.o(i.app_timer_start) refers to app_timer.o(i.NVIC_SetPendingIRQ) for NVIC_SetPendingIRQ
    app_timer.o(i.app_timer_start) refers to app_timer.o(.bss) for .bss
    app_timer.o(i.app_timer_stop) refers to app_timer.o(i.timer_stop_op_schedule) for timer_stop_op_schedule
    app_timer.o(i.app_timer_stop) refers to app_timer.o(.bss) for .bss
    app_timer.o(i.app_timer_stop_all) refers to app_timer.o(i.timer_stop_op_schedule) for timer_stop_op_schedule
    app_timer.o(i.app_timer_stop_all) refers to app_timer.o(.bss) for .bss
    app_timer.o(i.compare_reg_update) refers to app_timer.o(i.NVIC_ClearPendingIRQ) for NVIC_ClearPendingIRQ
    app_timer.o(i.compare_reg_update) refers to app_timer.o(i.NVIC_EnableIRQ) for NVIC_EnableIRQ
    app_timer.o(i.compare_reg_update) refers to app_timer.o(i.nrfx_coredep_delay_us) for nrfx_coredep_delay_us
    app_timer.o(i.compare_reg_update) refers to app_timer.o(i.NVIC_SetPendingIRQ) for NVIC_SetPendingIRQ
    app_timer.o(i.compare_reg_update) refers to app_timer.o(i.rtc1_stop) for rtc1_stop
    app_timer.o(i.compare_reg_update) refers to app_timer.o(.data) for .data
    app_timer.o(i.elapsed_ticks_acquire) refers to app_timer.o(.data) for .data
    app_timer.o(i.list_insertions_handler) refers to app_timer.o(i.timer_list_remove) for timer_list_remove
    app_timer.o(i.list_insertions_handler) refers to app_timer.o(i.timer_list_insert) for timer_list_insert
    app_timer.o(i.list_insertions_handler) refers to app_timer.o(.data) for .data
    app_timer.o(i.list_insertions_handler) refers to app_timer.o(.bss) for .bss
    app_timer.o(i.nrfx_coredep_delay_us) refers to app_timer.o(.constdata) for .constdata
    app_timer.o(i.rtc1_stop) refers to app_timer.o(i.nrfx_coredep_delay_us) for nrfx_coredep_delay_us
    app_timer.o(i.rtc1_stop) refers to app_timer.o(.data) for .data
    app_timer.o(i.timer_list_handler) refers to app_timer.o(i.elapsed_ticks_acquire) for elapsed_ticks_acquire
    app_timer.o(i.timer_list_handler) refers to app_timer.o(i.list_insertions_handler) for list_insertions_handler
    app_timer.o(i.timer_list_handler) refers to app_timer.o(i.compare_reg_update) for compare_reg_update
    app_timer.o(i.timer_list_handler) refers to app_timer.o(.data) for .data
    app_timer.o(i.timer_list_insert) refers to app_timer.o(.data) for .data
    app_timer.o(i.timer_list_remove) refers to app_timer.o(i.nrfx_coredep_delay_us) for nrfx_coredep_delay_us
    app_timer.o(i.timer_list_remove) refers to app_timer.o(.data) for .data
    app_timer.o(i.timer_stop_op_schedule) refers to app_util_platform.o(i.app_util_critical_region_enter) for app_util_critical_region_enter
    app_timer.o(i.timer_stop_op_schedule) refers to app_timer.o(i.user_op_alloc) for user_op_alloc
    app_timer.o(i.timer_stop_op_schedule) refers to app_util_platform.o(i.app_util_critical_region_exit) for app_util_critical_region_exit
    app_timer.o(i.timer_stop_op_schedule) refers to app_timer.o(i.NVIC_SetPendingIRQ) for NVIC_SetPendingIRQ
    app_timer.o(i.timer_stop_op_schedule) refers to app_timer.o(.bss) for .bss
    app_timer.o(i.timer_timeouts_check) refers to app_timer.o(i.NVIC_SetPendingIRQ) for NVIC_SetPendingIRQ
    app_timer.o(i.timer_timeouts_check) refers to app_timer.o(.data) for .data
    app_timer.o(i.user_op_alloc) refers to app_timer.o(.bss) for .bss
    app_uart_fifo.o(i.app_uart_close) refers to nrfx_uarte.o(i.nrfx_uarte_uninit) for nrfx_uarte_uninit
    app_uart_fifo.o(i.app_uart_close) refers to app_uart_fifo.o(.data) for .data
    app_uart_fifo.o(i.app_uart_flush) refers to app_fifo.o(i.app_fifo_flush) for app_fifo_flush
    app_uart_fifo.o(i.app_uart_flush) refers to app_uart_fifo.o(.bss) for .bss
    app_uart_fifo.o(i.app_uart_get) refers to app_fifo.o(i.app_fifo_get) for app_fifo_get
    app_uart_fifo.o(i.app_uart_get) refers to app_uart_fifo.o(i.nrf_drv_uart_rx) for nrf_drv_uart_rx
    app_uart_fifo.o(i.app_uart_get) refers to app_error.o(i.app_error_handler_bare) for app_error_handler_bare
    app_uart_fifo.o(i.app_uart_get) refers to app_uart_fifo.o(.data) for .data
    app_uart_fifo.o(i.app_uart_get) refers to app_uart_fifo.o(.bss) for .bss
    app_uart_fifo.o(i.app_uart_init) refers to app_fifo.o(i.app_fifo_init) for app_fifo_init
    app_uart_fifo.o(i.app_uart_init) refers to memcpya.o(.text) for __aeabi_memcpy4
    app_uart_fifo.o(i.app_uart_init) refers to nrf_drv_uart.o(i.nrf_drv_uart_init) for nrf_drv_uart_init
    app_uart_fifo.o(i.app_uart_init) refers to app_uart_fifo.o(i.nrf_drv_uart_rx) for nrf_drv_uart_rx
    app_uart_fifo.o(i.app_uart_init) refers to app_uart_fifo.o(.data) for .data
    app_uart_fifo.o(i.app_uart_init) refers to app_uart_fifo.o(.bss) for .bss
    app_uart_fifo.o(i.app_uart_init) refers to app_uart_fifo.o(.constdata) for .constdata
    app_uart_fifo.o(i.app_uart_init) refers to app_uart_fifo.o(i.uart_event_handler) for uart_event_handler
    app_uart_fifo.o(i.app_uart_put) refers to app_fifo.o(i.app_fifo_put) for app_fifo_put
    app_uart_fifo.o(i.app_uart_put) refers to nrfx_uarte.o(i.nrfx_uarte_tx_in_progress) for nrfx_uarte_tx_in_progress
    app_uart_fifo.o(i.app_uart_put) refers to app_fifo.o(i.app_fifo_get) for app_fifo_get
    app_uart_fifo.o(i.app_uart_put) refers to app_uart_fifo.o(i.nrf_drv_uart_tx) for nrf_drv_uart_tx
    app_uart_fifo.o(i.app_uart_put) refers to app_uart_fifo.o(.bss) for .bss
    app_uart_fifo.o(i.app_uart_put) refers to app_uart_fifo.o(.data) for .data
    app_uart_fifo.o(i.nrf_drv_uart_rx) refers to nrfx_uarte.o(i.nrfx_uarte_rx) for nrfx_uarte_rx
    app_uart_fifo.o(i.nrf_drv_uart_tx) refers to nrfx_uarte.o(i.nrfx_uarte_tx) for nrfx_uarte_tx
    app_uart_fifo.o(i.uart_event_handler) refers to app_uart_fifo.o(i.nrf_drv_uart_rx) for nrf_drv_uart_rx
    app_uart_fifo.o(i.uart_event_handler) refers to app_fifo.o(i.app_fifo_put) for app_fifo_put
    app_uart_fifo.o(i.uart_event_handler) refers to app_fifo.o(i.app_fifo_get) for app_fifo_get
    app_uart_fifo.o(i.uart_event_handler) refers to app_uart_fifo.o(i.nrf_drv_uart_tx) for nrf_drv_uart_tx
    app_uart_fifo.o(i.uart_event_handler) refers to app_uart_fifo.o(.data) for .data
    app_uart_fifo.o(i.uart_event_handler) refers to app_uart_fifo.o(.bss) for .bss
    app_util_platform.o(i.app_util_critical_region_enter) refers to app_util_platform.o(.bss) for .bss
    app_util_platform.o(i.app_util_critical_region_exit) refers to app_util_platform.o(.bss) for .bss
    app_util_platform.o(i.app_util_disable_irq) refers to app_util_platform.o(.data) for .data
    app_util_platform.o(i.app_util_enable_irq) refers to app_util_platform.o(.data) for .data
    nrf_assert.o(i.assert_nrf_callback) refers to app_error_weak.o(i.app_error_fault_handler) for app_error_fault_handler
    nrf_atfifo.o(i.nrf_atfifo_alloc_put) refers to nrf_atfifo.o(i.nrf_atfifo_item_alloc) for nrf_atfifo_item_alloc
    nrf_atfifo.o(i.nrf_atfifo_alloc_put) refers to memcpya.o(.text) for __aeabi_memcpy
    nrf_atfifo.o(i.nrf_atfifo_alloc_put) refers to nrf_atfifo.o(i.nrf_atfifo_item_put) for nrf_atfifo_item_put
    nrf_atfifo.o(i.nrf_atfifo_clear) refers to nrf_atfifo.o(.emb_text) for __asm___12_nrf_atfifo_c_51f461e1__nrf_atfifo_space_clear
    nrf_atfifo.o(i.nrf_atfifo_get_free) refers to nrf_atfifo.o(i.nrf_atfifo_item_get) for nrf_atfifo_item_get
    nrf_atfifo.o(i.nrf_atfifo_get_free) refers to memcpya.o(.text) for __aeabi_memcpy
    nrf_atfifo.o(i.nrf_atfifo_get_free) refers to nrf_atfifo.o(i.nrf_atfifo_item_free) for nrf_atfifo_item_free
    nrf_atfifo.o(i.nrf_atfifo_item_alloc) refers to nrf_atfifo.o(.emb_text) for __asm___12_nrf_atfifo_c_51f461e1__nrf_atfifo_wspace_req
    nrf_atfifo.o(i.nrf_atfifo_item_free) refers to nrf_atfifo.o(.emb_text) for __asm___12_nrf_atfifo_c_51f461e1__nrf_atfifo_rspace_close
    nrf_atfifo.o(i.nrf_atfifo_item_get) refers to nrf_atfifo.o(.emb_text) for __asm___12_nrf_atfifo_c_51f461e1__nrf_atfifo_rspace_req
    nrf_atfifo.o(i.nrf_atfifo_item_put) refers to nrf_atfifo.o(.emb_text) for __asm___12_nrf_atfifo_c_51f461e1__nrf_atfifo_wspace_close
    nrf_atflags.o(i.nrf_atflags_clear) refers to nrf_atomic.o(i.nrf_atomic_u32_and) for nrf_atomic_u32_and
    nrf_atflags.o(i.nrf_atflags_fetch_clear) refers to nrf_atomic.o(i.nrf_atomic_u32_fetch_and) for nrf_atomic_u32_fetch_and
    nrf_atflags.o(i.nrf_atflags_fetch_set) refers to nrf_atomic.o(i.nrf_atomic_u32_fetch_or) for nrf_atomic_u32_fetch_or
    nrf_atflags.o(i.nrf_atflags_find_and_clear_flag) refers to nrf_atflags.o(i.nrf_atflags_fetch_clear) for nrf_atflags_fetch_clear
    nrf_atflags.o(i.nrf_atflags_find_and_set_flag) refers to nrf_atflags.o(i.nrf_atflags_fetch_set) for nrf_atflags_fetch_set
    nrf_atflags.o(i.nrf_atflags_set) refers to nrf_atomic.o(i.nrf_atomic_u32_or) for nrf_atomic_u32_or
    nrf_atomic.o(i.nrf_atomic_flag_clear) refers to nrf_atomic.o(i.nrf_atomic_u32_and) for nrf_atomic_u32_and
    nrf_atomic.o(i.nrf_atomic_flag_clear_fetch) refers to nrf_atomic.o(i.nrf_atomic_u32_fetch_and) for nrf_atomic_u32_fetch_and
    nrf_atomic.o(i.nrf_atomic_flag_set) refers to nrf_atomic.o(i.nrf_atomic_u32_or) for nrf_atomic_u32_or
    nrf_atomic.o(i.nrf_atomic_flag_set_fetch) refers to nrf_atomic.o(i.nrf_atomic_u32_fetch_or) for nrf_atomic_u32_fetch_or
    nrf_atomic.o(i.nrf_atomic_u32_add) refers to nrf_atomic.o(.emb_text) for __asm___12_nrf_atomic_c_85ca2469__nrf_atomic_internal_add
    nrf_atomic.o(i.nrf_atomic_u32_and) refers to nrf_atomic.o(.emb_text) for __asm___12_nrf_atomic_c_85ca2469__nrf_atomic_internal_and
    nrf_atomic.o(i.nrf_atomic_u32_cmp_exch) refers to nrf_atomic.o(.emb_text) for __asm___12_nrf_atomic_c_85ca2469__nrf_atomic_internal_cmp_exch
    nrf_atomic.o(i.nrf_atomic_u32_fetch_add) refers to nrf_atomic.o(.emb_text) for __asm___12_nrf_atomic_c_85ca2469__nrf_atomic_internal_add
    nrf_atomic.o(i.nrf_atomic_u32_fetch_and) refers to nrf_atomic.o(.emb_text) for __asm___12_nrf_atomic_c_85ca2469__nrf_atomic_internal_and
    nrf_atomic.o(i.nrf_atomic_u32_fetch_or) refers to nrf_atomic.o(.emb_text) for __asm___12_nrf_atomic_c_85ca2469__nrf_atomic_internal_orr
    nrf_atomic.o(i.nrf_atomic_u32_fetch_store) refers to nrf_atomic.o(.emb_text) for __asm___12_nrf_atomic_c_85ca2469__nrf_atomic_internal_mov
    nrf_atomic.o(i.nrf_atomic_u32_fetch_sub) refers to nrf_atomic.o(.emb_text) for __asm___12_nrf_atomic_c_85ca2469__nrf_atomic_internal_sub
    nrf_atomic.o(i.nrf_atomic_u32_fetch_sub_hs) refers to nrf_atomic.o(.emb_text) for __asm___12_nrf_atomic_c_85ca2469__nrf_atomic_internal_sub_hs
    nrf_atomic.o(i.nrf_atomic_u32_fetch_xor) refers to nrf_atomic.o(.emb_text) for __asm___12_nrf_atomic_c_85ca2469__nrf_atomic_internal_eor
    nrf_atomic.o(i.nrf_atomic_u32_or) refers to nrf_atomic.o(.emb_text) for __asm___12_nrf_atomic_c_85ca2469__nrf_atomic_internal_orr
    nrf_atomic.o(i.nrf_atomic_u32_store) refers to nrf_atomic.o(.emb_text) for __asm___12_nrf_atomic_c_85ca2469__nrf_atomic_internal_mov
    nrf_atomic.o(i.nrf_atomic_u32_sub) refers to nrf_atomic.o(.emb_text) for __asm___12_nrf_atomic_c_85ca2469__nrf_atomic_internal_sub
    nrf_atomic.o(i.nrf_atomic_u32_sub_hs) refers to nrf_atomic.o(.emb_text) for __asm___12_nrf_atomic_c_85ca2469__nrf_atomic_internal_sub_hs
    nrf_atomic.o(i.nrf_atomic_u32_xor) refers to nrf_atomic.o(.emb_text) for __asm___12_nrf_atomic_c_85ca2469__nrf_atomic_internal_eor
    nrf_balloc.o(i.nrf_balloc_alloc) refers to app_util_platform.o(i.app_util_critical_region_enter) for app_util_critical_region_enter
    nrf_balloc.o(i.nrf_balloc_alloc) refers to app_util_platform.o(i.app_util_critical_region_exit) for app_util_critical_region_exit
    nrf_balloc.o(i.nrf_balloc_free) refers to app_util_platform.o(i.app_util_critical_region_enter) for app_util_critical_region_enter
    nrf_balloc.o(i.nrf_balloc_free) refers to app_util_platform.o(i.app_util_critical_region_exit) for app_util_critical_region_exit
    nrf_fprintf.o(i.nrf_fprintf) refers to nrf_fprintf_format.o(i.nrf_fprintf_fmt) for nrf_fprintf_fmt
    nrf_fprintf_format.o(i.buffer_add) refers to nrf_fprintf.o(i.nrf_fprintf_buffer_flush) for nrf_fprintf_buffer_flush
    nrf_fprintf_format.o(i.int_print) refers to nrf_fprintf_format.o(i.buffer_add) for buffer_add
    nrf_fprintf_format.o(i.int_print) refers to nrf_fprintf_format.o(i.unsigned_print) for unsigned_print
    nrf_fprintf_format.o(i.nrf_fprintf_fmt) refers to nrf_fprintf_format.o(i.buffer_add) for buffer_add
    nrf_fprintf_format.o(i.nrf_fprintf_fmt) refers to nrf_fprintf.o(i.nrf_fprintf_buffer_flush) for nrf_fprintf_buffer_flush
    nrf_fprintf_format.o(i.nrf_fprintf_fmt) refers to nrf_fprintf_format.o(i.int_print) for int_print
    nrf_fprintf_format.o(i.nrf_fprintf_fmt) refers to nrf_fprintf_format.o(i.unsigned_print) for unsigned_print
    nrf_fprintf_format.o(i.nrf_fprintf_fmt) refers to strlen.o(.text) for strlen
    nrf_fprintf_format.o(i.unsigned_print) refers to nrf_fprintf_format.o(i.buffer_add) for buffer_add
    nrf_fprintf_format.o(i.unsigned_print) refers to nrf_fprintf_format.o(.constdata) for .constdata
    nrf_memobj.o(i.memobj_op) refers to memcpya.o(.text) for __aeabi_memcpy
    nrf_memobj.o(i.nrf_memobj_alloc) refers to nrf_balloc.o(i.nrf_balloc_alloc) for nrf_balloc_alloc
    nrf_memobj.o(i.nrf_memobj_alloc) refers to nrf_memobj.o(i.nrf_memobj_free) for nrf_memobj_free
    nrf_memobj.o(i.nrf_memobj_free) refers to nrf_balloc.o(i.nrf_balloc_free) for nrf_balloc_free
    nrf_memobj.o(i.nrf_memobj_get) refers to nrf_atomic.o(i.nrf_atomic_u32_add) for nrf_atomic_u32_add
    nrf_memobj.o(i.nrf_memobj_pool_init) refers to nrf_balloc.o(i.nrf_balloc_init) for nrf_balloc_init
    nrf_memobj.o(i.nrf_memobj_put) refers to nrf_atomic.o(i.nrf_atomic_u32_sub) for nrf_atomic_u32_sub
    nrf_memobj.o(i.nrf_memobj_put) refers to nrf_memobj.o(i.nrf_memobj_free) for nrf_memobj_free
    nrf_memobj.o(i.nrf_memobj_read) refers to nrf_memobj.o(i.memobj_op) for memobj_op
    nrf_memobj.o(i.nrf_memobj_write) refers to nrf_memobj.o(i.memobj_op) for memobj_op
    nrf_pwr_mgmt.o(i.nrf_pwr_mgmt_init) refers to nrf_section_iter.o(i.nrf_section_iter_init) for nrf_section_iter_init
    nrf_pwr_mgmt.o(i.nrf_pwr_mgmt_init) refers to nrf_pwr_mgmt.o(.data) for .data
    nrf_pwr_mgmt.o(i.nrf_pwr_mgmt_init) refers to nrf_pwr_mgmt.o(.constdata) for .constdata
    nrf_pwr_mgmt.o(i.nrf_pwr_mgmt_init) refers to nrf_pwr_mgmt.o(.bss) for .bss
    nrf_pwr_mgmt.o(i.nrf_pwr_mgmt_run) refers to nrf_sdh.o(i.nrf_sdh_is_enabled) for nrf_sdh_is_enabled
    nrf_pwr_mgmt.o(i.nrf_pwr_mgmt_shutdown) refers to nrf_atomic.o(i.nrf_atomic_u32_fetch_store) for nrf_atomic_u32_fetch_store
    nrf_pwr_mgmt.o(i.nrf_pwr_mgmt_shutdown) refers to nrf_pwr_mgmt.o(i.shutdown_process) for shutdown_process
    nrf_pwr_mgmt.o(i.nrf_pwr_mgmt_shutdown) refers to nrf_pwr_mgmt.o(.data) for .data
    nrf_pwr_mgmt.o(i.shutdown_process) refers to nrf_section_iter.o(i.nrf_section_iter_next) for nrf_section_iter_next
    nrf_pwr_mgmt.o(i.shutdown_process) refers to nrf_log_frontend.o(i.nrf_log_panic) for nrf_log_panic
    nrf_pwr_mgmt.o(i.shutdown_process) refers to nrf_log_frontend.o(i.nrf_log_frontend_dequeue) for nrf_log_frontend_dequeue
    nrf_pwr_mgmt.o(i.shutdown_process) refers to nrf_sdh.o(i.nrf_sdh_is_enabled) for nrf_sdh_is_enabled
    nrf_pwr_mgmt.o(i.shutdown_process) refers to nrf_pwr_mgmt.o(.bss) for .bss
    nrf_pwr_mgmt.o(i.shutdown_process) refers to nrf_pwr_mgmt.o(.data) for .data
    nrf_pwr_mgmt.o(.constdata) refers to nrf_pwr_mgmt.o(.constdata) for pwr_mgmt_data_array
    nrf_pwr_mgmt.o(log_const_data) refers to nrf_pwr_mgmt.o(.conststrlit) for .conststrlit
    nrf_ringbuf.o(i.nrf_ringbuf_alloc) refers to nrf_atomic.o(i.nrf_atomic_flag_set_fetch) for nrf_atomic_flag_set_fetch
    nrf_ringbuf.o(i.nrf_ringbuf_alloc) refers to nrf_atomic.o(i.nrf_atomic_flag_clear) for nrf_atomic_flag_clear
    nrf_ringbuf.o(i.nrf_ringbuf_cpy_get) refers to nrf_atomic.o(i.nrf_atomic_flag_set_fetch) for nrf_atomic_flag_set_fetch
    nrf_ringbuf.o(i.nrf_ringbuf_cpy_get) refers to memcpya.o(.text) for __aeabi_memcpy
    nrf_ringbuf.o(i.nrf_ringbuf_cpy_get) refers to nrf_atomic.o(i.nrf_atomic_flag_clear) for nrf_atomic_flag_clear
    nrf_ringbuf.o(i.nrf_ringbuf_cpy_put) refers to nrf_atomic.o(i.nrf_atomic_flag_set_fetch) for nrf_atomic_flag_set_fetch
    nrf_ringbuf.o(i.nrf_ringbuf_cpy_put) refers to memcpya.o(.text) for __aeabi_memcpy
    nrf_ringbuf.o(i.nrf_ringbuf_cpy_put) refers to nrf_atomic.o(i.nrf_atomic_flag_clear) for nrf_atomic_flag_clear
    nrf_ringbuf.o(i.nrf_ringbuf_free) refers to nrf_atomic.o(i.nrf_atomic_flag_clear) for nrf_atomic_flag_clear
    nrf_ringbuf.o(i.nrf_ringbuf_get) refers to nrf_atomic.o(i.nrf_atomic_flag_set_fetch) for nrf_atomic_flag_set_fetch
    nrf_ringbuf.o(i.nrf_ringbuf_get) refers to nrf_atomic.o(i.nrf_atomic_flag_clear) for nrf_atomic_flag_clear
    nrf_ringbuf.o(i.nrf_ringbuf_put) refers to nrf_atomic.o(i.nrf_atomic_flag_clear_fetch) for nrf_atomic_flag_clear_fetch
    nrf_section_iter.o(i.nrf_section_iter_init) refers to nrf_section_iter.o(i.nrf_section_iter_item_set) for nrf_section_iter_item_set
    nrf_section_iter.o(i.nrf_section_iter_next) refers to nrf_section_iter.o(i.nrf_section_iter_item_set) for nrf_section_iter_item_set
    nrf_strerror.o(i.nrf_strerror_find) refers to nrf_strerror.o(.constdata) for .constdata
    nrf_strerror.o(i.nrf_strerror_get) refers to nrf_strerror.o(i.nrf_strerror_find) for nrf_strerror_find
    nrf_strerror.o(i.nrf_strerror_get) refers to nrf_strerror.o(.constdata) for .constdata
    nrf_strerror.o(.constdata) refers to nrf_strerror.o(.conststring) for .conststring
    retarget.o(i.fgetc) refers to app_uart_fifo.o(i.app_uart_get) for app_uart_get
    retarget.o(i.fputc) refers to app_uart_fifo.o(i.app_uart_put) for app_uart_put
    nrf_log_backend_rtt.o(i.nrf_log_backend_rtt_init) refers to segger_rtt.o(i.SEGGER_RTT_Init) for SEGGER_RTT_Init
    nrf_log_backend_rtt.o(i.nrf_log_backend_rtt_put) refers to nrf_log_backend_serial.o(i.nrf_log_backend_serial_put) for nrf_log_backend_serial_put
    nrf_log_backend_rtt.o(i.nrf_log_backend_rtt_put) refers to nrf_log_backend_rtt.o(i.serial_tx) for serial_tx
    nrf_log_backend_rtt.o(i.nrf_log_backend_rtt_put) refers to nrf_log_backend_rtt.o(.bss) for .bss
    nrf_log_backend_rtt.o(i.serial_tx) refers to segger_rtt.o(i.SEGGER_RTT_WriteNoLock) for SEGGER_RTT_WriteNoLock
    nrf_log_backend_rtt.o(i.serial_tx) refers to nrf_log_backend_rtt.o(.data) for .data
    nrf_log_backend_rtt.o(i.serial_tx) refers to nrf_log_backend_rtt.o(.constdata) for .constdata
    nrf_log_backend_rtt.o(.constdata) refers to nrf_log_backend_rtt.o(i.nrf_log_backend_rtt_put) for nrf_log_backend_rtt_put
    nrf_log_backend_rtt.o(.constdata) refers to nrf_log_backend_rtt.o(i.nrf_log_backend_rtt_panic_set) for nrf_log_backend_rtt_panic_set
    nrf_log_backend_rtt.o(.constdata) refers to nrf_log_backend_rtt.o(i.nrf_log_backend_rtt_flush) for nrf_log_backend_rtt_flush
    nrf_log_backend_serial.o(i.nrf_log_backend_serial_put) refers to nrf_memobj.o(i.nrf_memobj_get) for nrf_memobj_get
    nrf_log_backend_serial.o(i.nrf_log_backend_serial_put) refers to memseta.o(.text) for __aeabi_memclr4
    nrf_log_backend_serial.o(i.nrf_log_backend_serial_put) refers to nrf_memobj.o(i.nrf_memobj_read) for nrf_memobj_read
    nrf_log_backend_serial.o(i.nrf_log_backend_serial_put) refers to nrf_log_str_formatter.o(i.nrf_log_std_entry_process) for nrf_log_std_entry_process
    nrf_log_backend_serial.o(i.nrf_log_backend_serial_put) refers to nrf_log_str_formatter.o(i.nrf_log_hexdump_entry_process) for nrf_log_hexdump_entry_process
    nrf_log_backend_serial.o(i.nrf_log_backend_serial_put) refers to nrf_memobj.o(i.nrf_memobj_put) for nrf_memobj_put
    nrf_log_default_backends.o(i.nrf_log_default_backends_init) refers to nrf_log_backend_rtt.o(i.nrf_log_backend_rtt_init) for nrf_log_backend_rtt_init
    nrf_log_default_backends.o(i.nrf_log_default_backends_init) refers to nrf_log_frontend.o(i.nrf_log_backend_add) for nrf_log_backend_add
    nrf_log_default_backends.o(i.nrf_log_default_backends_init) refers to nrf_log_default_backends.o(log_backends) for log_backends
    nrf_log_default_backends.o(log_backends) refers to nrf_log_backend_rtt.o(.constdata) for nrf_log_backend_rtt_api
    nrf_log_default_backends.o(log_backends) refers to nrf_log_default_backends.o(.conststrlit) for .conststrlit
    nrf_log_default_backends.o(log_backends) refers to nrf_log_default_backends.o(.data) for log_backend_cb_rtt_log_backend
    nrf_log_frontend.o(i.buf_prealloc) refers to app_util_platform.o(i.app_util_critical_region_enter) for app_util_critical_region_enter
    nrf_log_frontend.o(i.buf_prealloc) refers to nrf_atomic.o(i.nrf_atomic_u32_add) for nrf_atomic_u32_add
    nrf_log_frontend.o(i.buf_prealloc) refers to nrf_log_frontend.o(i.log_skip) for log_skip
    nrf_log_frontend.o(i.buf_prealloc) refers to app_util_platform.o(i.app_util_critical_region_exit) for app_util_critical_region_exit
    nrf_log_frontend.o(i.buf_prealloc) refers to nrf_log_frontend.o(.bss) for .bss
    nrf_log_frontend.o(i.buffer_is_empty) refers to nrf_log_frontend.o(.bss) for .bss
    nrf_log_frontend.o(i.dropped_sat16_get) refers to nrf_atomic.o(i.nrf_atomic_u32_fetch_store) for nrf_atomic_u32_fetch_store
    nrf_log_frontend.o(i.dropped_sat16_get) refers to nrf_log_frontend.o(.bss) for .bss
    nrf_log_frontend.o(i.log_skip) refers to nrf_atomic.o(i.nrf_atomic_flag_set) for nrf_atomic_flag_set
    nrf_log_frontend.o(i.log_skip) refers to nrf_log_frontend.o(i.invalid_packets_omit) for invalid_packets_omit
    nrf_log_frontend.o(i.log_skip) refers to nrf_atomic.o(i.nrf_atomic_flag_clear_fetch) for nrf_atomic_flag_clear_fetch
    nrf_log_frontend.o(i.log_skip) refers to nrf_log_frontend.o(.bss) for .bss
    nrf_log_frontend.o(i.module_idx_get) refers to nrf_log_frontend.o(i.nrf_log_module_cnt_get) for nrf_log_module_cnt_get
    nrf_log_frontend.o(i.nrf_log_backend_add) refers to nrf_log_frontend.o(.bss) for .bss
    nrf_log_frontend.o(i.nrf_log_backend_remove) refers to nrf_log_frontend.o(.bss) for .bss
    nrf_log_frontend.o(i.nrf_log_frontend_dequeue) refers to nrf_log_frontend.o(i.buffer_is_empty) for buffer_is_empty
    nrf_log_frontend.o(i.nrf_log_frontend_dequeue) refers to nrf_log_frontend.o(i.invalid_packets_omit) for invalid_packets_omit
    nrf_log_frontend.o(i.nrf_log_frontend_dequeue) refers to nrf_memobj.o(i.nrf_memobj_alloc) for nrf_memobj_alloc
    nrf_log_frontend.o(i.nrf_log_frontend_dequeue) refers to nrf_memobj.o(i.nrf_memobj_get) for nrf_memobj_get
    nrf_log_frontend.o(i.nrf_log_frontend_dequeue) refers to nrf_memobj.o(i.nrf_memobj_write) for nrf_memobj_write
    nrf_log_frontend.o(i.nrf_log_frontend_dequeue) refers to nrf_memobj.o(i.nrf_memobj_put) for nrf_memobj_put
    nrf_log_frontend.o(i.nrf_log_frontend_dequeue) refers to app_util_platform.o(i.app_util_critical_region_enter) for app_util_critical_region_enter
    nrf_log_frontend.o(i.nrf_log_frontend_dequeue) refers to app_util_platform.o(i.app_util_critical_region_exit) for app_util_critical_region_exit
    nrf_log_frontend.o(i.nrf_log_frontend_dequeue) refers to nrf_log_frontend.o(i.nrf_log_frontend_std_0) for nrf_log_frontend_std_0
    nrf_log_frontend.o(i.nrf_log_frontend_dequeue) refers to nrf_log_frontend.o(.bss) for .bss
    nrf_log_frontend.o(i.nrf_log_frontend_dequeue) refers to nrf_log_frontend.o(nrf_balloc) for nrf_balloc
    nrf_log_frontend.o(i.nrf_log_frontend_dequeue) refers to nrf_log_frontend.o(log_const_data) for log_const_data
    nrf_log_frontend.o(i.nrf_log_frontend_hexdump) refers to nrf_log_frontend.o(i.buf_prealloc) for buf_prealloc
    nrf_log_frontend.o(i.nrf_log_frontend_hexdump) refers to memcpya.o(.text) for __aeabi_memcpy
    nrf_log_frontend.o(i.nrf_log_frontend_hexdump) refers to nrf_log_frontend.o(i.dropped_sat16_get) for dropped_sat16_get
    nrf_log_frontend.o(i.nrf_log_frontend_hexdump) refers to nrf_log_frontend.o(i.nrf_log_frontend_dequeue) for nrf_log_frontend_dequeue
    nrf_log_frontend.o(i.nrf_log_frontend_hexdump) refers to nrf_log_frontend.o(.bss) for .bss
    nrf_log_frontend.o(i.nrf_log_frontend_std_0) refers to nrf_log_frontend.o(i.std_n) for std_n
    nrf_log_frontend.o(i.nrf_log_frontend_std_1) refers to nrf_log_frontend.o(i.std_n) for std_n
    nrf_log_frontend.o(i.nrf_log_frontend_std_2) refers to nrf_log_frontend.o(i.std_n) for std_n
    nrf_log_frontend.o(i.nrf_log_frontend_std_3) refers to nrf_log_frontend.o(i.std_n) for std_n
    nrf_log_frontend.o(i.nrf_log_frontend_std_4) refers to nrf_log_frontend.o(i.std_n) for std_n
    nrf_log_frontend.o(i.nrf_log_frontend_std_5) refers to nrf_log_frontend.o(i.std_n) for std_n
    nrf_log_frontend.o(i.nrf_log_frontend_std_6) refers to nrf_log_frontend.o(i.std_n) for std_n
    nrf_log_frontend.o(i.nrf_log_init) refers to nrf_memobj.o(i.nrf_memobj_pool_init) for nrf_memobj_pool_init
    nrf_log_frontend.o(i.nrf_log_init) refers to nrf_ringbuf.o(i.nrf_ringbuf_init) for nrf_ringbuf_init
    nrf_log_frontend.o(i.nrf_log_init) refers to nrf_log_frontend.o(.bss) for .bss
    nrf_log_frontend.o(i.nrf_log_init) refers to nrf_log_frontend.o(nrf_balloc) for nrf_balloc
    nrf_log_frontend.o(i.nrf_log_init) refers to nrf_log_frontend.o(.constdata) for .constdata
    nrf_log_frontend.o(i.nrf_log_module_filter_get) refers to nrf_log_frontend.o(i.module_idx_get) for module_idx_get
    nrf_log_frontend.o(i.nrf_log_module_name_get) refers to nrf_log_frontend.o(i.module_idx_get) for module_idx_get
    nrf_log_frontend.o(i.nrf_log_panic) refers to nrf_log_frontend.o(.bss) for .bss
    nrf_log_frontend.o(i.nrf_log_push) refers to strlen.o(.text) for strlen
    nrf_log_frontend.o(i.nrf_log_push) refers to nrf_ringbuf.o(i.nrf_ringbuf_alloc) for nrf_ringbuf_alloc
    nrf_log_frontend.o(i.nrf_log_push) refers to memcpya.o(.text) for __aeabi_memcpy
    nrf_log_frontend.o(i.nrf_log_push) refers to nrf_ringbuf.o(i.nrf_ringbuf_put) for nrf_ringbuf_put
    nrf_log_frontend.o(i.nrf_log_push) refers to nrf_ringbuf.o(i.nrf_ringbuf_free) for nrf_ringbuf_free
    nrf_log_frontend.o(i.nrf_log_push) refers to nrf_log_frontend.o(.bss) for .bss
    nrf_log_frontend.o(i.nrf_log_push) refers to nrf_log_frontend.o(.constdata) for .constdata
    nrf_log_frontend.o(i.std_n) refers to nrf_log_frontend.o(i.buf_prealloc) for buf_prealloc
    nrf_log_frontend.o(i.std_n) refers to nrf_log_frontend.o(i.dropped_sat16_get) for dropped_sat16_get
    nrf_log_frontend.o(i.std_n) refers to nrf_log_frontend.o(i.nrf_log_frontend_dequeue) for nrf_log_frontend_dequeue
    nrf_log_frontend.o(i.std_n) refers to nrf_log_frontend.o(.bss) for .bss
    nrf_log_frontend.o(.constdata) refers to nrf_log_frontend.o(.bss) for m_log_push_ringbuf_buf
    nrf_log_frontend.o(.constdata) refers to nrf_log_frontend.o(.bss) for m_log_push_ringbuf_cb
    nrf_log_frontend.o(log_const_data) refers to nrf_log_frontend.o(.conststrlit) for .conststrlit
    nrf_log_frontend.o(nrf_balloc) refers to nrf_log_frontend.o(.data) for log_mempool_nrf_balloc_cb
    nrf_log_frontend.o(nrf_balloc) refers to nrf_log_frontend.o(.data) for log_mempool_nrf_balloc_pool_stack
    nrf_log_frontend.o(nrf_balloc) refers to nrf_log_frontend.o(.bss) for log_mempool_nrf_balloc_pool_mem
    nrf_log_str_formatter.o(i.nrf_log_hexdump_entry_process) refers to nrf_log_str_formatter.o(i.prefix_process) for prefix_process
    nrf_log_str_formatter.o(i.nrf_log_hexdump_entry_process) refers to nrf_fprintf.o(i.nrf_fprintf) for nrf_fprintf
    nrf_log_str_formatter.o(i.nrf_log_hexdump_entry_process) refers to ctype_o.o(.text) for __rt_ctype_table
    nrf_log_str_formatter.o(i.nrf_log_hexdump_entry_process) refers to nrf_log_str_formatter.o(i.postfix_process) for postfix_process
    nrf_log_str_formatter.o(i.nrf_log_std_entry_process) refers to nrf_log_str_formatter.o(i.prefix_process) for prefix_process
    nrf_log_str_formatter.o(i.nrf_log_std_entry_process) refers to nrf_fprintf.o(i.nrf_fprintf) for nrf_fprintf
    nrf_log_str_formatter.o(i.nrf_log_std_entry_process) refers to nrf_log_str_formatter.o(i.postfix_process) for postfix_process
    nrf_log_str_formatter.o(i.nrf_log_str_formatter_timestamp_freq_set) refers to nrf_log_str_formatter.o(.data) for .data
    nrf_log_str_formatter.o(i.postfix_process) refers to nrf_fprintf.o(i.nrf_fprintf) for nrf_fprintf
    nrf_log_str_formatter.o(i.postfix_process) refers to nrf_fprintf.o(i.nrf_fprintf_buffer_flush) for nrf_fprintf_buffer_flush
    nrf_log_str_formatter.o(i.postfix_process) refers to nrf_log_str_formatter.o(.data) for .data
    nrf_log_str_formatter.o(i.prefix_process) refers to nrf_fprintf.o(i.nrf_fprintf) for nrf_fprintf
    nrf_log_str_formatter.o(i.prefix_process) refers to nrf_log_frontend.o(i.nrf_log_color_id_get) for nrf_log_color_id_get
    nrf_log_str_formatter.o(i.prefix_process) refers to nrf_log_frontend.o(i.nrf_log_module_name_get) for nrf_log_module_name_get
    nrf_log_str_formatter.o(i.prefix_process) refers to nrf_log_str_formatter.o(.data) for .data
    nrf_log_str_formatter.o(.data) refers to nrf_log_str_formatter.o(.conststring) for .conststring
    segger_rtt.o(i.SEGGER_RTT_AllocDownBuffer) refers to segger_rtt.o(i._DoInit) for _DoInit
    segger_rtt.o(i.SEGGER_RTT_AllocDownBuffer) refers to app_util_platform.o(i.app_util_critical_region_enter) for app_util_critical_region_enter
    segger_rtt.o(i.SEGGER_RTT_AllocDownBuffer) refers to app_util_platform.o(i.app_util_critical_region_exit) for app_util_critical_region_exit
    segger_rtt.o(i.SEGGER_RTT_AllocDownBuffer) refers to segger_rtt.o(.bss) for .bss
    segger_rtt.o(i.SEGGER_RTT_AllocUpBuffer) refers to segger_rtt.o(i._DoInit) for _DoInit
    segger_rtt.o(i.SEGGER_RTT_AllocUpBuffer) refers to app_util_platform.o(i.app_util_critical_region_enter) for app_util_critical_region_enter
    segger_rtt.o(i.SEGGER_RTT_AllocUpBuffer) refers to app_util_platform.o(i.app_util_critical_region_exit) for app_util_critical_region_exit
    segger_rtt.o(i.SEGGER_RTT_AllocUpBuffer) refers to segger_rtt.o(.bss) for .bss
    segger_rtt.o(i.SEGGER_RTT_ConfigDownBuffer) refers to segger_rtt.o(i._DoInit) for _DoInit
    segger_rtt.o(i.SEGGER_RTT_ConfigDownBuffer) refers to app_util_platform.o(i.app_util_critical_region_enter) for app_util_critical_region_enter
    segger_rtt.o(i.SEGGER_RTT_ConfigDownBuffer) refers to app_util_platform.o(i.app_util_critical_region_exit) for app_util_critical_region_exit
    segger_rtt.o(i.SEGGER_RTT_ConfigDownBuffer) refers to segger_rtt.o(.bss) for .bss
    segger_rtt.o(i.SEGGER_RTT_ConfigUpBuffer) refers to segger_rtt.o(i._DoInit) for _DoInit
    segger_rtt.o(i.SEGGER_RTT_ConfigUpBuffer) refers to app_util_platform.o(i.app_util_critical_region_enter) for app_util_critical_region_enter
    segger_rtt.o(i.SEGGER_RTT_ConfigUpBuffer) refers to app_util_platform.o(i.app_util_critical_region_exit) for app_util_critical_region_exit
    segger_rtt.o(i.SEGGER_RTT_ConfigUpBuffer) refers to segger_rtt.o(.bss) for .bss
    segger_rtt.o(i.SEGGER_RTT_GetKey) refers to segger_rtt.o(i.SEGGER_RTT_Read) for SEGGER_RTT_Read
    segger_rtt.o(i.SEGGER_RTT_HasData) refers to segger_rtt.o(.bss) for .bss
    segger_rtt.o(i.SEGGER_RTT_HasKey) refers to segger_rtt.o(i._DoInit) for _DoInit
    segger_rtt.o(i.SEGGER_RTT_HasKey) refers to segger_rtt.o(.bss) for .bss
    segger_rtt.o(i.SEGGER_RTT_Init) refers to segger_rtt.o(i._DoInit) for _DoInit
    segger_rtt.o(i.SEGGER_RTT_PutChar) refers to segger_rtt.o(i._DoInit) for _DoInit
    segger_rtt.o(i.SEGGER_RTT_PutChar) refers to app_util_platform.o(i.app_util_critical_region_enter) for app_util_critical_region_enter
    segger_rtt.o(i.SEGGER_RTT_PutChar) refers to app_util_platform.o(i.app_util_critical_region_exit) for app_util_critical_region_exit
    segger_rtt.o(i.SEGGER_RTT_PutChar) refers to segger_rtt.o(.bss) for .bss
    segger_rtt.o(i.SEGGER_RTT_PutCharSkip) refers to segger_rtt.o(i._DoInit) for _DoInit
    segger_rtt.o(i.SEGGER_RTT_PutCharSkip) refers to app_util_platform.o(i.app_util_critical_region_enter) for app_util_critical_region_enter
    segger_rtt.o(i.SEGGER_RTT_PutCharSkip) refers to app_util_platform.o(i.app_util_critical_region_exit) for app_util_critical_region_exit
    segger_rtt.o(i.SEGGER_RTT_PutCharSkip) refers to segger_rtt.o(.bss) for .bss
    segger_rtt.o(i.SEGGER_RTT_PutCharSkipNoLock) refers to segger_rtt.o(.bss) for .bss
    segger_rtt.o(i.SEGGER_RTT_Read) refers to app_util_platform.o(i.app_util_critical_region_enter) for app_util_critical_region_enter
    segger_rtt.o(i.SEGGER_RTT_Read) refers to segger_rtt.o(i.SEGGER_RTT_ReadNoLock) for SEGGER_RTT_ReadNoLock
    segger_rtt.o(i.SEGGER_RTT_Read) refers to app_util_platform.o(i.app_util_critical_region_exit) for app_util_critical_region_exit
    segger_rtt.o(i.SEGGER_RTT_ReadNoLock) refers to segger_rtt.o(i._DoInit) for _DoInit
    segger_rtt.o(i.SEGGER_RTT_ReadNoLock) refers to memcpya.o(.text) for __aeabi_memcpy
    segger_rtt.o(i.SEGGER_RTT_ReadNoLock) refers to segger_rtt.o(.bss) for .bss
    segger_rtt.o(i.SEGGER_RTT_SetFlagsDownBuffer) refers to segger_rtt.o(i._DoInit) for _DoInit
    segger_rtt.o(i.SEGGER_RTT_SetFlagsDownBuffer) refers to app_util_platform.o(i.app_util_critical_region_enter) for app_util_critical_region_enter
    segger_rtt.o(i.SEGGER_RTT_SetFlagsDownBuffer) refers to app_util_platform.o(i.app_util_critical_region_exit) for app_util_critical_region_exit
    segger_rtt.o(i.SEGGER_RTT_SetFlagsDownBuffer) refers to segger_rtt.o(.bss) for .bss
    segger_rtt.o(i.SEGGER_RTT_SetFlagsUpBuffer) refers to segger_rtt.o(i._DoInit) for _DoInit
    segger_rtt.o(i.SEGGER_RTT_SetFlagsUpBuffer) refers to app_util_platform.o(i.app_util_critical_region_enter) for app_util_critical_region_enter
    segger_rtt.o(i.SEGGER_RTT_SetFlagsUpBuffer) refers to app_util_platform.o(i.app_util_critical_region_exit) for app_util_critical_region_exit
    segger_rtt.o(i.SEGGER_RTT_SetFlagsUpBuffer) refers to segger_rtt.o(.bss) for .bss
    segger_rtt.o(i.SEGGER_RTT_SetNameDownBuffer) refers to segger_rtt.o(i._DoInit) for _DoInit
    segger_rtt.o(i.SEGGER_RTT_SetNameDownBuffer) refers to app_util_platform.o(i.app_util_critical_region_enter) for app_util_critical_region_enter
    segger_rtt.o(i.SEGGER_RTT_SetNameDownBuffer) refers to app_util_platform.o(i.app_util_critical_region_exit) for app_util_critical_region_exit
    segger_rtt.o(i.SEGGER_RTT_SetNameDownBuffer) refers to segger_rtt.o(.bss) for .bss
    segger_rtt.o(i.SEGGER_RTT_SetNameUpBuffer) refers to segger_rtt.o(i._DoInit) for _DoInit
    segger_rtt.o(i.SEGGER_RTT_SetNameUpBuffer) refers to app_util_platform.o(i.app_util_critical_region_enter) for app_util_critical_region_enter
    segger_rtt.o(i.SEGGER_RTT_SetNameUpBuffer) refers to app_util_platform.o(i.app_util_critical_region_exit) for app_util_critical_region_exit
    segger_rtt.o(i.SEGGER_RTT_SetNameUpBuffer) refers to segger_rtt.o(.bss) for .bss
    segger_rtt.o(i.SEGGER_RTT_SetTerminal) refers to segger_rtt.o(i._DoInit) for _DoInit
    segger_rtt.o(i.SEGGER_RTT_SetTerminal) refers to app_util_platform.o(i.app_util_critical_region_enter) for app_util_critical_region_enter
    segger_rtt.o(i.SEGGER_RTT_SetTerminal) refers to segger_rtt.o(i._GetAvailWriteSpace) for _GetAvailWriteSpace
    segger_rtt.o(i.SEGGER_RTT_SetTerminal) refers to segger_rtt.o(i._WriteNoCheck) for _WriteNoCheck
    segger_rtt.o(i.SEGGER_RTT_SetTerminal) refers to segger_rtt.o(i._WriteBlocking) for _WriteBlocking
    segger_rtt.o(i.SEGGER_RTT_SetTerminal) refers to app_util_platform.o(i.app_util_critical_region_exit) for app_util_critical_region_exit
    segger_rtt.o(i.SEGGER_RTT_SetTerminal) refers to segger_rtt.o(.bss) for .bss
    segger_rtt.o(i.SEGGER_RTT_SetTerminal) refers to segger_rtt.o(.data) for .data
    segger_rtt.o(i.SEGGER_RTT_TerminalOut) refers to segger_rtt.o(i._DoInit) for _DoInit
    segger_rtt.o(i.SEGGER_RTT_TerminalOut) refers to strlen.o(.text) for strlen
    segger_rtt.o(i.SEGGER_RTT_TerminalOut) refers to app_util_platform.o(i.app_util_critical_region_enter) for app_util_critical_region_enter
    segger_rtt.o(i.SEGGER_RTT_TerminalOut) refers to segger_rtt.o(i._GetAvailWriteSpace) for _GetAvailWriteSpace
    segger_rtt.o(i.SEGGER_RTT_TerminalOut) refers to segger_rtt.o(i._PostTerminalSwitch) for _PostTerminalSwitch
    segger_rtt.o(i.SEGGER_RTT_TerminalOut) refers to segger_rtt.o(i._WriteBlocking) for _WriteBlocking
    segger_rtt.o(i.SEGGER_RTT_TerminalOut) refers to app_util_platform.o(i.app_util_critical_region_exit) for app_util_critical_region_exit
    segger_rtt.o(i.SEGGER_RTT_TerminalOut) refers to segger_rtt.o(.bss) for .bss
    segger_rtt.o(i.SEGGER_RTT_TerminalOut) refers to segger_rtt.o(.data) for .data
    segger_rtt.o(i.SEGGER_RTT_WaitKey) refers to segger_rtt.o(i.SEGGER_RTT_GetKey) for SEGGER_RTT_GetKey
    segger_rtt.o(i.SEGGER_RTT_Write) refers to segger_rtt.o(i._DoInit) for _DoInit
    segger_rtt.o(i.SEGGER_RTT_Write) refers to app_util_platform.o(i.app_util_critical_region_enter) for app_util_critical_region_enter
    segger_rtt.o(i.SEGGER_RTT_Write) refers to segger_rtt.o(i.SEGGER_RTT_WriteNoLock) for SEGGER_RTT_WriteNoLock
    segger_rtt.o(i.SEGGER_RTT_Write) refers to app_util_platform.o(i.app_util_critical_region_exit) for app_util_critical_region_exit
    segger_rtt.o(i.SEGGER_RTT_Write) refers to segger_rtt.o(.bss) for .bss
    segger_rtt.o(i.SEGGER_RTT_WriteNoLock) refers to segger_rtt.o(i._GetAvailWriteSpace) for _GetAvailWriteSpace
    segger_rtt.o(i.SEGGER_RTT_WriteNoLock) refers to segger_rtt.o(i._WriteNoCheck) for _WriteNoCheck
    segger_rtt.o(i.SEGGER_RTT_WriteNoLock) refers to segger_rtt.o(i._WriteBlocking) for _WriteBlocking
    segger_rtt.o(i.SEGGER_RTT_WriteNoLock) refers to segger_rtt.o(.bss) for .bss
    segger_rtt.o(i.SEGGER_RTT_WriteSkipNoLock) refers to memcpya.o(.text) for __aeabi_memcpy
    segger_rtt.o(i.SEGGER_RTT_WriteSkipNoLock) refers to segger_rtt.o(.bss) for .bss
    segger_rtt.o(i.SEGGER_RTT_WriteString) refers to strlen.o(.text) for strlen
    segger_rtt.o(i.SEGGER_RTT_WriteString) refers to segger_rtt.o(i.SEGGER_RTT_Write) for SEGGER_RTT_Write
    segger_rtt.o(i.SEGGER_RTT_WriteWithOverwriteNoLock) refers to memcpya.o(.text) for __aeabi_memcpy
    segger_rtt.o(i.SEGGER_RTT_WriteWithOverwriteNoLock) refers to segger_rtt.o(.bss) for .bss
    segger_rtt.o(i._DoInit) refers to strcpy.o(.text) for strcpy
    segger_rtt.o(i._DoInit) refers to segger_rtt.o(.bss) for .bss
    segger_rtt.o(i._PostTerminalSwitch) refers to segger_rtt.o(i._WriteBlocking) for _WriteBlocking
    segger_rtt.o(i._PostTerminalSwitch) refers to segger_rtt.o(.data) for .data
    segger_rtt.o(i._WriteBlocking) refers to memcpya.o(.text) for __aeabi_memcpy
    segger_rtt.o(i._WriteNoCheck) refers to memcpya.o(.text) for __aeabi_memcpy
    segger_rtt_printf.o(i.SEGGER_RTT_printf) refers to segger_rtt_printf.o(i.SEGGER_RTT_vprintf) for SEGGER_RTT_vprintf
    segger_rtt_printf.o(i.SEGGER_RTT_vprintf) refers to segger_rtt_printf.o(i._StoreChar) for _StoreChar
    segger_rtt_printf.o(i.SEGGER_RTT_vprintf) refers to segger_rtt_printf.o(i._PrintInt) for _PrintInt
    segger_rtt_printf.o(i.SEGGER_RTT_vprintf) refers to segger_rtt_printf.o(i._PrintUnsigned) for _PrintUnsigned
    segger_rtt_printf.o(i.SEGGER_RTT_vprintf) refers to segger_rtt.o(i.SEGGER_RTT_Write) for SEGGER_RTT_Write
    segger_rtt_printf.o(i._PrintInt) refers to segger_rtt_printf.o(i._StoreChar) for _StoreChar
    segger_rtt_printf.o(i._PrintInt) refers to segger_rtt_printf.o(i._PrintUnsigned) for _PrintUnsigned
    segger_rtt_printf.o(i._PrintUnsigned) refers to segger_rtt_printf.o(i._StoreChar) for _StoreChar
    segger_rtt_printf.o(i._PrintUnsigned) refers to segger_rtt_printf.o(.constdata) for .constdata
    segger_rtt_printf.o(i._StoreChar) refers to segger_rtt.o(i.SEGGER_RTT_Write) for SEGGER_RTT_Write
    nrf_sdh.o(i.SWI2_IRQHandler) refers to nrf_sdh.o(i.nrf_sdh_evts_poll) for nrf_sdh_evts_poll
    nrf_sdh.o(i.nrf_sdh_disable_request) refers to nrf_sdh.o(i.sdh_request_observer_notify) for sdh_request_observer_notify
    nrf_sdh.o(i.nrf_sdh_disable_request) refers to nrf_sdh.o(i.sdh_state_observer_notify) for sdh_state_observer_notify
    nrf_sdh.o(i.nrf_sdh_disable_request) refers to app_util_platform.o(i.app_util_critical_region_enter) for app_util_critical_region_enter
    nrf_sdh.o(i.nrf_sdh_disable_request) refers to app_util_platform.o(i.app_util_critical_region_exit) for app_util_critical_region_exit
    nrf_sdh.o(i.nrf_sdh_disable_request) refers to nrf_sdh.o(i.softdevice_evt_irq_disable) for softdevice_evt_irq_disable
    nrf_sdh.o(i.nrf_sdh_disable_request) refers to nrf_sdh.o(.data) for .data
    nrf_sdh.o(i.nrf_sdh_enable_request) refers to nrf_sdh.o(i.sdh_request_observer_notify) for sdh_request_observer_notify
    nrf_sdh.o(i.nrf_sdh_enable_request) refers to nrf_sdh.o(i.sdh_state_observer_notify) for sdh_state_observer_notify
    nrf_sdh.o(i.nrf_sdh_enable_request) refers to app_util_platform.o(i.app_util_critical_region_enter) for app_util_critical_region_enter
    nrf_sdh.o(i.nrf_sdh_enable_request) refers to app_util_platform.o(i.app_util_critical_region_exit) for app_util_critical_region_exit
    nrf_sdh.o(i.nrf_sdh_enable_request) refers to nrf_sdh.o(i.softdevices_evt_irq_enable) for softdevices_evt_irq_enable
    nrf_sdh.o(i.nrf_sdh_enable_request) refers to nrf_sdh.o(.data) for .data
    nrf_sdh.o(i.nrf_sdh_enable_request) refers to nrf_sdh.o(.constdata) for .constdata
    nrf_sdh.o(i.nrf_sdh_enable_request) refers to app_error_weak.o(i.app_error_fault_handler) for app_error_fault_handler
    nrf_sdh.o(i.nrf_sdh_evts_poll) refers to nrf_section_iter.o(i.nrf_section_iter_init) for nrf_section_iter_init
    nrf_sdh.o(i.nrf_sdh_evts_poll) refers to nrf_section_iter.o(i.nrf_section_iter_next) for nrf_section_iter_next
    nrf_sdh.o(i.nrf_sdh_evts_poll) refers to nrf_sdh.o(.constdata) for .constdata
    nrf_sdh.o(i.nrf_sdh_is_enabled) refers to nrf_sdh.o(.data) for .data
    nrf_sdh.o(i.nrf_sdh_is_suspended) refers to nrf_sdh.o(.data) for .data
    nrf_sdh.o(i.nrf_sdh_request_continue) refers to nrf_sdh.o(i.nrf_sdh_disable_request) for nrf_sdh_disable_request
    nrf_sdh.o(i.nrf_sdh_request_continue) refers to nrf_sdh.o(i.nrf_sdh_enable_request) for nrf_sdh_enable_request
    nrf_sdh.o(i.nrf_sdh_request_continue) refers to nrf_sdh.o(.data) for .data
    nrf_sdh.o(i.nrf_sdh_resume) refers to nrf_sdh.o(i.__sd_nvic_app_accessible_irq) for __sd_nvic_app_accessible_irq
    nrf_sdh.o(i.nrf_sdh_resume) refers to app_error.o(i.app_error_handler_bare) for app_error_handler_bare
    nrf_sdh.o(i.nrf_sdh_resume) refers to nrf_sdh.o(i.softdevices_evt_irq_enable) for softdevices_evt_irq_enable
    nrf_sdh.o(i.nrf_sdh_resume) refers to nrf_sdh.o(.data) for .data
    nrf_sdh.o(i.nrf_sdh_suspend) refers to nrf_sdh.o(i.softdevice_evt_irq_disable) for softdevice_evt_irq_disable
    nrf_sdh.o(i.nrf_sdh_suspend) refers to nrf_sdh.o(.data) for .data
    nrf_sdh.o(i.sdh_request_observer_notify) refers to nrf_section_iter.o(i.nrf_section_iter_init) for nrf_section_iter_init
    nrf_sdh.o(i.sdh_request_observer_notify) refers to nrf_section_iter.o(i.nrf_section_iter_next) for nrf_section_iter_next
    nrf_sdh.o(i.sdh_request_observer_notify) refers to nrf_sdh.o(.constdata) for .constdata
    nrf_sdh.o(i.sdh_state_observer_notify) refers to nrf_section_iter.o(i.nrf_section_iter_init) for nrf_section_iter_init
    nrf_sdh.o(i.sdh_state_observer_notify) refers to nrf_section_iter.o(i.nrf_section_iter_next) for nrf_section_iter_next
    nrf_sdh.o(i.sdh_state_observer_notify) refers to nrf_sdh.o(.constdata) for .constdata
    nrf_sdh.o(i.softdevice_evt_irq_disable) refers to nrf_sdh.o(i.__sd_nvic_app_accessible_irq) for __sd_nvic_app_accessible_irq
    nrf_sdh.o(i.softdevice_evt_irq_disable) refers to app_error.o(i.app_error_handler_bare) for app_error_handler_bare
    nrf_sdh.o(i.softdevice_evt_irq_disable) refers to app_util_platform.o(.bss) for nrf_nvic_state
    nrf_sdh.o(i.softdevices_evt_irq_enable) refers to nrf_sdh.o(i.__sd_nvic_app_accessible_irq) for __sd_nvic_app_accessible_irq
    nrf_sdh.o(i.softdevices_evt_irq_enable) refers to app_error.o(i.app_error_handler_bare) for app_error_handler_bare
    nrf_sdh.o(i.softdevices_evt_irq_enable) refers to app_util_platform.o(.bss) for nrf_nvic_state
    nrf_sdh.o(.constdata) refers to nrf_sdh.o(.constdata) for sdh_req_observers_array
    nrf_sdh.o(.constdata) refers to nrf_sdh.o(.constdata) for sdh_state_observers_array
    nrf_sdh.o(.constdata) refers to nrf_sdh.o(.constdata) for sdh_stack_observers_array
    nrf_sdh.o(log_const_data) refers to nrf_sdh.o(.conststrlit) for .conststrlit
    nrf_sdh_ble.o(i.nrf_sdh_ble_app_ram_start_get) refers to nrf_sdh_ble.o(.constdata) for .constdata
    nrf_sdh_ble.o(i.nrf_sdh_ble_default_cfg_set) refers to nrf_sdh_ble.o(i.nrf_sdh_ble_app_ram_start_get) for nrf_sdh_ble_app_ram_start_get
    nrf_sdh_ble.o(i.nrf_sdh_ble_default_cfg_set) refers to nrf_strerror.o(i.nrf_strerror_get) for nrf_strerror_get
    nrf_sdh_ble.o(i.nrf_sdh_ble_default_cfg_set) refers to nrf_log_frontend.o(i.nrf_log_frontend_std_1) for nrf_log_frontend_std_1
    nrf_sdh_ble.o(i.nrf_sdh_ble_default_cfg_set) refers to nrf_sdh_ble.o(log_const_data) for log_const_data
    nrf_sdh_ble.o(i.nrf_sdh_ble_default_cfg_set) refers to nrf_sdh_ble.o(.conststring) for .conststring
    nrf_sdh_ble.o(i.nrf_sdh_ble_enable) refers to nrf_log_frontend.o(i.nrf_log_frontend_std_0) for nrf_log_frontend_std_0
    nrf_sdh_ble.o(i.nrf_sdh_ble_enable) refers to nrf_log_frontend.o(i.nrf_log_frontend_std_2) for nrf_log_frontend_std_2
    nrf_sdh_ble.o(i.nrf_sdh_ble_enable) refers to nrf_log_frontend.o(i.nrf_log_frontend_std_1) for nrf_log_frontend_std_1
    nrf_sdh_ble.o(i.nrf_sdh_ble_enable) refers to nrf_strerror.o(i.nrf_strerror_get) for nrf_strerror_get
    nrf_sdh_ble.o(i.nrf_sdh_ble_enable) refers to nrf_sdh_ble.o(log_const_data) for log_const_data
    nrf_sdh_ble.o(i.nrf_sdh_ble_enable) refers to nrf_sdh_ble.o(.data) for .data
    nrf_sdh_ble.o(i.nrf_sdh_ble_evts_poll) refers to app_error.o(i.app_error_handler_bare) for app_error_handler_bare
    nrf_sdh_ble.o(i.nrf_sdh_ble_evts_poll) refers to nrf_section_iter.o(i.nrf_section_iter_init) for nrf_section_iter_init
    nrf_sdh_ble.o(i.nrf_sdh_ble_evts_poll) refers to nrf_section_iter.o(i.nrf_section_iter_next) for nrf_section_iter_next
    nrf_sdh_ble.o(i.nrf_sdh_ble_evts_poll) refers to nrf_sdh_ble.o(.data) for .data
    nrf_sdh_ble.o(i.nrf_sdh_ble_evts_poll) refers to nrf_sdh_ble.o(.constdata) for .constdata
    nrf_sdh_ble.o(.constdata) refers to nrf_sdh_ble.o(.constdata) for sdh_ble_observers_array
    nrf_sdh_ble.o(log_const_data) refers to nrf_sdh_ble.o(.conststrlit) for .conststrlit
    nrf_sdh_ble.o(sdh_stack_observers0) refers to nrf_sdh_ble.o(i.nrf_sdh_ble_evts_poll) for nrf_sdh_ble_evts_poll
    nrf_sdh_soc.o(i.nrf_sdh_soc_evts_poll) refers to app_error.o(i.app_error_handler_bare) for app_error_handler_bare
    nrf_sdh_soc.o(i.nrf_sdh_soc_evts_poll) refers to nrf_section_iter.o(i.nrf_section_iter_init) for nrf_section_iter_init
    nrf_sdh_soc.o(i.nrf_sdh_soc_evts_poll) refers to nrf_section_iter.o(i.nrf_section_iter_next) for nrf_section_iter_next
    nrf_sdh_soc.o(i.nrf_sdh_soc_evts_poll) refers to nrf_sdh_soc.o(.constdata) for .constdata
    nrf_sdh_soc.o(.constdata) refers to nrf_sdh_soc.o(.constdata) for sdh_soc_observers_array
    nrf_sdh_soc.o(log_const_data) refers to nrf_sdh_soc.o(.conststrlit) for .conststrlit
    nrf_sdh_soc.o(sdh_stack_observers0) refers to nrf_sdh_soc.o(i.nrf_sdh_soc_evts_poll) for nrf_sdh_soc_evts_poll
    arm_startup_nrf52810.o(RESET) refers to arm_startup_nrf52810.o(STACK) for __initial_sp
    arm_startup_nrf52810.o(RESET) refers to arm_startup_nrf52810.o(.text) for Reset_Handler
    arm_startup_nrf52810.o(RESET) refers to nrfx_clock.o(i.POWER_CLOCK_IRQHandler) for POWER_CLOCK_IRQHandler
    arm_startup_nrf52810.o(RESET) refers to nrfx_uarte.o(i.UARTE0_IRQHandler) for UARTE0_IRQHandler
    arm_startup_nrf52810.o(RESET) refers to nrfx_twim.o(i.TWIM0_TWIS0_IRQHandler) for TWIM0_TWIS0_IRQHandler
    arm_startup_nrf52810.o(RESET) refers to nrfx_gpiote.o(i.GPIOTE_IRQHandler) for GPIOTE_IRQHandler
    arm_startup_nrf52810.o(RESET) refers to app_timer.o(i.RTC1_IRQHandler) for RTC1_IRQHandler
    arm_startup_nrf52810.o(RESET) refers to app_timer.o(i.SWI0_EGU0_IRQHandler) for SWI0_EGU0_IRQHandler
    arm_startup_nrf52810.o(RESET) refers to nrf_sdh.o(i.SWI2_IRQHandler) for SWI2_IRQHandler
    arm_startup_nrf52810.o(.text) refers to system_nrf52810.o(i.SystemInit) for SystemInit
    arm_startup_nrf52810.o(.text) refers to entry.o(.ARM.Collect$$$$00000000) for __main
    system_nrf52810.o(i.SystemCoreClockUpdate) refers to system_nrf52810.o(.data) for .data
    system_nrf52810.o(i.SystemInit) refers to system_nrf52810.o(.data) for .data
    entry.o(.ARM.Collect$$$$00000000) refers (Special) to entry10a.o(.ARM.Collect$$$$0000000D) for __rt_final_cpp
    entry.o(.ARM.Collect$$$$00000000) refers (Special) to entry11a.o(.ARM.Collect$$$$0000000F) for __rt_final_exit
    entry.o(.ARM.Collect$$$$00000000) refers (Special) to entry7b.o(.ARM.Collect$$$$00000008) for _main_clock
    entry.o(.ARM.Collect$$$$00000000) refers (Special) to entry8b.o(.ARM.Collect$$$$0000000A) for _main_cpp_init
    entry.o(.ARM.Collect$$$$00000000) refers (Special) to entry9a.o(.ARM.Collect$$$$0000000B) for _main_init
    entry.o(.ARM.Collect$$$$00000000) refers (Special) to entry5.o(.ARM.Collect$$$$00000004) for _main_scatterload
    entry.o(.ARM.Collect$$$$00000000) refers (Special) to entry2.o(.ARM.Collect$$$$00000001) for _main_stk
    uldiv.o(.text) refers to llushr.o(.text) for __aeabi_llsr
    uldiv.o(.text) refers to llshl.o(.text) for __aeabi_llsl
    ctype_o.o(.text) refers to ctype_o.o(.constdata) for .constdata
    ctype_o.o(.constdata) refers to ctype_o.o(.constdata) for __ctype_table
    isalnum_o.o(.text) refers to ctype_o.o(.text) for __rt_ctype_table
    isalpha_o.o(.text) refers to ctype_o.o(.text) for __rt_ctype_table
    isblank_o.o(.text) refers to ctype_o.o(.constdata) for __ctype_table
    iscntrl_o.o(.text) refers to ctype_o.o(.text) for __rt_ctype_table
    isdigit_o.o(.text) refers to ctype_o.o(.text) for __rt_ctype_table
    isgraph_o.o(.text) refers to ctype_o.o(.text) for __rt_ctype_table
    islower_o.o(.text) refers to ctype_o.o(.text) for __rt_ctype_table
    isprint_o.o(.text) refers to ctype_o.o(.text) for __rt_ctype_table
    ispunct_o.o(.text) refers to ctype_o.o(.text) for __rt_ctype_table
    isspace_o.o(.text) refers to ctype_o.o(.text) for __rt_ctype_table
    isupper_o.o(.text) refers to ctype_o.o(.text) for __rt_ctype_table
    isxdigit_o.o(.text) refers to ctype_o.o(.text) for __rt_ctype_table
    malloc.o(i.free) refers to mvars.o(.data) for __microlib_freelist
    malloc.o(i.malloc) refers to mvars.o(.data) for __microlib_freelist_initialised
    malloc.o(i.malloc) refers to mvars.o(.data) for __microlib_freelist
    malloc.o(i.malloc) refers to arm_startup_nrf52810.o(HEAP) for __heap_base
    mallocr.o(i.__free$realloc) refers to mvars.o(.data) for __microlib_freelist
    mallocr.o(i.__malloc$realloc) refers to mallocr.o(i.internal_alloc) for internal_alloc
    mallocr.o(i.__malloc$realloc) refers to mvars.o(.data) for __microlib_freelist_initialised
    mallocr.o(i.__malloc$realloc) refers to arm_startup_nrf52810.o(HEAP) for __heap_base
    mallocr.o(i.__malloc$realloc) refers to mvars.o(.data) for __microlib_freelist
    mallocr.o(i.internal_alloc) refers to memcpya.o(.text) for __aeabi_memcpy
    mallocr.o(i.internal_alloc) refers to mvars.o(.data) for __microlib_freelist
    mallocr.o(i.realloc) refers to mallocr.o(i.__free$realloc) for __free$realloc
    mallocr.o(i.realloc) refers to mallocr.o(i.internal_alloc) for internal_alloc
    mallocr.o(i.realloc) refers to mallocr.o(i.__malloc$realloc) for __malloc$realloc
    mallocr.o(i.realloc) refers to mvars.o(.data) for __microlib_freelist
    malloca.o(i.__aligned_malloc) refers to mvars.o(.data) for __microlib_freelist_initialised
    malloca.o(i.__aligned_malloc) refers to mvars.o(.data) for __microlib_freelist
    malloca.o(i.__aligned_malloc) refers to arm_startup_nrf52810.o(HEAP) for __heap_base
    malloca.o(i.__free$memalign) refers to mvars.o(.data) for __microlib_freelist
    malloca.o(i.__malloc$memalign) refers to malloca.o(i.__aligned_malloc) for __aligned_malloc
    mallocra.o(i.__aligned_malloc$realloc) refers to mallocra.o(i.internal_alloc) for internal_alloc
    mallocra.o(i.__aligned_malloc$realloc) refers to mvars.o(.data) for __microlib_freelist_initialised
    mallocra.o(i.__aligned_malloc$realloc) refers to arm_startup_nrf52810.o(HEAP) for __heap_base
    mallocra.o(i.__aligned_malloc$realloc) refers to mvars.o(.data) for __microlib_freelist
    mallocra.o(i.__free$realloc$memalign) refers to mvars.o(.data) for __microlib_freelist
    mallocra.o(i.__malloc$realloc$memalign) refers to mallocra.o(i.__aligned_malloc$realloc) for __aligned_malloc$realloc
    mallocra.o(i.__realloc$memalign) refers to mallocra.o(i.__free$realloc$memalign) for __free$realloc$memalign
    mallocra.o(i.__realloc$memalign) refers to mallocra.o(i.internal_alloc) for internal_alloc
    mallocra.o(i.__realloc$memalign) refers to mallocra.o(i.__malloc$realloc$memalign) for __malloc$realloc$memalign
    mallocra.o(i.__realloc$memalign) refers to mvars.o(.data) for __microlib_freelist
    mallocra.o(i.internal_alloc) refers to memcpya.o(.text) for __aeabi_memcpy
    mallocra.o(i.internal_alloc) refers to mvars.o(.data) for __microlib_freelist
    fadd.o(.text) refers (Special) to iusefp.o(.text) for __I$use$fp
    fadd.o(.text) refers to fepilogue.o(.text) for _float_epilogue
    fscalb.o(.text) refers (Special) to iusefp.o(.text) for __I$use$fp
    ffltui.o(.text) refers (Special) to iusefp.o(.text) for __I$use$fp
    ffltui.o(.text) refers to fepilogue.o(.text) for _float_epilogue
    ffixui.o(.text) refers (Special) to iusefp.o(.text) for __I$use$fp
    entry2.o(.ARM.Collect$$$$00000001) refers to entry2.o(.ARM.Collect$$$$00002712) for __lit__00000000
    entry2.o(.ARM.Collect$$$$00002712) refers to arm_startup_nrf52810.o(STACK) for __initial_sp
    entry2.o(__vectab_stack_and_reset_area) refers to arm_startup_nrf52810.o(STACK) for __initial_sp
    entry2.o(__vectab_stack_and_reset_area) refers to entry.o(.ARM.Collect$$$$00000000) for __main
    entry5.o(.ARM.Collect$$$$00000004) refers to init.o(.text) for __scatterload
    entry9a.o(.ARM.Collect$$$$0000000B) refers to main.o(i.main) for main
    entry9b.o(.ARM.Collect$$$$0000000C) refers to main.o(i.main) for main
    init.o(.text) refers to entry5.o(.ARM.Collect$$$$00000004) for __main_after_scatterload


==============================================================================

Removing Unused input sections from the image.

    Removing main.o(.rev16_text), (4 bytes).
    Removing main.o(.revsh_text), (4 bytes).
    Removing main.o(.rrx_text), (6 bytes).
    Removing main.o(i.assert_nrf_callback), (16 bytes).
    Removing main.o(i.bsp_event_handler), (76 bytes).
    Removing main.o(.constdata), (1 bytes).
    Removing main.o(.constdata), (1 bytes).
    Removing main.o(.constdata), (1 bytes).
    Removing main.o(.constdata), (1 bytes).
    Removing main.o(.constdata), (1 bytes).
    Removing main.o(.constdata), (1 bytes).
    Removing main.o(.constdata), (1 bytes).
    Removing main.o(.constdata), (1 bytes).
    Removing main.o(.constdata), (1 bytes).
    Removing main.o(.constdata), (1 bytes).
    Removing main.o(.constdata), (1 bytes).
    Removing main.o(.constdata), (1 bytes).
    Removing main.o(.constdata), (1 bytes).
    Removing main.o(.constdata), (1 bytes).
    Removing boards.o(.rev16_text), (4 bytes).
    Removing boards.o(.revsh_text), (4 bytes).
    Removing boards.o(.rrx_text), (6 bytes).
    Removing boards.o(i.bsp_board_button_state_get), (32 bytes).
    Removing boards.o(i.bsp_board_init), (84 bytes).
    Removing boards.o(i.bsp_board_led_idx_to_pin), (12 bytes).
    Removing boards.o(i.bsp_board_pin_to_led_idx), (36 bytes).
    Removing boards.o(i.nrf_gpio_cfg), (36 bytes).
    Removing bsp.o(.rev16_text), (4 bytes).
    Removing bsp.o(.revsh_text), (4 bytes).
    Removing bsp.o(.rrx_text), (6 bytes).
    Removing bsp.o(i.alert_timer_handler), (6 bytes).
    Removing bsp.o(i.bsp_button_is_pressed), (12 bytes).
    Removing bsp.o(i.bsp_buttons_disable), (4 bytes).
    Removing bsp.o(i.bsp_buttons_enable), (4 bytes).
    Removing bsp.o(i.bsp_init), (148 bytes).
    Removing bsp.o(i.bsp_wakeup_button_disable), (6 bytes).
    Removing bsp.o(i.button_timer_handler), (8 bytes).
    Removing bsp.o(i.leds_timer_handler), (20 bytes).
    Removing bsp_btn_ble.o(.rev16_text), (4 bytes).
    Removing bsp_btn_ble.o(.revsh_text), (4 bytes).
    Removing bsp_btn_ble.o(.rrx_text), (6 bytes).
    Removing bsp_btn_ble.o(i.bsp_btn_ble_init), (56 bytes).
    Removing utf.o(i.utf16DecodeRune), (74 bytes).
    Removing utf.o(i.utf16EncodeRune), (64 bytes).
    Removing utf.o(i.utf16RuneCount), (60 bytes).
    Removing utf.o(i.utf16UTF8Count), (78 bytes).
    Removing utf.o(i.utf8DecodeRune), (174 bytes).
    Removing utf.o(i.utf8EncodeRune), (160 bytes).
    Removing utf.o(i.utf8RuneCount), (58 bytes).
    Removing utf.o(i.utf8UTF16Count), (76 bytes).
    Removing ble_advdata.o(.rev16_text), (4 bytes).
    Removing ble_advdata.o(.revsh_text), (4 bytes).
    Removing ble_advdata.o(.rrx_text), (6 bytes).
    Removing ble_advdata.o(i.ble_advdata_appearance_find), (52 bytes).
    Removing ble_advdata.o(i.ble_advdata_name_find), (68 bytes).
    Removing ble_advdata.o(i.ble_advdata_short_name_find), (74 bytes).
    Removing ble_advdata.o(i.ble_advdata_uuid_find), (182 bytes).
    Removing ble_advertising.o(.rev16_text), (4 bytes).
    Removing ble_advertising.o(.revsh_text), (4 bytes).
    Removing ble_advertising.o(.rrx_text), (6 bytes).
    Removing ble_advertising.o(i.ble_advertising_advdata_update), (32 bytes).
    Removing ble_advertising.o(i.ble_advertising_modes_config_set), (8 bytes).
    Removing ble_advertising.o(i.ble_advertising_peer_addr_reply), (34 bytes).
    Removing ble_advertising.o(i.ble_advertising_restart_without_whitelist), (58 bytes).
    Removing ble_advertising.o(i.ble_advertising_whitelist_reply), (36 bytes).
    Removing ble_conn_params.o(.rev16_text), (4 bytes).
    Removing ble_conn_params.o(.revsh_text), (4 bytes).
    Removing ble_conn_params.o(.rrx_text), (6 bytes).
    Removing ble_conn_params.o(i.ble_conn_params_change_conn_params), (64 bytes).
    Removing ble_conn_params.o(i.ble_conn_params_stop), (36 bytes).
    Removing ble_conn_state.o(.rev16_text), (4 bytes).
    Removing ble_conn_state.o(.revsh_text), (4 bytes).
    Removing ble_conn_state.o(.rrx_text), (6 bytes).
    Removing ble_conn_state.o(i.active_flag_count), (28 bytes).
    Removing ble_conn_state.o(i.bcs_internal_state_reset), (12 bytes).
    Removing ble_conn_state.o(i.ble_conn_state_central_conn_count), (28 bytes).
    Removing ble_conn_state.o(i.ble_conn_state_central_handles), (32 bytes).
    Removing ble_conn_state.o(i.ble_conn_state_conn_count), (12 bytes).
    Removing ble_conn_state.o(i.ble_conn_state_conn_handles), (12 bytes).
    Removing ble_conn_state.o(i.ble_conn_state_encrypted), (32 bytes).
    Removing ble_conn_state.o(i.ble_conn_state_for_each_connected), (20 bytes).
    Removing ble_conn_state.o(i.ble_conn_state_for_each_set_user_flag), (44 bytes).
    Removing ble_conn_state.o(i.ble_conn_state_init), (4 bytes).
    Removing ble_conn_state.o(i.ble_conn_state_mitm_protected), (32 bytes).
    Removing ble_conn_state.o(i.ble_conn_state_periph_handles), (36 bytes).
    Removing ble_conn_state.o(i.ble_conn_state_peripheral_conn_count), (32 bytes).
    Removing ble_conn_state.o(i.ble_conn_state_role), (16 bytes).
    Removing ble_conn_state.o(i.ble_conn_state_status), (36 bytes).
    Removing ble_conn_state.o(i.ble_conn_state_user_flag_acquire), (24 bytes).
    Removing ble_conn_state.o(i.ble_conn_state_user_flag_get), (48 bytes).
    Removing ble_conn_state.o(i.ble_conn_state_user_flag_set), (64 bytes).
    Removing ble_conn_state.o(i.for_each_set_flag), (48 bytes).
    Removing ble_conn_state.o(i.user_flag_is_acquired), (12 bytes).
    Removing ble_link_ctx_manager.o(.rev16_text), (4 bytes).
    Removing ble_link_ctx_manager.o(.revsh_text), (4 bytes).
    Removing ble_link_ctx_manager.o(.rrx_text), (6 bytes).
    Removing ble_srv_common.o(.rev16_text), (4 bytes).
    Removing ble_srv_common.o(.revsh_text), (4 bytes).
    Removing ble_srv_common.o(.rrx_text), (6 bytes).
    Removing ble_srv_common.o(i.ble_srv_ascii_to_utf8), (18 bytes).
    Removing ble_srv_common.o(i.ble_srv_is_indication_enabled), (8 bytes).
    Removing ble_srv_common.o(i.ble_srv_report_ref_encode), (12 bytes).
    Removing ble_srv_common.o(i.descriptor_add), (170 bytes).
    Removing nrf_ble_gatt.o(.rev16_text), (4 bytes).
    Removing nrf_ble_gatt.o(.revsh_text), (4 bytes).
    Removing nrf_ble_gatt.o(.rrx_text), (6 bytes).
    Removing nrf_ble_gatt.o(i.nrf_ble_gatt_att_mtu_central_set), (24 bytes).
    Removing nrf_ble_gatt.o(i.nrf_ble_gatt_eff_mtu_get), (12 bytes).
    Removing nrf_ble_qwr.o(.rev16_text), (4 bytes).
    Removing nrf_ble_qwr.o(.revsh_text), (4 bytes).
    Removing nrf_ble_qwr.o(.rrx_text), (6 bytes).
    Removing nrf_ble_qwr.o(i.nrf_ble_qwr_conn_handle_assign), (22 bytes).
    Removing ble_nus.o(.rev16_text), (4 bytes).
    Removing ble_nus.o(.revsh_text), (4 bytes).
    Removing ble_nus.o(.rrx_text), (6 bytes).
    Removing nrf_drv_clock.o(.rev16_text), (4 bytes).
    Removing nrf_drv_clock.o(.revsh_text), (4 bytes).
    Removing nrf_drv_clock.o(.rrx_text), (6 bytes).
    Removing nrf_drv_clock.o(i.item_enqueue), (22 bytes).
    Removing nrf_drv_clock.o(i.nrf_drv_clock_calibration_abort), (4 bytes).
    Removing nrf_drv_clock.o(i.nrf_drv_clock_calibration_start), (4 bytes).
    Removing nrf_drv_clock.o(i.nrf_drv_clock_hfclk_is_running), (44 bytes).
    Removing nrf_drv_clock.o(i.nrf_drv_clock_hfclk_release), (56 bytes).
    Removing nrf_drv_clock.o(i.nrf_drv_clock_hfclk_request), (92 bytes).
    Removing nrf_drv_clock.o(i.nrf_drv_clock_init_check), (12 bytes).
    Removing nrf_drv_clock.o(i.nrf_drv_clock_is_calibrating), (4 bytes).
    Removing nrf_drv_clock.o(i.nrf_drv_clock_lfclk_is_running), (28 bytes).
    Removing nrf_drv_clock.o(i.nrf_drv_clock_lfclk_request), (84 bytes).
    Removing nrf_drv_clock.o(i.nrf_drv_clock_uninit), (24 bytes).
    Removing nrf_drv_clock.o(.constdata), (19 bytes).
    Removing nrf_drv_clock.o(.constdata), (32 bytes).
    Removing nrf_drv_clock.o(.constdata), (32 bytes).
    Removing nrf_drv_clock.o(.constdata), (29 bytes).
    Removing nrf_drv_uart.o(.rev16_text), (4 bytes).
    Removing nrf_drv_uart.o(.revsh_text), (4 bytes).
    Removing nrf_drv_uart.o(.rrx_text), (6 bytes).
    Removing nrfx_clock.o(.rev16_text), (4 bytes).
    Removing nrfx_clock.o(.revsh_text), (4 bytes).
    Removing nrfx_clock.o(.rrx_text), (6 bytes).
    Removing nrfx_clock.o(i.nrfx_clock_calibration_start), (4 bytes).
    Removing nrfx_clock.o(i.nrfx_clock_calibration_timer_start), (44 bytes).
    Removing nrfx_clock.o(i.nrfx_clock_calibration_timer_stop), (20 bytes).
    Removing nrfx_clock.o(i.nrfx_clock_disable), (22 bytes).
    Removing nrfx_clock.o(i.nrfx_clock_hfclk_start), (22 bytes).
    Removing nrfx_clock.o(i.nrfx_clock_hfclk_stop), (44 bytes).
    Removing nrfx_clock.o(i.nrfx_clock_is_calibrating), (4 bytes).
    Removing nrfx_clock.o(i.nrfx_clock_lfclk_start), (32 bytes).
    Removing nrfx_clock.o(i.nrfx_clock_uninit), (24 bytes).
    Removing nrfx_clock.o(.constdata), (16 bytes).
    Removing nrfx_clock.o(.constdata), (29 bytes).
    Removing nrfx_gpiote.o(.rev16_text), (4 bytes).
    Removing nrfx_gpiote.o(.revsh_text), (4 bytes).
    Removing nrfx_gpiote.o(.rrx_text), (6 bytes).
    Removing nrfx_gpiote.o(i.channel_free), (28 bytes).
    Removing nrfx_gpiote.o(i.channel_port_alloc), (72 bytes).
    Removing nrfx_gpiote.o(i.nrf_gpio_cfg), (36 bytes).
    Removing nrfx_gpiote.o(i.nrf_gpio_cfg_default), (18 bytes).
    Removing nrfx_gpiote.o(i.nrfx_gpiote_clr_task_addr_get), (24 bytes).
    Removing nrfx_gpiote.o(i.nrfx_gpiote_clr_task_trigger), (28 bytes).
    Removing nrfx_gpiote.o(i.nrfx_gpiote_in_event_addr_get), (40 bytes).
    Removing nrfx_gpiote.o(i.nrfx_gpiote_in_event_disable), (72 bytes).
    Removing nrfx_gpiote.o(i.nrfx_gpiote_in_event_enable), (164 bytes).
    Removing nrfx_gpiote.o(i.nrfx_gpiote_in_init), (208 bytes).
    Removing nrfx_gpiote.o(i.nrfx_gpiote_in_is_set), (20 bytes).
    Removing nrfx_gpiote.o(i.nrfx_gpiote_in_uninit), (88 bytes).
    Removing nrfx_gpiote.o(i.nrfx_gpiote_init), (112 bytes).
    Removing nrfx_gpiote.o(i.nrfx_gpiote_is_init), (20 bytes).
    Removing nrfx_gpiote.o(i.nrfx_gpiote_out_clear), (14 bytes).
    Removing nrfx_gpiote.o(i.nrfx_gpiote_out_init), (192 bytes).
    Removing nrfx_gpiote.o(i.nrfx_gpiote_out_set), (14 bytes).
    Removing nrfx_gpiote.o(i.nrfx_gpiote_out_task_addr_get), (20 bytes).
    Removing nrfx_gpiote.o(i.nrfx_gpiote_out_task_disable), (36 bytes).
    Removing nrfx_gpiote.o(i.nrfx_gpiote_out_task_enable), (36 bytes).
    Removing nrfx_gpiote.o(i.nrfx_gpiote_out_task_force), (40 bytes).
    Removing nrfx_gpiote.o(i.nrfx_gpiote_out_task_trigger), (24 bytes).
    Removing nrfx_gpiote.o(i.nrfx_gpiote_out_toggle), (28 bytes).
    Removing nrfx_gpiote.o(i.nrfx_gpiote_out_uninit), (88 bytes).
    Removing nrfx_gpiote.o(i.nrfx_gpiote_set_task_addr_get), (24 bytes).
    Removing nrfx_gpiote.o(i.nrfx_gpiote_set_task_trigger), (28 bytes).
    Removing nrfx_gpiote.o(i.nrfx_gpiote_uninit), (56 bytes).
    Removing nrfx_gpiote.o(i.pin_configured_check), (20 bytes).
    Removing nrfx_gpiote.o(i.pin_configured_clear), (28 bytes).
    Removing nrfx_gpiote.o(i.pin_in_use_by_port), (24 bytes).
    Removing nrfx_gpiote.o(i.pin_in_use_by_te), (24 bytes).
    Removing nrfx_gpiote.o(.constdata), (17 bytes).
    Removing nrfx_gpiote.o(.constdata), (21 bytes).
    Removing nrfx_gpiote.o(.constdata), (20 bytes).
    Removing nrfx_power_clock.o(.rev16_text), (4 bytes).
    Removing nrfx_power_clock.o(.revsh_text), (4 bytes).
    Removing nrfx_power_clock.o(.rrx_text), (6 bytes).
    Removing nrfx_prs.o(.rev16_text), (4 bytes).
    Removing nrfx_prs.o(.revsh_text), (4 bytes).
    Removing nrfx_prs.o(.rrx_text), (6 bytes).
    Removing nrfx_prs.o(i.nrfx_prs_release), (2 bytes).
    Removing nrfx_prs.o(.constdata), (17 bytes).
    Removing nrfx_uarte.o(.rev16_text), (4 bytes).
    Removing nrfx_uarte.o(.revsh_text), (4 bytes).
    Removing nrfx_uarte.o(.rrx_text), (6 bytes).
    Removing nrfx_uarte.o(i.nrf_gpio_cfg_default), (18 bytes).
    Removing nrfx_uarte.o(i.nrfx_uarte_errorsrc_get), (26 bytes).
    Removing nrfx_uarte.o(i.nrfx_uarte_rx_abort), (8 bytes).
    Removing nrfx_uarte.o(i.nrfx_uarte_rx_ready), (14 bytes).
    Removing nrfx_uarte.o(i.nrfx_uarte_tx_abort), (56 bytes).
    Removing nrfx_uarte.o(i.nrfx_uarte_uninit), (176 bytes).
    Removing nrfx_uarte.o(.constdata), (16 bytes).
    Removing nrfx_uarte.o(.constdata), (14 bytes).
    Removing nrfx_uarte.o(.constdata), (14 bytes).
    Removing nrfx_twi.o(.rev16_text), (4 bytes).
    Removing nrfx_twi.o(.revsh_text), (4 bytes).
    Removing nrfx_twi.o(.rrx_text), (6 bytes).
    Removing nrfx_twim.o(.rev16_text), (4 bytes).
    Removing nrfx_twim.o(.revsh_text), (4 bytes).
    Removing nrfx_twim.o(.rrx_text), (6 bytes).
    Removing nrfx_twim.o(i.nrf_gpio_cfg_default), (18 bytes).
    Removing nrfx_twim.o(i.nrfx_twim_disable), (60 bytes).
    Removing nrfx_twim.o(i.nrfx_twim_is_busy), (28 bytes).
    Removing nrfx_twim.o(i.nrfx_twim_start_task_get), (16 bytes).
    Removing nrfx_twim.o(i.nrfx_twim_stopped_event_get), (8 bytes).
    Removing nrfx_twim.o(i.nrfx_twim_uninit), (100 bytes).
    Removing nrfx_twim.o(.constdata), (15 bytes).
    Removing nrfx_twim.o(.constdata), (10 bytes).
    Removing nrfx_twim.o(.constdata), (15 bytes).
    Removing nrf_drv_twi.o(.rev16_text), (4 bytes).
    Removing nrf_drv_twi.o(.revsh_text), (4 bytes).
    Removing nrf_drv_twi.o(.rrx_text), (6 bytes).
    Removing app_button.o(.rev16_text), (4 bytes).
    Removing app_button.o(.revsh_text), (4 bytes).
    Removing app_button.o(.rrx_text), (6 bytes).
    Removing app_button.o(i.app_button_disable), (48 bytes).
    Removing app_button.o(i.app_button_enable), (36 bytes).
    Removing app_button.o(i.app_button_init), (120 bytes).
    Removing app_button.o(i.app_button_is_pushed), (36 bytes).
    Removing app_button.o(i.detection_delay_timeout_handler), (152 bytes).
    Removing app_button.o(i.gpiote_event_handler), (132 bytes).
    Removing app_button.o(.bss), (32 bytes).
    Removing app_button.o(.constdata), (8 bytes).
    Removing app_button.o(.data), (32 bytes).
    Removing app_error.o(.rev16_text), (4 bytes).
    Removing app_error.o(.revsh_text), (4 bytes).
    Removing app_error.o(.rrx_text), (6 bytes).
    Removing app_error.o(i.app_error_save_and_stop), (100 bytes).
    Removing app_error.o(.bss), (32 bytes).
    Removing app_error_handler_keil.o(.rev16_text), (4 bytes).
    Removing app_error_handler_keil.o(.revsh_text), (4 bytes).
    Removing app_error_handler_keil.o(.rrx_text), (6 bytes).
    Removing app_error_handler_keil.o(.emb_text), (26 bytes).
    Removing app_error_weak.o(.rev16_text), (4 bytes).
    Removing app_error_weak.o(.revsh_text), (4 bytes).
    Removing app_error_weak.o(.rrx_text), (6 bytes).
    Removing app_fifo.o(.rev16_text), (4 bytes).
    Removing app_fifo.o(.revsh_text), (4 bytes).
    Removing app_fifo.o(.rrx_text), (6 bytes).
    Removing app_fifo.o(i.app_fifo_flush), (8 bytes).
    Removing app_fifo.o(i.app_fifo_peek), (34 bytes).
    Removing app_fifo.o(i.app_fifo_read), (74 bytes).
    Removing app_fifo.o(i.app_fifo_write), (82 bytes).
    Removing app_scheduler.o(.rev16_text), (4 bytes).
    Removing app_scheduler.o(.revsh_text), (4 bytes).
    Removing app_scheduler.o(.rrx_text), (6 bytes).
    Removing app_scheduler.o(i.app_sched_event_put), (160 bytes).
    Removing app_scheduler.o(i.app_sched_execute), (64 bytes).
    Removing app_scheduler.o(i.app_sched_init), (44 bytes).
    Removing app_scheduler.o(i.app_sched_queue_space_get), (36 bytes).
    Removing app_scheduler.o(.data), (16 bytes).
    Removing app_timer.o(.rev16_text), (4 bytes).
    Removing app_timer.o(.revsh_text), (4 bytes).
    Removing app_timer.o(.rrx_text), (6 bytes).
    Removing app_timer.o(i.app_timer_cnt_diff_compute), (8 bytes).
    Removing app_timer.o(i.app_timer_cnt_get), (12 bytes).
    Removing app_timer.o(i.app_timer_pause), (12 bytes).
    Removing app_timer.o(i.app_timer_resume), (12 bytes).
    Removing app_timer.o(i.app_timer_stop_all), (24 bytes).
    Removing app_uart_fifo.o(.rev16_text), (4 bytes).
    Removing app_uart_fifo.o(.revsh_text), (4 bytes).
    Removing app_uart_fifo.o(.rrx_text), (6 bytes).
    Removing app_uart_fifo.o(i.app_uart_close), (16 bytes).
    Removing app_uart_fifo.o(i.app_uart_flush), (32 bytes).
    Removing app_uart_fifo.o(i.app_uart_put), (64 bytes).
    Removing app_util_platform.o(.rev16_text), (4 bytes).
    Removing app_util_platform.o(.revsh_text), (4 bytes).
    Removing app_util_platform.o(.rrx_text), (6 bytes).
    Removing app_util_platform.o(i.app_util_disable_irq), (16 bytes).
    Removing app_util_platform.o(i.app_util_enable_irq), (20 bytes).
    Removing app_util_platform.o(i.current_int_priority_get), (48 bytes).
    Removing app_util_platform.o(i.privilege_level_get), (26 bytes).
    Removing app_util_platform.o(.data), (4 bytes).
    Removing hardfault_implementation.o(.rev16_text), (4 bytes).
    Removing hardfault_implementation.o(.revsh_text), (4 bytes).
    Removing hardfault_implementation.o(.rrx_text), (6 bytes).
    Removing nrf_assert.o(.rev16_text), (4 bytes).
    Removing nrf_assert.o(.revsh_text), (4 bytes).
    Removing nrf_assert.o(.rrx_text), (6 bytes).
    Removing nrf_assert.o(i.assert_nrf_callback), (22 bytes).
    Removing nrf_atfifo.o(.rev16_text), (4 bytes).
    Removing nrf_atfifo.o(.revsh_text), (4 bytes).
    Removing nrf_atfifo.o(.rrx_text), (6 bytes).
    Removing nrf_atfifo.o(.emb_text), (200 bytes).
    Removing nrf_atfifo.o(i.nrf_atfifo_alloc_put), (46 bytes).
    Removing nrf_atfifo.o(i.nrf_atfifo_clear), (16 bytes).
    Removing nrf_atfifo.o(i.nrf_atfifo_get_free), (48 bytes).
    Removing nrf_atfifo.o(i.nrf_atfifo_init), (38 bytes).
    Removing nrf_atfifo.o(i.nrf_atfifo_item_alloc), (22 bytes).
    Removing nrf_atfifo.o(i.nrf_atfifo_item_free), (22 bytes).
    Removing nrf_atfifo.o(i.nrf_atfifo_item_get), (22 bytes).
    Removing nrf_atfifo.o(i.nrf_atfifo_item_put), (22 bytes).
    Removing nrf_atflags.o(.rev16_text), (4 bytes).
    Removing nrf_atflags.o(.revsh_text), (4 bytes).
    Removing nrf_atflags.o(.rrx_text), (6 bytes).
    Removing nrf_atflags.o(i.nrf_atflags_fetch_clear), (32 bytes).
    Removing nrf_atflags.o(i.nrf_atflags_fetch_set), (32 bytes).
    Removing nrf_atflags.o(i.nrf_atflags_find_and_clear_flag), (72 bytes).
    Removing nrf_atflags.o(i.nrf_atflags_find_and_set_flag), (74 bytes).
    Removing nrf_atflags.o(i.nrf_atflags_init), (36 bytes).
    Removing nrf_atomic.o(.rev16_text), (4 bytes).
    Removing nrf_atomic.o(.revsh_text), (4 bytes).
    Removing nrf_atomic.o(.rrx_text), (6 bytes).
    Removing nrf_atomic.o(i.nrf_atomic_flag_clear), (6 bytes).
    Removing nrf_atomic.o(i.nrf_atomic_flag_set_fetch), (6 bytes).
    Removing nrf_atomic.o(i.nrf_atomic_u32_cmp_exch), (4 bytes).
    Removing nrf_atomic.o(i.nrf_atomic_u32_fetch_add), (10 bytes).
    Removing nrf_atomic.o(i.nrf_atomic_u32_fetch_or), (10 bytes).
    Removing nrf_atomic.o(i.nrf_atomic_u32_fetch_sub), (10 bytes).
    Removing nrf_atomic.o(i.nrf_atomic_u32_fetch_sub_hs), (10 bytes).
    Removing nrf_atomic.o(i.nrf_atomic_u32_fetch_xor), (10 bytes).
    Removing nrf_atomic.o(i.nrf_atomic_u32_store), (12 bytes).
    Removing nrf_atomic.o(i.nrf_atomic_u32_sub_hs), (12 bytes).
    Removing nrf_atomic.o(i.nrf_atomic_u32_xor), (12 bytes).
    Removing nrf_balloc.o(.rev16_text), (4 bytes).
    Removing nrf_balloc.o(.revsh_text), (4 bytes).
    Removing nrf_balloc.o(.rrx_text), (6 bytes).
    Removing nrf_fprintf.o(.rev16_text), (4 bytes).
    Removing nrf_fprintf.o(.revsh_text), (4 bytes).
    Removing nrf_fprintf.o(.rrx_text), (6 bytes).
    Removing nrf_fprintf_format.o(.rev16_text), (4 bytes).
    Removing nrf_fprintf_format.o(.revsh_text), (4 bytes).
    Removing nrf_fprintf_format.o(.rrx_text), (6 bytes).
    Removing nrf_memobj.o(.rev16_text), (4 bytes).
    Removing nrf_memobj.o(.revsh_text), (4 bytes).
    Removing nrf_memobj.o(.rrx_text), (6 bytes).
    Removing nrf_pwr_mgmt.o(.rev16_text), (4 bytes).
    Removing nrf_pwr_mgmt.o(.revsh_text), (4 bytes).
    Removing nrf_pwr_mgmt.o(.rrx_text), (6 bytes).
    Removing nrf_pwr_mgmt.o(i.nrf_pwr_mgmt_feed), (2 bytes).
    Removing nrf_pwr_mgmt.o(i.nrf_pwr_mgmt_shutdown), (60 bytes).
    Removing nrf_pwr_mgmt.o(i.shutdown_process), (124 bytes).
    Removing nrf_ringbuf.o(.rev16_text), (4 bytes).
    Removing nrf_ringbuf.o(.revsh_text), (4 bytes).
    Removing nrf_ringbuf.o(.rrx_text), (6 bytes).
    Removing nrf_ringbuf.o(i.nrf_ringbuf_alloc), (112 bytes).
    Removing nrf_ringbuf.o(i.nrf_ringbuf_cpy_get), (124 bytes).
    Removing nrf_ringbuf.o(i.nrf_ringbuf_cpy_put), (114 bytes).
    Removing nrf_ringbuf.o(i.nrf_ringbuf_free), (38 bytes).
    Removing nrf_ringbuf.o(i.nrf_ringbuf_get), (112 bytes).
    Removing nrf_ringbuf.o(i.nrf_ringbuf_put), (48 bytes).
    Removing nrf_section_iter.o(.rev16_text), (4 bytes).
    Removing nrf_section_iter.o(.revsh_text), (4 bytes).
    Removing nrf_section_iter.o(.rrx_text), (6 bytes).
    Removing nrf_strerror.o(.rev16_text), (4 bytes).
    Removing nrf_strerror.o(.revsh_text), (4 bytes).
    Removing nrf_strerror.o(.rrx_text), (6 bytes).
    Removing retarget.o(.rev16_text), (4 bytes).
    Removing retarget.o(.revsh_text), (4 bytes).
    Removing retarget.o(.rrx_text), (6 bytes).
    Removing retarget.o(i.fgetc), (18 bytes).
    Removing retarget.o(i.fputc), (14 bytes).
    Removing retarget.o(.data), (4 bytes).
    Removing retarget.o(.data), (4 bytes).
    Removing nrf_log_backend_rtt.o(.rev16_text), (4 bytes).
    Removing nrf_log_backend_rtt.o(.revsh_text), (4 bytes).
    Removing nrf_log_backend_rtt.o(.rrx_text), (6 bytes).
    Removing nrf_log_backend_serial.o(.rev16_text), (4 bytes).
    Removing nrf_log_backend_serial.o(.revsh_text), (4 bytes).
    Removing nrf_log_backend_serial.o(.rrx_text), (6 bytes).
    Removing nrf_log_default_backends.o(.rev16_text), (4 bytes).
    Removing nrf_log_default_backends.o(.revsh_text), (4 bytes).
    Removing nrf_log_default_backends.o(.rrx_text), (6 bytes).
    Removing nrf_log_frontend.o(.rev16_text), (4 bytes).
    Removing nrf_log_frontend.o(.revsh_text), (4 bytes).
    Removing nrf_log_frontend.o(.rrx_text), (6 bytes).
    Removing nrf_log_frontend.o(i.nrf_log_backend_remove), (52 bytes).
    Removing nrf_log_frontend.o(i.nrf_log_frontend_hexdump), (168 bytes).
    Removing nrf_log_frontend.o(i.nrf_log_frontend_std_3), (18 bytes).
    Removing nrf_log_frontend.o(i.nrf_log_frontend_std_4), (20 bytes).
    Removing nrf_log_frontend.o(i.nrf_log_frontend_std_5), (28 bytes).
    Removing nrf_log_frontend.o(i.nrf_log_frontend_std_6), (28 bytes).
    Removing nrf_log_frontend.o(i.nrf_log_module_filter_get), (36 bytes).
    Removing nrf_log_frontend.o(i.nrf_log_module_filter_set), (2 bytes).
    Removing nrf_log_frontend.o(i.nrf_log_push), (96 bytes).
    Removing nrf_log_str_formatter.o(.rev16_text), (4 bytes).
    Removing nrf_log_str_formatter.o(.revsh_text), (4 bytes).
    Removing nrf_log_str_formatter.o(.rrx_text), (6 bytes).
    Removing nrf_log_str_formatter.o(i.nrf_log_str_formatter_timestamp_freq_set), (32 bytes).
    Removing segger_rtt.o(.rev16_text), (4 bytes).
    Removing segger_rtt.o(.revsh_text), (4 bytes).
    Removing segger_rtt.o(.rrx_text), (6 bytes).
    Removing segger_rtt.o(i.SEGGER_RTT_AllocDownBuffer), (112 bytes).
    Removing segger_rtt.o(i.SEGGER_RTT_AllocUpBuffer), (112 bytes).
    Removing segger_rtt.o(i.SEGGER_RTT_ConfigDownBuffer), (96 bytes).
    Removing segger_rtt.o(i.SEGGER_RTT_ConfigUpBuffer), (96 bytes).
    Removing segger_rtt.o(i.SEGGER_RTT_GetKey), (28 bytes).
    Removing segger_rtt.o(i.SEGGER_RTT_HasData), (24 bytes).
    Removing segger_rtt.o(i.SEGGER_RTT_HasKey), (32 bytes).
    Removing segger_rtt.o(i.SEGGER_RTT_PutChar), (96 bytes).
    Removing segger_rtt.o(i.SEGGER_RTT_PutCharSkip), (84 bytes).
    Removing segger_rtt.o(i.SEGGER_RTT_PutCharSkipNoLock), (52 bytes).
    Removing segger_rtt.o(i.SEGGER_RTT_Read), (44 bytes).
    Removing segger_rtt.o(i.SEGGER_RTT_ReadNoLock), (120 bytes).
    Removing segger_rtt.o(i.SEGGER_RTT_SetFlagsDownBuffer), (68 bytes).
    Removing segger_rtt.o(i.SEGGER_RTT_SetFlagsUpBuffer), (68 bytes).
    Removing segger_rtt.o(i.SEGGER_RTT_SetNameDownBuffer), (68 bytes).
    Removing segger_rtt.o(i.SEGGER_RTT_SetNameUpBuffer), (68 bytes).
    Removing segger_rtt.o(i.SEGGER_RTT_SetTerminal), (136 bytes).
    Removing segger_rtt.o(i.SEGGER_RTT_TerminalOut), (176 bytes).
    Removing segger_rtt.o(i.SEGGER_RTT_WaitKey), (14 bytes).
    Removing segger_rtt.o(i.SEGGER_RTT_Write), (60 bytes).
    Removing segger_rtt.o(i.SEGGER_RTT_WriteSkipNoLock), (116 bytes).
    Removing segger_rtt.o(i.SEGGER_RTT_WriteString), (26 bytes).
    Removing segger_rtt.o(i.SEGGER_RTT_WriteWithOverwriteNoLock), (148 bytes).
    Removing segger_rtt.o(i._PostTerminalSwitch), (32 bytes).
    Removing segger_rtt.o(.data), (17 bytes).
    Removing segger_rtt_printf.o(.rev16_text), (4 bytes).
    Removing segger_rtt_printf.o(.revsh_text), (4 bytes).
    Removing segger_rtt_printf.o(.rrx_text), (6 bytes).
    Removing segger_rtt_printf.o(i.SEGGER_RTT_printf), (22 bytes).
    Removing segger_rtt_printf.o(i.SEGGER_RTT_vprintf), (406 bytes).
    Removing segger_rtt_printf.o(i._PrintInt), (198 bytes).
    Removing segger_rtt_printf.o(i._PrintUnsigned), (212 bytes).
    Removing segger_rtt_printf.o(i._StoreChar), (62 bytes).
    Removing segger_rtt_printf.o(.constdata), (16 bytes).
    Removing nrf_sdh.o(.rev16_text), (4 bytes).
    Removing nrf_sdh.o(.revsh_text), (4 bytes).
    Removing nrf_sdh.o(.rrx_text), (6 bytes).
    Removing nrf_sdh.o(i.nrf_sdh_disable_request), (84 bytes).
    Removing nrf_sdh.o(i.nrf_sdh_is_suspended), (20 bytes).
    Removing nrf_sdh.o(i.nrf_sdh_request_continue), (28 bytes).
    Removing nrf_sdh.o(i.nrf_sdh_resume), (56 bytes).
    Removing nrf_sdh.o(i.nrf_sdh_suspend), (24 bytes).
    Removing nrf_sdh.o(i.softdevice_evt_irq_disable), (56 bytes).
    Removing nrf_sdh_ble.o(.rev16_text), (4 bytes).
    Removing nrf_sdh_ble.o(.revsh_text), (4 bytes).
    Removing nrf_sdh_ble.o(.rrx_text), (6 bytes).
    Removing nrf_sdh_soc.o(.rev16_text), (4 bytes).
    Removing nrf_sdh_soc.o(.revsh_text), (4 bytes).
    Removing nrf_sdh_soc.o(.rrx_text), (6 bytes).
    Removing system_nrf52810.o(.rev16_text), (4 bytes).
    Removing system_nrf52810.o(.revsh_text), (4 bytes).
    Removing system_nrf52810.o(.rrx_text), (6 bytes).
    Removing system_nrf52810.o(i.SystemCoreClockUpdate), (16 bytes).

448 unused section(s) (total 13375 bytes) removed from the image.

==============================================================================

Image Symbol Table

    Local Symbols

    Symbol Name                              Value     Ov Type        Size  Object(Section)

    ../clib/microlib/ctype/ctype.c           0x00000000   Number         0  isalpha_o.o ABSOLUTE
    ../clib/microlib/ctype/ctype.c           0x00000000   Number         0  isprint_o.o ABSOLUTE
    ../clib/microlib/ctype/ctype.c           0x00000000   Number         0  iscntrl_o.o ABSOLUTE
    ../clib/microlib/ctype/ctype.c           0x00000000   Number         0  ctype_o.o ABSOLUTE
    ../clib/microlib/ctype/ctype.c           0x00000000   Number         0  isalnum_o.o ABSOLUTE
    ../clib/microlib/ctype/ctype.c           0x00000000   Number         0  isgraph_o.o ABSOLUTE
    ../clib/microlib/ctype/ctype.c           0x00000000   Number         0  isxdigit_o.o ABSOLUTE
    ../clib/microlib/ctype/ctype.c           0x00000000   Number         0  isblank_o.o ABSOLUTE
    ../clib/microlib/ctype/ctype.c           0x00000000   Number         0  isupper_o.o ABSOLUTE
    ../clib/microlib/ctype/ctype.c           0x00000000   Number         0  isdigit_o.o ABSOLUTE
    ../clib/microlib/ctype/ctype.c           0x00000000   Number         0  isspace_o.o ABSOLUTE
    ../clib/microlib/ctype/ctype.c           0x00000000   Number         0  islower_o.o ABSOLUTE
    ../clib/microlib/ctype/ctype.c           0x00000000   Number         0  ispunct_o.o ABSOLUTE
    ../clib/microlib/division.c              0x00000000   Number         0  uldiv.o ABSOLUTE
    ../clib/microlib/init/entry.s            0x00000000   Number         0  entry2.o ABSOLUTE
    ../clib/microlib/init/entry.s            0x00000000   Number         0  entry11b.o ABSOLUTE
    ../clib/microlib/init/entry.s            0x00000000   Number         0  entry7a.o ABSOLUTE
    ../clib/microlib/init/entry.s            0x00000000   Number         0  entry10b.o ABSOLUTE
    ../clib/microlib/init/entry.s            0x00000000   Number         0  entry11a.o ABSOLUTE
    ../clib/microlib/init/entry.s            0x00000000   Number         0  entry10a.o ABSOLUTE
    ../clib/microlib/init/entry.s            0x00000000   Number         0  entry9b.o ABSOLUTE
    ../clib/microlib/init/entry.s            0x00000000   Number         0  entry9a.o ABSOLUTE
    ../clib/microlib/init/entry.s            0x00000000   Number         0  entry8b.o ABSOLUTE
    ../clib/microlib/init/entry.s            0x00000000   Number         0  entry8a.o ABSOLUTE
    ../clib/microlib/init/entry.s            0x00000000   Number         0  entry7b.o ABSOLUTE
    ../clib/microlib/init/entry.s            0x00000000   Number         0  entry.o ABSOLUTE
    ../clib/microlib/init/entry.s            0x00000000   Number         0  entry5.o ABSOLUTE
    ../clib/microlib/longlong.c              0x00000000   Number         0  llushr.o ABSOLUTE
    ../clib/microlib/longlong.c              0x00000000   Number         0  llshl.o ABSOLUTE
    ../clib/microlib/malloc/malloc.c         0x00000000   Number         0  mallocr.o ABSOLUTE
    ../clib/microlib/malloc/malloc.c         0x00000000   Number         0  malloc.o ABSOLUTE
    ../clib/microlib/malloc/malloc.c         0x00000000   Number         0  mallocra.o ABSOLUTE
    ../clib/microlib/malloc/malloc.c         0x00000000   Number         0  malloca.o ABSOLUTE
    ../clib/microlib/malloc/mvars.c          0x00000000   Number         0  mvars.o ABSOLUTE
    ../clib/microlib/string/memcmp.c         0x00000000   Number         0  memcmp.o ABSOLUTE
    ../clib/microlib/string/memcpy.c         0x00000000   Number         0  memcpya.o ABSOLUTE
    ../clib/microlib/string/memcpy.c         0x00000000   Number         0  memcpyb.o ABSOLUTE
    ../clib/microlib/string/memset.c         0x00000000   Number         0  memseta.o ABSOLUTE
    ../clib/microlib/string/strcpy.c         0x00000000   Number         0  strcpy.o ABSOLUTE
    ../clib/microlib/string/strlen.c         0x00000000   Number         0  strlen.o ABSOLUTE
    ../clib/microlib/stubs.s                 0x00000000   Number         0  iusefp.o ABSOLUTE
    ../fplib/microlib/fpadd.c                0x00000000   Number         0  fadd.o ABSOLUTE
    ../fplib/microlib/fpepilogue.c           0x00000000   Number         0  fepilogue.o ABSOLUTE
    ../fplib/microlib/fpfix.c                0x00000000   Number         0  ffixui.o ABSOLUTE
    ../fplib/microlib/fpflt.c                0x00000000   Number         0  ffltui.o ABSOLUTE
    ../fplib/microlib/fpscalb.c              0x00000000   Number         0  fscalb.o ABSOLUTE
    ..\..\..\..\..\..\components\ble\ble_advertising\ble_advertising.c 0x00000000   Number         0  ble_advertising.o ABSOLUTE
    ..\..\..\..\..\..\components\ble\ble_link_ctx_manager\ble_link_ctx_manager.c 0x00000000   Number         0  ble_link_ctx_manager.o ABSOLUTE
    ..\..\..\..\..\..\components\ble\ble_services\ble_nus\ble_nus.c 0x00000000   Number         0  ble_nus.o ABSOLUTE
    ..\..\..\..\..\..\components\ble\common\ble_advdata.c 0x00000000   Number         0  ble_advdata.o ABSOLUTE
    ..\..\..\..\..\..\components\ble\common\ble_conn_params.c 0x00000000   Number         0  ble_conn_params.o ABSOLUTE
    ..\..\..\..\..\..\components\ble\common\ble_conn_state.c 0x00000000   Number         0  ble_conn_state.o ABSOLUTE
    ..\..\..\..\..\..\components\ble\common\ble_srv_common.c 0x00000000   Number         0  ble_srv_common.o ABSOLUTE
    ..\..\..\..\..\..\components\ble\nrf_ble_gatt\nrf_ble_gatt.c 0x00000000   Number         0  nrf_ble_gatt.o ABSOLUTE
    ..\..\..\..\..\..\components\ble\nrf_ble_qwr\nrf_ble_qwr.c 0x00000000   Number         0  nrf_ble_qwr.o ABSOLUTE
    ..\..\..\..\..\..\components\boards\boards.c 0x00000000   Number         0  boards.o ABSOLUTE
    ..\..\..\..\..\..\components\libraries\atomic\nrf_atomic.c 0x00000000   Number         0  nrf_atomic.o ABSOLUTE
    ..\..\..\..\..\..\components\libraries\atomic_fifo\nrf_atfifo.c 0x00000000   Number         0  nrf_atfifo.o ABSOLUTE
    ..\..\..\..\..\..\components\libraries\atomic_flags\nrf_atflags.c 0x00000000   Number         0  nrf_atflags.o ABSOLUTE
    ..\..\..\..\..\..\components\libraries\balloc\nrf_balloc.c 0x00000000   Number         0  nrf_balloc.o ABSOLUTE
    ..\..\..\..\..\..\components\libraries\bsp\bsp.c 0x00000000   Number         0  bsp.o ABSOLUTE
    ..\..\..\..\..\..\components\libraries\bsp\bsp_btn_ble.c 0x00000000   Number         0  bsp_btn_ble.o ABSOLUTE
    ..\..\..\..\..\..\components\libraries\button\app_button.c 0x00000000   Number         0  app_button.o ABSOLUTE
    ..\..\..\..\..\..\components\libraries\experimental_section_vars\nrf_section_iter.c 0x00000000   Number         0  nrf_section_iter.o ABSOLUTE
    ..\..\..\..\..\..\components\libraries\fifo\app_fifo.c 0x00000000   Number         0  app_fifo.o ABSOLUTE
    ..\..\..\..\..\..\components\libraries\hardfault\hardfault_implementation.c 0x00000000   Number         0  hardfault_implementation.o ABSOLUTE
    ..\..\..\..\..\..\components\libraries\log\src\nrf_log_backend_rtt.c 0x00000000   Number         0  nrf_log_backend_rtt.o ABSOLUTE
    ..\..\..\..\..\..\components\libraries\log\src\nrf_log_backend_serial.c 0x00000000   Number         0  nrf_log_backend_serial.o ABSOLUTE
    ..\..\..\..\..\..\components\libraries\log\src\nrf_log_default_backends.c 0x00000000   Number         0  nrf_log_default_backends.o ABSOLUTE
    ..\..\..\..\..\..\components\libraries\log\src\nrf_log_frontend.c 0x00000000   Number         0  nrf_log_frontend.o ABSOLUTE
    ..\..\..\..\..\..\components\libraries\log\src\nrf_log_str_formatter.c 0x00000000   Number         0  nrf_log_str_formatter.o ABSOLUTE
    ..\..\..\..\..\..\components\libraries\memobj\nrf_memobj.c 0x00000000   Number         0  nrf_memobj.o ABSOLUTE
    ..\..\..\..\..\..\components\libraries\pwr_mgmt\nrf_pwr_mgmt.c 0x00000000   Number         0  nrf_pwr_mgmt.o ABSOLUTE
    ..\..\..\..\..\..\components\libraries\ringbuf\nrf_ringbuf.c 0x00000000   Number         0  nrf_ringbuf.o ABSOLUTE
    ..\..\..\..\..\..\components\libraries\scheduler\app_scheduler.c 0x00000000   Number         0  app_scheduler.o ABSOLUTE
    ..\..\..\..\..\..\components\libraries\strerror\nrf_strerror.c 0x00000000   Number         0  nrf_strerror.o ABSOLUTE
    ..\..\..\..\..\..\components\libraries\timer\app_timer.c 0x00000000   Number         0  app_timer.o ABSOLUTE
    ..\..\..\..\..\..\components\libraries\uart\app_uart_fifo.c 0x00000000   Number         0  app_uart_fifo.o ABSOLUTE
    ..\..\..\..\..\..\components\libraries\uart\retarget.c 0x00000000   Number         0  retarget.o ABSOLUTE
    ..\..\..\..\..\..\components\libraries\util\app_error.c 0x00000000   Number         0  app_error.o ABSOLUTE
    ..\..\..\..\..\..\components\libraries\util\app_error_handler_keil.c 0x00000000   Number         0  app_error_handler_keil.o ABSOLUTE
    ..\..\..\..\..\..\components\libraries\util\app_error_weak.c 0x00000000   Number         0  app_error_weak.o ABSOLUTE
    ..\..\..\..\..\..\components\libraries\util\app_util_platform.c 0x00000000   Number         0  app_util_platform.o ABSOLUTE
    ..\..\..\..\..\..\components\libraries\util\nrf_assert.c 0x00000000   Number         0  nrf_assert.o ABSOLUTE
    ..\..\..\..\..\..\components\softdevice\common\nrf_sdh.c 0x00000000   Number         0  nrf_sdh.o ABSOLUTE
    ..\..\..\..\..\..\components\softdevice\common\nrf_sdh_ble.c 0x00000000   Number         0  nrf_sdh_ble.o ABSOLUTE
    ..\..\..\..\..\..\components\softdevice\common\nrf_sdh_soc.c 0x00000000   Number         0  nrf_sdh_soc.o ABSOLUTE
    ..\..\..\..\..\..\external\fprintf\nrf_fprintf.c 0x00000000   Number         0  nrf_fprintf.o ABSOLUTE
    ..\..\..\..\..\..\external\fprintf\nrf_fprintf_format.c 0x00000000   Number         0  nrf_fprintf_format.o ABSOLUTE
    ..\..\..\..\..\..\external\segger_rtt\SEGGER_RTT.c 0x00000000   Number         0  segger_rtt.o ABSOLUTE
    ..\..\..\..\..\..\external\segger_rtt\SEGGER_RTT_Syscalls_KEIL.c 0x00000000   Number         0  segger_rtt_syscalls_keil.o ABSOLUTE
    ..\..\..\..\..\..\external\segger_rtt\SEGGER_RTT_printf.c 0x00000000   Number         0  segger_rtt_printf.o ABSOLUTE
    ..\..\..\..\..\..\external\utf_converter\utf.c 0x00000000   Number         0  utf.o ABSOLUTE
    ..\..\..\..\..\..\integration\nrfx\legacy\nrf_drv_clock.c 0x00000000   Number         0  nrf_drv_clock.o ABSOLUTE
    ..\..\..\..\..\..\integration\nrfx\legacy\nrf_drv_twi.c 0x00000000   Number         0  nrf_drv_twi.o ABSOLUTE
    ..\..\..\..\..\..\integration\nrfx\legacy\nrf_drv_uart.c 0x00000000   Number         0  nrf_drv_uart.o ABSOLUTE
    ..\..\..\..\..\..\modules\nrfx\drivers\src\nrfx_clock.c 0x00000000   Number         0  nrfx_clock.o ABSOLUTE
    ..\..\..\..\..\..\modules\nrfx\drivers\src\nrfx_gpiote.c 0x00000000   Number         0  nrfx_gpiote.o ABSOLUTE
    ..\..\..\..\..\..\modules\nrfx\drivers\src\nrfx_power_clock.c 0x00000000   Number         0  nrfx_power_clock.o ABSOLUTE
    ..\..\..\..\..\..\modules\nrfx\drivers\src\nrfx_twi.c 0x00000000   Number         0  nrfx_twi.o ABSOLUTE
    ..\..\..\..\..\..\modules\nrfx\drivers\src\nrfx_twim.c 0x00000000   Number         0  nrfx_twim.o ABSOLUTE
    ..\..\..\..\..\..\modules\nrfx\drivers\src\nrfx_uarte.c 0x00000000   Number         0  nrfx_uarte.o ABSOLUTE
    ..\..\..\..\..\..\modules\nrfx\drivers\src\prs\nrfx_prs.c 0x00000000   Number         0  nrfx_prs.o ABSOLUTE
    ..\..\..\main.c                          0x00000000   Number         0  main.o ABSOLUTE
    ..\\..\\..\\..\\..\\..\\components\\ble\\ble_advertising\\ble_advertising.c 0x00000000   Number         0  ble_advertising.o ABSOLUTE
    ..\\..\\..\\..\\..\\..\\components\\ble\\ble_link_ctx_manager\\ble_link_ctx_manager.c 0x00000000   Number         0  ble_link_ctx_manager.o ABSOLUTE
    ..\\..\\..\\..\\..\\..\\components\\ble\\ble_services\\ble_nus\\ble_nus.c 0x00000000   Number         0  ble_nus.o ABSOLUTE
    ..\\..\\..\\..\\..\\..\\components\\ble\\common\\ble_advdata.c 0x00000000   Number         0  ble_advdata.o ABSOLUTE
    ..\\..\\..\\..\\..\\..\\components\\ble\\common\\ble_conn_params.c 0x00000000   Number         0  ble_conn_params.o ABSOLUTE
    ..\\..\\..\\..\\..\\..\\components\\ble\\common\\ble_conn_state.c 0x00000000   Number         0  ble_conn_state.o ABSOLUTE
    ..\\..\\..\\..\\..\\..\\components\\ble\\common\\ble_srv_common.c 0x00000000   Number         0  ble_srv_common.o ABSOLUTE
    ..\\..\\..\\..\\..\\..\\components\\ble\\nrf_ble_gatt\\nrf_ble_gatt.c 0x00000000   Number         0  nrf_ble_gatt.o ABSOLUTE
    ..\\..\\..\\..\\..\\..\\components\\ble\\nrf_ble_qwr\\nrf_ble_qwr.c 0x00000000   Number         0  nrf_ble_qwr.o ABSOLUTE
    ..\\..\\..\\..\\..\\..\\components\\boards\\boards.c 0x00000000   Number         0  boards.o ABSOLUTE
    ..\\..\\..\\..\\..\\..\\components\\libraries\\atomic\\nrf_atomic.c 0x00000000   Number         0  nrf_atomic.o ABSOLUTE
    ..\\..\\..\\..\\..\\..\\components\\libraries\\atomic_fifo\\nrf_atfifo.c 0x00000000   Number         0  nrf_atfifo.o ABSOLUTE
    ..\\..\\..\\..\\..\\..\\components\\libraries\\atomic_flags\\nrf_atflags.c 0x00000000   Number         0  nrf_atflags.o ABSOLUTE
    ..\\..\\..\\..\\..\\..\\components\\libraries\\balloc\\nrf_balloc.c 0x00000000   Number         0  nrf_balloc.o ABSOLUTE
    ..\\..\\..\\..\\..\\..\\components\\libraries\\bsp\\bsp.c 0x00000000   Number         0  bsp.o ABSOLUTE
    ..\\..\\..\\..\\..\\..\\components\\libraries\\bsp\\bsp_btn_ble.c 0x00000000   Number         0  bsp_btn_ble.o ABSOLUTE
    ..\\..\\..\\..\\..\\..\\components\\libraries\\button\\app_button.c 0x00000000   Number         0  app_button.o ABSOLUTE
    ..\\..\\..\\..\\..\\..\\components\\libraries\\experimental_section_vars\\nrf_section_iter.c 0x00000000   Number         0  nrf_section_iter.o ABSOLUTE
    ..\\..\\..\\..\\..\\..\\components\\libraries\\fifo\\app_fifo.c 0x00000000   Number         0  app_fifo.o ABSOLUTE
    ..\\..\\..\\..\\..\\..\\components\\libraries\\hardfault\\hardfault_implementation.c 0x00000000   Number         0  hardfault_implementation.o ABSOLUTE
    ..\\..\\..\\..\\..\\..\\components\\libraries\\log\\src\\nrf_log_backend_rtt.c 0x00000000   Number         0  nrf_log_backend_rtt.o ABSOLUTE
    ..\\..\\..\\..\\..\\..\\components\\libraries\\log\\src\\nrf_log_backend_serial.c 0x00000000   Number         0  nrf_log_backend_serial.o ABSOLUTE
    ..\\..\\..\\..\\..\\..\\components\\libraries\\log\\src\\nrf_log_default_backends.c 0x00000000   Number         0  nrf_log_default_backends.o ABSOLUTE
    ..\\..\\..\\..\\..\\..\\components\\libraries\\log\\src\\nrf_log_frontend.c 0x00000000   Number         0  nrf_log_frontend.o ABSOLUTE
    ..\\..\\..\\..\\..\\..\\components\\libraries\\log\\src\\nrf_log_str_formatter.c 0x00000000   Number         0  nrf_log_str_formatter.o ABSOLUTE
    ..\\..\\..\\..\\..\\..\\components\\libraries\\memobj\\nrf_memobj.c 0x00000000   Number         0  nrf_memobj.o ABSOLUTE
    ..\\..\\..\\..\\..\\..\\components\\libraries\\pwr_mgmt\\nrf_pwr_mgmt.c 0x00000000   Number         0  nrf_pwr_mgmt.o ABSOLUTE
    ..\\..\\..\\..\\..\\..\\components\\libraries\\ringbuf\\nrf_ringbuf.c 0x00000000   Number         0  nrf_ringbuf.o ABSOLUTE
    ..\\..\\..\\..\\..\\..\\components\\libraries\\scheduler\\app_scheduler.c 0x00000000   Number         0  app_scheduler.o ABSOLUTE
    ..\\..\\..\\..\\..\\..\\components\\libraries\\strerror\\nrf_strerror.c 0x00000000   Number         0  nrf_strerror.o ABSOLUTE
    ..\\..\\..\\..\\..\\..\\components\\libraries\\timer\\app_timer.c 0x00000000   Number         0  app_timer.o ABSOLUTE
    ..\\..\\..\\..\\..\\..\\components\\libraries\\uart\\app_uart_fifo.c 0x00000000   Number         0  app_uart_fifo.o ABSOLUTE
    ..\\..\\..\\..\\..\\..\\components\\libraries\\uart\\retarget.c 0x00000000   Number         0  retarget.o ABSOLUTE
    ..\\..\\..\\..\\..\\..\\components\\libraries\\util\\app_error.c 0x00000000   Number         0  app_error.o ABSOLUTE
    ..\\..\\..\\..\\..\\..\\components\\libraries\\util\\app_error_handler_keil.c 0x00000000   Number         0  app_error_handler_keil.o ABSOLUTE
    ..\\..\\..\\..\\..\\..\\components\\libraries\\util\\app_error_weak.c 0x00000000   Number         0  app_error_weak.o ABSOLUTE
    ..\\..\\..\\..\\..\\..\\components\\libraries\\util\\app_util_platform.c 0x00000000   Number         0  app_util_platform.o ABSOLUTE
    ..\\..\\..\\..\\..\\..\\components\\libraries\\util\\nrf_assert.c 0x00000000   Number         0  nrf_assert.o ABSOLUTE
    ..\\..\\..\\..\\..\\..\\components\\softdevice\\common\\nrf_sdh.c 0x00000000   Number         0  nrf_sdh.o ABSOLUTE
    ..\\..\\..\\..\\..\\..\\components\\softdevice\\common\\nrf_sdh_ble.c 0x00000000   Number         0  nrf_sdh_ble.o ABSOLUTE
    ..\\..\\..\\..\\..\\..\\components\\softdevice\\common\\nrf_sdh_soc.c 0x00000000   Number         0  nrf_sdh_soc.o ABSOLUTE
    ..\\..\\..\\..\\..\\..\\external\\fprintf\\nrf_fprintf.c 0x00000000   Number         0  nrf_fprintf.o ABSOLUTE
    ..\\..\\..\\..\\..\\..\\external\\fprintf\\nrf_fprintf_format.c 0x00000000   Number         0  nrf_fprintf_format.o ABSOLUTE
    ..\\..\\..\\..\\..\\..\\external\\segger_rtt\\SEGGER_RTT.c 0x00000000   Number         0  segger_rtt.o ABSOLUTE
    ..\\..\\..\\..\\..\\..\\external\\segger_rtt\\SEGGER_RTT_printf.c 0x00000000   Number         0  segger_rtt_printf.o ABSOLUTE
    ..\\..\\..\\..\\..\\..\\integration\\nrfx\\legacy\\nrf_drv_clock.c 0x00000000   Number         0  nrf_drv_clock.o ABSOLUTE
    ..\\..\\..\\..\\..\\..\\integration\\nrfx\\legacy\\nrf_drv_twi.c 0x00000000   Number         0  nrf_drv_twi.o ABSOLUTE
    ..\\..\\..\\..\\..\\..\\integration\\nrfx\\legacy\\nrf_drv_uart.c 0x00000000   Number         0  nrf_drv_uart.o ABSOLUTE
    ..\\..\\..\\..\\..\\..\\modules\\nrfx\\drivers\\src\\nrfx_clock.c 0x00000000   Number         0  nrfx_clock.o ABSOLUTE
    ..\\..\\..\\..\\..\\..\\modules\\nrfx\\drivers\\src\\nrfx_gpiote.c 0x00000000   Number         0  nrfx_gpiote.o ABSOLUTE
    ..\\..\\..\\..\\..\\..\\modules\\nrfx\\drivers\\src\\nrfx_power_clock.c 0x00000000   Number         0  nrfx_power_clock.o ABSOLUTE
    ..\\..\\..\\..\\..\\..\\modules\\nrfx\\drivers\\src\\nrfx_twi.c 0x00000000   Number         0  nrfx_twi.o ABSOLUTE
    ..\\..\\..\\..\\..\\..\\modules\\nrfx\\drivers\\src\\nrfx_twim.c 0x00000000   Number         0  nrfx_twim.o ABSOLUTE
    ..\\..\\..\\..\\..\\..\\modules\\nrfx\\drivers\\src\\nrfx_uarte.c 0x00000000   Number         0  nrfx_uarte.o ABSOLUTE
    ..\\..\\..\\..\\..\\..\\modules\\nrfx\\drivers\\src\\prs\\nrfx_prs.c 0x00000000   Number         0  nrfx_prs.o ABSOLUTE
    ..\\..\\..\\main.c                       0x00000000   Number         0  main.o ABSOLUTE
    RTE\Device\nRF52810_xxAA\arm_startup_nrf52810.s 0x00000000   Number         0  arm_startup_nrf52810.o ABSOLUTE
    RTE\Device\nRF52810_xxAA\system_nrf52810.c 0x00000000   Number         0  system_nrf52810.o ABSOLUTE
    RTE\\Device\\nRF52810_xxAA\\system_nrf52810.c 0x00000000   Number         0  system_nrf52810.o ABSOLUTE
    dc.s                                     0x00000000   Number         0  dc.o ABSOLUTE
    handlers.s                               0x00000000   Number         0  handlers.o ABSOLUTE
    init.s                                   0x00000000   Number         0  init.o ABSOLUTE
    RESET                                    0x00019000   Section      512  arm_startup_nrf52810.o(RESET)
    .ARM.Collect$$$$00000000                 0x00019200   Section        0  entry.o(.ARM.Collect$$$$00000000)
    .ARM.Collect$$$$00000001                 0x00019200   Section        4  entry2.o(.ARM.Collect$$$$00000001)
    .ARM.Collect$$$$00000004                 0x00019204   Section        4  entry5.o(.ARM.Collect$$$$00000004)
    .ARM.Collect$$$$00000008                 0x00019208   Section        0  entry7b.o(.ARM.Collect$$$$00000008)
    .ARM.Collect$$$$0000000A                 0x00019208   Section        0  entry8b.o(.ARM.Collect$$$$0000000A)
    .ARM.Collect$$$$0000000B                 0x00019208   Section        8  entry9a.o(.ARM.Collect$$$$0000000B)
    .ARM.Collect$$$$0000000D                 0x00019210   Section        0  entry10a.o(.ARM.Collect$$$$0000000D)
    .ARM.Collect$$$$0000000F                 0x00019210   Section        0  entry11a.o(.ARM.Collect$$$$0000000F)
    .ARM.Collect$$$$00002712                 0x00019210   Section        4  entry2.o(.ARM.Collect$$$$00002712)
    __lit__00000000                          0x00019210   Data           4  entry2.o(.ARM.Collect$$$$00002712)
    .emb_text                                0x00019214   Section      226  nrf_atomic.o(.emb_text)
    .text                                    0x000192f8   Section       36  arm_startup_nrf52810.o(.text)
    .text                                    0x0001931c   Section        0  uldiv.o(.text)
    .text                                    0x0001937e   Section        0  llshl.o(.text)
    .text                                    0x0001939c   Section        0  ctype_o.o(.text)
    .text                                    0x000193a4   Section        0  memcpya.o(.text)
    .text                                    0x000193c8   Section        0  memseta.o(.text)
    .text                                    0x000193ec   Section        0  strlen.o(.text)
    .text                                    0x000193fa   Section        0  strcpy.o(.text)
    .text                                    0x0001940c   Section        0  fadd.o(.text)
    .text                                    0x000194bc   Section        0  fscalb.o(.text)
    .text                                    0x000194d4   Section        0  ffltui.o(.text)
    .text                                    0x000194de   Section        0  ffixui.o(.text)
    .text                                    0x00019506   Section        0  llushr.o(.text)
    .text                                    0x00019526   Section        0  iusefp.o(.text)
    .text                                    0x00019526   Section        0  fepilogue.o(.text)
    .text                                    0x00019594   Section       36  init.o(.text)
    i.ENS210_set_mode                        0x000195b8   Section        0  main.o(i.ENS210_set_mode)
    i.GPIOTE_IRQHandler                      0x0001969c   Section        0  nrfx_gpiote.o(i.GPIOTE_IRQHandler)
    i.NVIC_ClearPendingIRQ                   0x00019800   Section        0  app_timer.o(i.NVIC_ClearPendingIRQ)
    NVIC_ClearPendingIRQ                     0x00019801   Thumb Code    22  app_timer.o(i.NVIC_ClearPendingIRQ)
    i.NVIC_EnableIRQ                         0x00019816   Section        0  app_timer.o(i.NVIC_EnableIRQ)
    NVIC_EnableIRQ                           0x00019817   Thumb Code    22  app_timer.o(i.NVIC_EnableIRQ)
    i.NVIC_SetPendingIRQ                     0x0001982c   Section        0  app_timer.o(i.NVIC_SetPendingIRQ)
    NVIC_SetPendingIRQ                       0x0001982d   Thumb Code    22  app_timer.o(i.NVIC_SetPendingIRQ)
    i.NVIC_SetPriority                       0x00019842   Section        0  app_timer.o(i.NVIC_SetPriority)
    NVIC_SetPriority                         0x00019843   Thumb Code    32  app_timer.o(i.NVIC_SetPriority)
    i.POWER_CLOCK_IRQHandler                 0x00019864   Section        0  nrfx_clock.o(i.POWER_CLOCK_IRQHandler)
    i.RTC1_IRQHandler                        0x000198bc   Section        0  app_timer.o(i.RTC1_IRQHandler)
    i.SEGGER_RTT_Init                        0x000198e0   Section        0  segger_rtt.o(i.SEGGER_RTT_Init)
    i.SEGGER_RTT_WriteNoLock                 0x000198e4   Section        0  segger_rtt.o(i.SEGGER_RTT_WriteNoLock)
    i.SWI0_EGU0_IRQHandler                   0x00019940   Section        0  app_timer.o(i.SWI0_EGU0_IRQHandler)
    i.SWI2_IRQHandler                        0x00019944   Section        0  nrf_sdh.o(i.SWI2_IRQHandler)
    i.SystemInit                             0x00019948   Section        0  system_nrf52810.o(i.SystemInit)
    i.TWIM0_TWIS0_IRQHandler                 0x00019c34   Section        0  nrfx_twim.o(i.TWIM0_TWIS0_IRQHandler)
    i.UARTE0_IRQHandler                      0x00019c44   Section        0  nrfx_uarte.o(i.UARTE0_IRQHandler)
    i._DoInit                                0x00019c54   Section        0  segger_rtt.o(i._DoInit)
    _DoInit                                  0x00019c55   Thumb Code    76  segger_rtt.o(i._DoInit)
    i._GetAvailWriteSpace                    0x00019cbc   Section        0  segger_rtt.o(i._GetAvailWriteSpace)
    _GetAvailWriteSpace                      0x00019cbd   Thumb Code    22  segger_rtt.o(i._GetAvailWriteSpace)
    i._WriteBlocking                         0x00019cd2   Section        0  segger_rtt.o(i._WriteBlocking)
    _WriteBlocking                           0x00019cd3   Thumb Code    90  segger_rtt.o(i._WriteBlocking)
    i._WriteNoCheck                          0x00019d2c   Section        0  segger_rtt.o(i._WriteNoCheck)
    _WriteNoCheck                            0x00019d2d   Thumb Code    66  segger_rtt.o(i._WriteNoCheck)
    i.__scatterload_copy                     0x00019d6e   Section       14  handlers.o(i.__scatterload_copy)
    i.__scatterload_null                     0x00019d7c   Section        2  handlers.o(i.__scatterload_null)
    i.__scatterload_zeroinit                 0x00019d7e   Section       14  handlers.o(i.__scatterload_zeroinit)
    i.__sd_nvic_app_accessible_irq           0x00019d8c   Section        0  nrf_sdh.o(i.__sd_nvic_app_accessible_irq)
    __sd_nvic_app_accessible_irq             0x00019d8d   Thumb Code    32  nrf_sdh.o(i.__sd_nvic_app_accessible_irq)
    i.advertising_buttons_configure          0x00019db0   Section        0  bsp_btn_ble.o(i.advertising_buttons_configure)
    advertising_buttons_configure            0x00019db1   Thumb Code    54  bsp_btn_ble.o(i.advertising_buttons_configure)
    i.app_error_fault_handler                0x00019de8   Section        0  app_error_weak.o(i.app_error_fault_handler)
    i.app_error_handler_bare                 0x00019e6c   Section        0  app_error.o(i.app_error_handler_bare)
    i.app_fifo_get                           0x00019e82   Section        0  app_fifo.o(i.app_fifo_get)
    i.app_fifo_init                          0x00019e98   Section        0  app_fifo.o(i.app_fifo_init)
    i.app_fifo_put                           0x00019eb8   Section        0  app_fifo.o(i.app_fifo_put)
    i.app_timer_create                       0x00019ed4   Section        0  app_timer.o(i.app_timer_create)
    i.app_timer_init                         0x00019ef8   Section        0  app_timer.o(i.app_timer_init)
    i.app_timer_start                        0x00019f4c   Section        0  app_timer.o(i.app_timer_start)
    i.app_timer_stop                         0x00019fd4   Section        0  app_timer.o(i.app_timer_stop)
    i.app_uart_get                           0x00019ff4   Section        0  app_uart_fifo.o(i.app_uart_get)
    i.app_uart_init                          0x0001a028   Section        0  app_uart_fifo.o(i.app_uart_init)
    i.app_util_critical_region_enter         0x0001a0cc   Section        0  app_util_platform.o(i.app_util_critical_region_enter)
    i.app_util_critical_region_exit          0x0001a114   Section        0  app_util_platform.o(i.app_util_critical_region_exit)
    i.apply_config                           0x0001a148   Section        0  nrfx_uarte.o(i.apply_config)
    apply_config                             0x0001a149   Thumb Code   136  nrfx_uarte.o(i.apply_config)
    i.blcm_link_ctx_get                      0x0001a1d0   Section        0  ble_link_ctx_manager.o(i.blcm_link_ctx_get)
    i.ble_advdata_encode                     0x0001a218   Section        0  ble_advdata.o(i.ble_advdata_encode)
    i.ble_advdata_parse                      0x0001a39a   Section        0  ble_advdata.o(i.ble_advdata_parse)
    i.ble_advdata_search                     0x0001a3ba   Section        0  ble_advdata.o(i.ble_advdata_search)
    i.ble_advertising_conn_cfg_tag_set       0x0001a3f2   Section        0  ble_advertising.o(i.ble_advertising_conn_cfg_tag_set)
    i.ble_advertising_init                   0x0001a3f8   Section        0  ble_advertising.o(i.ble_advertising_init)
    i.ble_advertising_on_ble_evt             0x0001a4f2   Section        0  ble_advertising.o(i.ble_advertising_on_ble_evt)
    i.ble_advertising_on_sys_evt             0x0001a55c   Section        0  ble_advertising.o(i.ble_advertising_on_sys_evt)
    i.ble_advertising_start                  0x0001a55e   Section        0  ble_advertising.o(i.ble_advertising_start)
    i.ble_conn_params_init                   0x0001a760   Section        0  ble_conn_params.o(i.ble_conn_params_init)
    i.ble_conn_state_conn_idx                0x0001a7c8   Section        0  ble_conn_state.o(i.ble_conn_state_conn_idx)
    i.ble_conn_state_valid                   0x0001a7dc   Section        0  ble_conn_state.o(i.ble_conn_state_valid)
    i.ble_device_addr_encode                 0x0001a7f0   Section        0  ble_advdata.o(i.ble_device_addr_encode)
    ble_device_addr_encode                   0x0001a7f1   Thumb Code    96  ble_advdata.o(i.ble_device_addr_encode)
    i.ble_evt_handler                        0x0001a850   Section        0  main.o(i.ble_evt_handler)
    ble_evt_handler                          0x0001a851   Thumb Code   164  main.o(i.ble_evt_handler)
    i.ble_evt_handler                        0x0001a91c   Section        0  bsp_btn_ble.o(i.ble_evt_handler)
    ble_evt_handler                          0x0001a91d   Thumb Code   106  bsp_btn_ble.o(i.ble_evt_handler)
    i.ble_evt_handler                        0x0001a98c   Section        0  ble_conn_params.o(i.ble_evt_handler)
    ble_evt_handler                          0x0001a98d   Thumb Code   242  ble_conn_params.o(i.ble_evt_handler)
    i.ble_evt_handler                        0x0001aa88   Section        0  ble_conn_state.o(i.ble_evt_handler)
    ble_evt_handler                          0x0001aa89   Thumb Code   254  ble_conn_state.o(i.ble_evt_handler)
    i.ble_nus_data_send                      0x0001ab8c   Section        0  ble_nus.o(i.ble_nus_data_send)
    i.ble_nus_init                           0x0001abf4   Section        0  ble_nus.o(i.ble_nus_init)
    i.ble_nus_on_ble_evt                     0x0001acc8   Section        0  ble_nus.o(i.ble_nus_on_ble_evt)
    i.ble_srv_is_notification_enabled        0x0001ad38   Section        0  ble_srv_common.o(i.ble_srv_is_notification_enabled)
    i.bsp_board_button_idx_to_pin            0x0001ad40   Section        0  boards.o(i.bsp_board_button_idx_to_pin)
    i.bsp_board_led_invert                   0x0001ad4c   Section        0  boards.o(i.bsp_board_led_invert)
    i.bsp_board_led_off                      0x0001ad70   Section        0  boards.o(i.bsp_board_led_off)
    i.bsp_board_led_on                       0x0001ad80   Section        0  boards.o(i.bsp_board_led_on)
    i.bsp_board_led_state_get                0x0001ad90   Section        0  boards.o(i.bsp_board_led_state_get)
    i.bsp_board_leds_off                     0x0001adb0   Section        0  boards.o(i.bsp_board_leds_off)
    i.bsp_board_leds_on                      0x0001adc2   Section        0  boards.o(i.bsp_board_leds_on)
    i.bsp_board_pin_to_button_idx            0x0001add4   Section        0  boards.o(i.bsp_board_pin_to_button_idx)
    i.bsp_btn_ble_sleep_mode_prepare         0x0001adf8   Section        0  bsp_btn_ble.o(i.bsp_btn_ble_sleep_mode_prepare)
    i.bsp_button_event_handler               0x0001ae18   Section        0  bsp.o(i.bsp_button_event_handler)
    bsp_button_event_handler                 0x0001ae19   Thumb Code   132  bsp.o(i.bsp_button_event_handler)
    i.bsp_event_to_button_action_assign      0x0001aea8   Section        0  bsp.o(i.bsp_event_to_button_action_assign)
    i.bsp_indication_set                     0x0001aeec   Section        0  bsp.o(i.bsp_indication_set)
    i.bsp_led_indication                     0x0001af04   Section        0  bsp.o(i.bsp_led_indication)
    bsp_led_indication                       0x0001af05   Thumb Code   446  bsp.o(i.bsp_led_indication)
    i.bsp_wakeup_button_enable               0x0001b0cc   Section        0  bsp.o(i.bsp_wakeup_button_enable)
    i.buf_prealloc                           0x0001b0d4   Section        0  nrf_log_frontend.o(i.buf_prealloc)
    buf_prealloc                             0x0001b0d5   Thumb Code   138  nrf_log_frontend.o(i.buf_prealloc)
    i.buffer_add                             0x0001b164   Section        0  nrf_fprintf_format.o(i.buffer_add)
    buffer_add                               0x0001b165   Thumb Code    30  nrf_fprintf_format.o(i.buffer_add)
    i.buffer_is_empty                        0x0001b184   Section        0  nrf_log_frontend.o(i.buffer_is_empty)
    i.buttons_leds_init                      0x0001b198   Section        0  main.o(i.buttons_leds_init)
    buttons_leds_init                        0x0001b199   Thumb Code   136  main.o(i.buttons_leds_init)
    i.channel_port_get                       0x0001b220   Section        0  nrfx_gpiote.o(i.channel_port_get)
    channel_port_get                         0x0001b221   Thumb Code    10  nrfx_gpiote.o(i.channel_port_get)
    i.characteristic_add                     0x0001b230   Section        0  ble_srv_common.o(i.characteristic_add)
    i.clock_clk_started_notify               0x0001b3c0   Section        0  nrf_drv_clock.o(i.clock_clk_started_notify)
    clock_clk_started_notify                 0x0001b3c1   Thumb Code    34  nrf_drv_clock.o(i.clock_clk_started_notify)
    i.clock_irq_handler                      0x0001b3e8   Section        0  nrf_drv_clock.o(i.clock_irq_handler)
    clock_irq_handler                        0x0001b3e9   Thumb Code    24  nrf_drv_clock.o(i.clock_irq_handler)
    i.compare_reg_update                     0x0001b404   Section        0  app_timer.o(i.compare_reg_update)
    compare_reg_update                       0x0001b405   Thumb Code   160  app_timer.o(i.compare_reg_update)
    i.conn_handle_list_get                   0x0001b4b0   Section        0  ble_conn_state.o(i.conn_handle_list_get)
    i.conn_int_encode                        0x0001b4ee   Section        0  ble_advdata.o(i.conn_int_encode)
    conn_int_encode                          0x0001b4ef   Thumb Code   136  ble_advdata.o(i.conn_int_encode)
    i.conn_params_error_handler              0x0001b576   Section        0  main.o(i.conn_params_error_handler)
    conn_params_error_handler                0x0001b577   Thumb Code     4  main.o(i.conn_params_error_handler)
    i.conn_params_negotiation                0x0001b57c   Section        0  ble_conn_params.o(i.conn_params_negotiation)
    conn_params_negotiation                  0x0001b57d   Thumb Code    68  ble_conn_params.o(i.conn_params_negotiation)
    i.dropped_sat16_get                      0x0001b5c4   Section        0  nrf_log_frontend.o(i.dropped_sat16_get)
    dropped_sat16_get                        0x0001b5c5   Thumb Code    16  nrf_log_frontend.o(i.dropped_sat16_get)
    i.elapsed_ticks_acquire                  0x0001b5d8   Section        0  app_timer.o(i.elapsed_ticks_acquire)
    elapsed_ticks_acquire                    0x0001b5d9   Thumb Code    58  app_timer.o(i.elapsed_ticks_acquire)
    i.fifo_get                               0x0001b618   Section        0  app_fifo.o(i.fifo_get)
    fifo_get                                 0x0001b619   Thumb Code    20  app_fifo.o(i.fifo_get)
    i.fifo_put                               0x0001b62c   Section        0  app_fifo.o(i.fifo_put)
    fifo_put                                 0x0001b62d   Thumb Code    18  app_fifo.o(i.fifo_put)
    i.flags_set                              0x0001b63e   Section        0  ble_advertising.o(i.flags_set)
    flags_set                                0x0001b63f   Thumb Code    40  ble_advertising.o(i.flags_set)
    i.free                                   0x0001b668   Section        0  malloc.o(i.free)
    i.gatt_evt_handler                       0x0001b6b8   Section        0  main.o(i.gatt_evt_handler)
    i.gatt_init                              0x0001b714   Section        0  main.o(i.gatt_init)
    i.heart_rate_meas_timeout_handler        0x0001b744   Section        0  main.o(i.heart_rate_meas_timeout_handler)
    heart_rate_meas_timeout_handler          0x0001b745   Thumb Code   118  main.o(i.heart_rate_meas_timeout_handler)
    i.instance_get                           0x0001b7c0   Section        0  ble_conn_params.o(i.instance_get)
    instance_get                             0x0001b7c1   Thumb Code    14  ble_conn_params.o(i.instance_get)
    i.int_print                              0x0001b7d4   Section        0  nrf_fprintf_format.o(i.int_print)
    int_print                                0x0001b7d5   Thumb Code   166  nrf_fprintf_format.o(i.int_print)
    i.interrupts_enable                      0x0001b87c   Section        0  nrfx_uarte.o(i.interrupts_enable)
    interrupts_enable                        0x0001b87d   Thumb Code   122  nrfx_uarte.o(i.interrupts_enable)
    i.invalid_packets_omit                   0x0001b8fc   Section        0  nrf_log_frontend.o(i.invalid_packets_omit)
    invalid_packets_omit                     0x0001b8fd   Thumb Code    52  nrf_log_frontend.o(i.invalid_packets_omit)
    i.is_conn_params_ok                      0x0001b930   Section        0  ble_conn_params.o(i.is_conn_params_ok)
    is_conn_params_ok                        0x0001b931   Thumb Code    68  ble_conn_params.o(i.is_conn_params_ok)
    i.leds_off                               0x0001b974   Section        0  bsp.o(i.leds_off)
    leds_off                                 0x0001b975   Thumb Code    42  bsp.o(i.leds_off)
    i.link_init                              0x0001b9a4   Section        0  nrf_ble_gatt.o(i.link_init)
    link_init                                0x0001b9a5   Thumb Code    16  nrf_ble_gatt.o(i.link_init)
    i.list_insertions_handler                0x0001b9b4   Section        0  app_timer.o(i.list_insertions_handler)
    list_insertions_handler                  0x0001b9b5   Thumb Code   234  app_timer.o(i.list_insertions_handler)
    i.log_skip                               0x0001baac   Section        0  nrf_log_frontend.o(i.log_skip)
    log_skip                                 0x0001baad   Thumb Code   148  nrf_log_frontend.o(i.log_skip)
    i.main                                   0x0001bb48   Section        0  main.o(i.main)
    i.malloc                                 0x0001bd9c   Section        0  malloc.o(i.malloc)
    i.manuf_specific_data_encode             0x0001be08   Section        0  ble_advdata.o(i.manuf_specific_data_encode)
    manuf_specific_data_encode               0x0001be09   Thumb Code   100  ble_advdata.o(i.manuf_specific_data_encode)
    i.memobj_op                              0x0001be6c   Section        0  nrf_memobj.o(i.memobj_op)
    memobj_op                                0x0001be6d   Thumb Code   126  nrf_memobj.o(i.memobj_op)
    i.module_idx_get                         0x0001beec   Section        0  nrf_log_frontend.o(i.module_idx_get)
    module_idx_get                           0x0001beed   Thumb Code    42  nrf_log_frontend.o(i.module_idx_get)
    i.name_encode                            0x0001bf1c   Section        0  ble_advdata.o(i.name_encode)
    name_encode                              0x0001bf1d   Thumb Code   166  ble_advdata.o(i.name_encode)
    i.nrf_atflags_clear                      0x0001bfc2   Section        0  nrf_atflags.o(i.nrf_atflags_clear)
    i.nrf_atflags_get                        0x0001bfd8   Section        0  nrf_atflags.o(i.nrf_atflags_get)
    i.nrf_atflags_set                        0x0001bfee   Section        0  nrf_atflags.o(i.nrf_atflags_set)
    i.nrf_atomic_flag_clear_fetch            0x0001c002   Section        0  nrf_atomic.o(i.nrf_atomic_flag_clear_fetch)
    i.nrf_atomic_flag_set                    0x0001c008   Section        0  nrf_atomic.o(i.nrf_atomic_flag_set)
    i.nrf_atomic_u32_add                     0x0001c00e   Section        0  nrf_atomic.o(i.nrf_atomic_u32_add)
    i.nrf_atomic_u32_and                     0x0001c01a   Section        0  nrf_atomic.o(i.nrf_atomic_u32_and)
    i.nrf_atomic_u32_fetch_and               0x0001c026   Section        0  nrf_atomic.o(i.nrf_atomic_u32_fetch_and)
    i.nrf_atomic_u32_fetch_store             0x0001c030   Section        0  nrf_atomic.o(i.nrf_atomic_u32_fetch_store)
    i.nrf_atomic_u32_or                      0x0001c03a   Section        0  nrf_atomic.o(i.nrf_atomic_u32_or)
    i.nrf_atomic_u32_sub                     0x0001c046   Section        0  nrf_atomic.o(i.nrf_atomic_u32_sub)
    i.nrf_balloc_alloc                       0x0001c052   Section        0  nrf_balloc.o(i.nrf_balloc_alloc)
    i.nrf_balloc_free                        0x0001c096   Section        0  nrf_balloc.o(i.nrf_balloc_free)
    i.nrf_balloc_init                        0x0001c0c6   Section        0  nrf_balloc.o(i.nrf_balloc_init)
    i.nrf_bitmask_bit_is_set                 0x0001c0f6   Section        0  nrfx_gpiote.o(i.nrf_bitmask_bit_is_set)
    nrf_bitmask_bit_is_set                   0x0001c0f7   Thumb Code    16  nrfx_gpiote.o(i.nrf_bitmask_bit_is_set)
    i.nrf_bitmask_bit_set                    0x0001c106   Section        0  nrfx_gpiote.o(i.nrf_bitmask_bit_set)
    nrf_bitmask_bit_set                      0x0001c107   Thumb Code    20  nrfx_gpiote.o(i.nrf_bitmask_bit_set)
    i.nrf_ble_gatt_att_mtu_periph_set        0x0001c11a   Section        0  nrf_ble_gatt.o(i.nrf_ble_gatt_att_mtu_periph_set)
    i.nrf_ble_gatt_init                      0x0001c132   Section        0  nrf_ble_gatt.o(i.nrf_ble_gatt_init)
    i.nrf_ble_gatt_on_ble_evt                0x0001c154   Section        0  nrf_ble_gatt.o(i.nrf_ble_gatt_on_ble_evt)
    i.nrf_ble_qwr_init                       0x0001c248   Section        0  nrf_ble_qwr.o(i.nrf_ble_qwr_init)
    i.nrf_ble_qwr_on_ble_evt                 0x0001c26c   Section        0  nrf_ble_qwr.o(i.nrf_ble_qwr_on_ble_evt)
    i.nrf_clock_event_check                  0x0001c322   Section        0  nrfx_clock.o(i.nrf_clock_event_check)
    nrf_clock_event_check                    0x0001c323   Thumb Code    14  nrfx_clock.o(i.nrf_clock_event_check)
    i.nrf_clock_event_clear                  0x0001c330   Section        0  nrfx_clock.o(i.nrf_clock_event_clear)
    nrf_clock_event_clear                    0x0001c331   Thumb Code    16  nrfx_clock.o(i.nrf_clock_event_clear)
    i.nrf_delay_ms                           0x0001c340   Section        0  main.o(i.nrf_delay_ms)
    nrf_delay_ms                             0x0001c341   Thumb Code    28  main.o(i.nrf_delay_ms)
    i.nrf_drv_clock_init                     0x0001c360   Section        0  nrf_drv_clock.o(i.nrf_drv_clock_init)
    i.nrf_drv_clock_lfclk_release            0x0001c398   Section        0  nrf_drv_clock.o(i.nrf_drv_clock_lfclk_release)
    i.nrf_drv_twi_init                       0x0001c3c8   Section        0  nrf_drv_twi.o(i.nrf_drv_twi_init)
    i.nrf_drv_twi_rx                         0x0001c408   Section        0  main.o(i.nrf_drv_twi_rx)
    nrf_drv_twi_rx                           0x0001c409   Thumb Code     6  main.o(i.nrf_drv_twi_rx)
    i.nrf_drv_twi_tx                         0x0001c40e   Section        0  main.o(i.nrf_drv_twi_tx)
    nrf_drv_twi_tx                           0x0001c40f   Thumb Code    14  main.o(i.nrf_drv_twi_tx)
    i.nrf_drv_uart_init                      0x0001c41c   Section        0  nrf_drv_uart.o(i.nrf_drv_uart_init)
    i.nrf_drv_uart_rx                        0x0001c45c   Section        0  app_uart_fifo.o(i.nrf_drv_uart_rx)
    nrf_drv_uart_rx                          0x0001c45d   Thumb Code     6  app_uart_fifo.o(i.nrf_drv_uart_rx)
    i.nrf_drv_uart_tx                        0x0001c462   Section        0  app_uart_fifo.o(i.nrf_drv_uart_tx)
    nrf_drv_uart_tx                          0x0001c463   Thumb Code     6  app_uart_fifo.o(i.nrf_drv_uart_tx)
    i.nrf_fprintf                            0x0001c468   Section        0  nrf_fprintf.o(i.nrf_fprintf)
    i.nrf_fprintf_buffer_flush               0x0001c482   Section        0  nrf_fprintf.o(i.nrf_fprintf_buffer_flush)
    i.nrf_fprintf_fmt                        0x0001c49a   Section        0  nrf_fprintf_format.o(i.nrf_fprintf_fmt)
    i.nrf_gpio_cfg                           0x0001c674   Section        0  nrfx_uarte.o(i.nrf_gpio_cfg)
    nrf_gpio_cfg                             0x0001c675   Thumb Code    36  nrfx_uarte.o(i.nrf_gpio_cfg)
    i.nrf_gpio_cfg                           0x0001c698   Section        0  nrfx_twim.o(i.nrf_gpio_cfg)
    nrf_gpio_cfg                             0x0001c699   Thumb Code    36  nrfx_twim.o(i.nrf_gpio_cfg)
    i.nrf_gpio_cfg_input                     0x0001c6bc   Section        0  nrfx_uarte.o(i.nrf_gpio_cfg_input)
    nrf_gpio_cfg_input                       0x0001c6bd   Thumb Code    18  nrfx_uarte.o(i.nrf_gpio_cfg_input)
    i.nrf_gpio_cfg_output                    0x0001c6ce   Section        0  main.o(i.nrf_gpio_cfg_output)
    nrf_gpio_cfg_output                      0x0001c6cf   Thumb Code    16  main.o(i.nrf_gpio_cfg_output)
    i.nrf_gpio_cfg_output                    0x0001c6de   Section        0  nrfx_uarte.o(i.nrf_gpio_cfg_output)
    nrf_gpio_cfg_output                      0x0001c6df   Thumb Code    20  nrfx_uarte.o(i.nrf_gpio_cfg_output)
    i.nrf_gpio_cfg_sense_set                 0x0001c6f2   Section        0  nrfx_gpiote.o(i.nrf_gpio_cfg_sense_set)
    nrf_gpio_cfg_sense_set                   0x0001c6f3   Thumb Code    34  nrfx_gpiote.o(i.nrf_gpio_cfg_sense_set)
    i.nrf_gpio_pin_clear                     0x0001c714   Section        0  main.o(i.nrf_gpio_pin_clear)
    nrf_gpio_pin_clear                       0x0001c715   Thumb Code    14  main.o(i.nrf_gpio_pin_clear)
    i.nrf_gpio_pin_set                       0x0001c722   Section        0  main.o(i.nrf_gpio_pin_set)
    nrf_gpio_pin_set                         0x0001c723   Thumb Code    14  main.o(i.nrf_gpio_pin_set)
    i.nrf_gpio_pin_set                       0x0001c730   Section        0  nrf_drv_twi.o(i.nrf_gpio_pin_set)
    nrf_gpio_pin_set                         0x0001c731   Thumb Code    14  nrf_drv_twi.o(i.nrf_gpio_pin_set)
    i.nrf_gpio_pin_write                     0x0001c73e   Section        0  boards.o(i.nrf_gpio_pin_write)
    nrf_gpio_pin_write                       0x0001c73f   Thumb Code    22  boards.o(i.nrf_gpio_pin_write)
    i.nrf_gpio_ports_read                    0x0001c754   Section        0  nrfx_gpiote.o(i.nrf_gpio_ports_read)
    nrf_gpio_ports_read                      0x0001c755   Thumb Code    34  nrfx_gpiote.o(i.nrf_gpio_ports_read)
    i.nrf_gpiote_event_clear                 0x0001c77c   Section        0  nrfx_gpiote.o(i.nrf_gpiote_event_clear)
    nrf_gpiote_event_clear                   0x0001c77d   Thumb Code    16  nrfx_gpiote.o(i.nrf_gpiote_event_clear)
    i.nrf_gpiote_event_is_set                0x0001c790   Section        0  nrfx_gpiote.o(i.nrf_gpiote_event_is_set)
    nrf_gpiote_event_is_set                  0x0001c791   Thumb Code    12  nrfx_gpiote.o(i.nrf_gpiote_event_is_set)
    i.nrf_log_backend_add                    0x0001c7a0   Section        0  nrf_log_frontend.o(i.nrf_log_backend_add)
    i.nrf_log_backend_rtt_flush              0x0001c7fc   Section        0  nrf_log_backend_rtt.o(i.nrf_log_backend_rtt_flush)
    nrf_log_backend_rtt_flush                0x0001c7fd   Thumb Code     2  nrf_log_backend_rtt.o(i.nrf_log_backend_rtt_flush)
    i.nrf_log_backend_rtt_init               0x0001c7fe   Section        0  nrf_log_backend_rtt.o(i.nrf_log_backend_rtt_init)
    i.nrf_log_backend_rtt_panic_set          0x0001c802   Section        0  nrf_log_backend_rtt.o(i.nrf_log_backend_rtt_panic_set)
    nrf_log_backend_rtt_panic_set            0x0001c803   Thumb Code     2  nrf_log_backend_rtt.o(i.nrf_log_backend_rtt_panic_set)
    i.nrf_log_backend_rtt_put                0x0001c804   Section        0  nrf_log_backend_rtt.o(i.nrf_log_backend_rtt_put)
    nrf_log_backend_rtt_put                  0x0001c805   Thumb Code    16  nrf_log_backend_rtt.o(i.nrf_log_backend_rtt_put)
    i.nrf_log_backend_serial_put             0x0001c81c   Section        0  nrf_log_backend_serial.o(i.nrf_log_backend_serial_put)
    i.nrf_log_color_id_get                   0x0001c8e4   Section        0  nrf_log_frontend.o(i.nrf_log_color_id_get)
    i.nrf_log_default_backends_init          0x0001c914   Section        0  nrf_log_default_backends.o(i.nrf_log_default_backends_init)
    i.nrf_log_frontend_dequeue               0x0001c930   Section        0  nrf_log_frontend.o(i.nrf_log_frontend_dequeue)
    i.nrf_log_frontend_std_0                 0x0001cb64   Section        0  nrf_log_frontend.o(i.nrf_log_frontend_std_0)
    i.nrf_log_frontend_std_1                 0x0001cb6c   Section        0  nrf_log_frontend.o(i.nrf_log_frontend_std_1)
    i.nrf_log_frontend_std_2                 0x0001cb7a   Section        0  nrf_log_frontend.o(i.nrf_log_frontend_std_2)
    i.nrf_log_hexdump_entry_process          0x0001cb8c   Section        0  nrf_log_str_formatter.o(i.nrf_log_hexdump_entry_process)
    i.nrf_log_init                           0x0001cc38   Section        0  nrf_log_frontend.o(i.nrf_log_init)
    i.nrf_log_module_cnt_get                 0x0001cc74   Section        0  nrf_log_frontend.o(i.nrf_log_module_cnt_get)
    i.nrf_log_module_name_get                0x0001cc88   Section        0  nrf_log_frontend.o(i.nrf_log_module_name_get)
    i.nrf_log_panic                          0x0001cca4   Section        0  nrf_log_frontend.o(i.nrf_log_panic)
    i.nrf_log_std_entry_process              0x0001ccd0   Section        0  nrf_log_str_formatter.o(i.nrf_log_std_entry_process)
    i.nrf_memobj_alloc                       0x0001cd86   Section        0  nrf_memobj.o(i.nrf_memobj_alloc)
    i.nrf_memobj_free                        0x0001cde6   Section        0  nrf_memobj.o(i.nrf_memobj_free)
    i.nrf_memobj_get                         0x0001ce18   Section        0  nrf_memobj.o(i.nrf_memobj_get)
    i.nrf_memobj_pool_init                   0x0001ce20   Section        0  nrf_memobj.o(i.nrf_memobj_pool_init)
    i.nrf_memobj_put                         0x0001ce24   Section        0  nrf_memobj.o(i.nrf_memobj_put)
    i.nrf_memobj_read                        0x0001ce42   Section        0  nrf_memobj.o(i.nrf_memobj_read)
    i.nrf_memobj_write                       0x0001ce52   Section        0  nrf_memobj.o(i.nrf_memobj_write)
    i.nrf_pwr_mgmt_init                      0x0001ce64   Section        0  nrf_pwr_mgmt.o(i.nrf_pwr_mgmt_init)
    i.nrf_pwr_mgmt_run                       0x0001ce8c   Section        0  nrf_pwr_mgmt.o(i.nrf_pwr_mgmt_run)
    i.nrf_qwr_error_handler                  0x0001cea0   Section        0  main.o(i.nrf_qwr_error_handler)
    nrf_qwr_error_handler                    0x0001cea1   Thumb Code     4  main.o(i.nrf_qwr_error_handler)
    i.nrf_ringbuf_init                       0x0001cea4   Section        0  nrf_ringbuf.o(i.nrf_ringbuf_init)
    i.nrf_sdh_ble_app_ram_start_get          0x0001cec0   Section        0  nrf_sdh_ble.o(i.nrf_sdh_ble_app_ram_start_get)
    i.nrf_sdh_ble_default_cfg_set            0x0001ced4   Section        0  nrf_sdh_ble.o(i.nrf_sdh_ble_default_cfg_set)
    i.nrf_sdh_ble_enable                     0x0001cffc   Section        0  nrf_sdh_ble.o(i.nrf_sdh_ble_enable)
    i.nrf_sdh_ble_evts_poll                  0x0001d12c   Section        0  nrf_sdh_ble.o(i.nrf_sdh_ble_evts_poll)
    nrf_sdh_ble_evts_poll                    0x0001d12d   Thumb Code    88  nrf_sdh_ble.o(i.nrf_sdh_ble_evts_poll)
    i.nrf_sdh_enable_request                 0x0001d18c   Section        0  nrf_sdh.o(i.nrf_sdh_enable_request)
    i.nrf_sdh_evts_poll                      0x0001d200   Section        0  nrf_sdh.o(i.nrf_sdh_evts_poll)
    i.nrf_sdh_is_enabled                     0x0001d224   Section        0  nrf_sdh.o(i.nrf_sdh_is_enabled)
    i.nrf_sdh_soc_evts_poll                  0x0001d230   Section        0  nrf_sdh_soc.o(i.nrf_sdh_soc_evts_poll)
    nrf_sdh_soc_evts_poll                    0x0001d231   Thumb Code    56  nrf_sdh_soc.o(i.nrf_sdh_soc_evts_poll)
    i.nrf_section_iter_init                  0x0001d26c   Section        0  nrf_section_iter.o(i.nrf_section_iter_init)
    i.nrf_section_iter_item_set              0x0001d276   Section        0  nrf_section_iter.o(i.nrf_section_iter_item_set)
    nrf_section_iter_item_set                0x0001d277   Thumb Code    36  nrf_section_iter.o(i.nrf_section_iter_item_set)
    i.nrf_section_iter_next                  0x0001d29a   Section        0  nrf_section_iter.o(i.nrf_section_iter_next)
    i.nrf_strerror_find                      0x0001d2bc   Section        0  nrf_strerror.o(i.nrf_strerror_find)
    i.nrf_strerror_get                       0x0001d2f4   Section        0  nrf_strerror.o(i.nrf_strerror_get)
    i.nrf_twim_event_check                   0x0001d308   Section        0  nrfx_twim.o(i.nrf_twim_event_check)
    nrf_twim_event_check                     0x0001d309   Thumb Code    10  nrfx_twim.o(i.nrf_twim_event_check)
    i.nrf_twim_event_clear                   0x0001d312   Section        0  nrfx_twim.o(i.nrf_twim_event_clear)
    nrf_twim_event_clear                     0x0001d313   Thumb Code    12  nrfx_twim.o(i.nrf_twim_event_clear)
    i.nrf_uarte_event_check                  0x0001d31e   Section        0  nrfx_uarte.o(i.nrf_uarte_event_check)
    nrf_uarte_event_check                    0x0001d31f   Thumb Code    10  nrfx_uarte.o(i.nrf_uarte_event_check)
    i.nrf_uarte_event_clear                  0x0001d328   Section        0  nrfx_uarte.o(i.nrf_uarte_event_clear)
    nrf_uarte_event_clear                    0x0001d329   Thumb Code    12  nrfx_uarte.o(i.nrf_uarte_event_clear)
    i.nrfx_clock_enable                      0x0001d334   Section        0  nrfx_clock.o(i.nrfx_clock_enable)
    i.nrfx_clock_init                        0x0001d364   Section        0  nrfx_clock.o(i.nrfx_clock_init)
    i.nrfx_clock_lfclk_stop                  0x0001d384   Section        0  nrfx_clock.o(i.nrfx_clock_lfclk_stop)
    i.nrfx_coredep_delay_us                  0x0001d3a0   Section        0  nrf_drv_twi.o(i.nrfx_coredep_delay_us)
    nrfx_coredep_delay_us                    0x0001d3a1   Thumb Code    12  nrf_drv_twi.o(i.nrfx_coredep_delay_us)
    i.nrfx_coredep_delay_us                  0x0001d3b0   Section        0  app_timer.o(i.nrfx_coredep_delay_us)
    nrfx_coredep_delay_us                    0x0001d3b1   Thumb Code    12  app_timer.o(i.nrfx_coredep_delay_us)
    i.nrfx_is_in_ram                         0x0001d3c0   Section        0  nrfx_uarte.o(i.nrfx_is_in_ram)
    nrfx_is_in_ram                           0x0001d3c1   Thumb Code    16  nrfx_uarte.o(i.nrfx_is_in_ram)
    i.nrfx_is_in_ram                         0x0001d3d0   Section        0  nrfx_twim.o(i.nrfx_is_in_ram)
    nrfx_is_in_ram                           0x0001d3d1   Thumb Code    16  nrfx_twim.o(i.nrfx_is_in_ram)
    i.nrfx_prs_acquire                       0x0001d3e0   Section        0  nrfx_prs.o(i.nrfx_prs_acquire)
    i.nrfx_twim_enable                       0x0001d3e4   Section        0  nrfx_twim.o(i.nrfx_twim_enable)
    i.nrfx_twim_init                         0x0001d408   Section        0  nrfx_twim.o(i.nrfx_twim_init)
    i.nrfx_twim_rx                           0x0001d4ec   Section        0  nrfx_twim.o(i.nrfx_twim_rx)
    i.nrfx_twim_tx                           0x0001d51c   Section        0  nrfx_twim.o(i.nrfx_twim_tx)
    i.nrfx_twim_xfer                         0x0001d554   Section        0  nrfx_twim.o(i.nrfx_twim_xfer)
    i.nrfx_uarte_init                        0x0001d57c   Section        0  nrfx_uarte.o(i.nrfx_uarte_init)
    i.nrfx_uarte_rx                          0x0001d5e8   Section        0  nrfx_uarte.o(i.nrfx_uarte_rx)
    i.nrfx_uarte_tx                          0x0001d6ec   Section        0  nrfx_uarte.o(i.nrfx_uarte_tx)
    i.nrfx_uarte_tx_in_progress              0x0001d77c   Section        0  nrfx_uarte.o(i.nrfx_uarte_tx_in_progress)
    i.nus_data_handler                       0x0001d798   Section        0  main.o(i.nus_data_handler)
    nus_data_handler                         0x0001d799   Thumb Code    28  main.o(i.nus_data_handler)
    i.on_adv_evt                             0x0001d7cc   Section        0  main.o(i.on_adv_evt)
    on_adv_evt                               0x0001d7cd   Thumb Code    36  main.o(i.on_adv_evt)
    i.on_conn_params_evt                     0x0001d7f0   Section        0  main.o(i.on_conn_params_evt)
    on_conn_params_evt                       0x0001d7f1   Thumb Code    24  main.o(i.on_conn_params_evt)
    i.on_connect                             0x0001d80c   Section        0  ble_nus.o(i.on_connect)
    on_connect                               0x0001d80d   Thumb Code   106  ble_nus.o(i.on_connect)
    i.on_connected_evt                       0x0001d878   Section        0  nrf_ble_gatt.o(i.on_connected_evt)
    on_connected_evt                         0x0001d879   Thumb Code    80  nrf_ble_gatt.o(i.on_connected_evt)
    i.on_exchange_mtu_request_evt            0x0001d904   Section        0  nrf_ble_gatt.o(i.on_exchange_mtu_request_evt)
    on_exchange_mtu_request_evt              0x0001d905   Thumb Code   114  nrf_ble_gatt.o(i.on_exchange_mtu_request_evt)
    i.on_write                               0x0001d9b4   Section        0  ble_nus.o(i.on_write)
    on_write                                 0x0001d9b5   Thumb Code   132  ble_nus.o(i.on_write)
    i.phy_is_valid                           0x0001da38   Section        0  ble_advertising.o(i.phy_is_valid)
    phy_is_valid                             0x0001da39   Thumb Code    18  ble_advertising.o(i.phy_is_valid)
    i.postfix_process                        0x0001da4c   Section        0  nrf_log_str_formatter.o(i.postfix_process)
    postfix_process                          0x0001da4d   Thumb Code    48  nrf_log_str_formatter.o(i.postfix_process)
    i.prefix_process                         0x0001da88   Section        0  nrf_log_str_formatter.o(i.prefix_process)
    prefix_process                           0x0001da89   Thumb Code    90  nrf_log_str_formatter.o(i.prefix_process)
    i.read_ENS210_sensor_data                0x0001db20   Section        0  main.o(i.read_ENS210_sensor_data)
    read_ENS210_sensor_data                  0x0001db21   Thumb Code    74  main.o(i.read_ENS210_sensor_data)
    i.rtc1_stop                              0x0001db74   Section        0  app_timer.o(i.rtc1_stop)
    rtc1_stop                                0x0001db75   Thumb Code    52  app_timer.o(i.rtc1_stop)
    i.rx_done_event                          0x0001dbb0   Section        0  nrfx_uarte.o(i.rx_done_event)
    rx_done_event                            0x0001dbb1   Thumb Code    24  nrfx_uarte.o(i.rx_done_event)
    i.sd_state_evt_handler                   0x0001dbc8   Section        0  nrf_drv_clock.o(i.sd_state_evt_handler)
    sd_state_evt_handler                     0x0001dbc9   Thumb Code    76  nrf_drv_clock.o(i.sd_state_evt_handler)
    i.sdh_request_observer_notify            0x0001dc18   Section        0  nrf_sdh.o(i.sdh_request_observer_notify)
    sdh_request_observer_notify              0x0001dc19   Thumb Code    44  nrf_sdh.o(i.sdh_request_observer_notify)
    i.sdh_state_observer_notify              0x0001dc48   Section        0  nrf_sdh.o(i.sdh_state_observer_notify)
    sdh_state_observer_notify                0x0001dc49   Thumb Code    38  nrf_sdh.o(i.sdh_state_observer_notify)
    i.send_error_evt                         0x0001dc74   Section        0  ble_conn_params.o(i.send_error_evt)
    send_error_evt                           0x0001dc75   Thumb Code    12  ble_conn_params.o(i.send_error_evt)
    i.serial_tx                              0x0001dc84   Section        0  nrf_log_backend_rtt.o(i.serial_tx)
    serial_tx                                0x0001dc85   Thumb Code    70  nrf_log_backend_rtt.o(i.serial_tx)
    i.service_data_encode                    0x0001dcd4   Section        0  ble_advdata.o(i.service_data_encode)
    service_data_encode                      0x0001dcd5   Thumb Code   136  ble_advdata.o(i.service_data_encode)
    i.set_security_req                       0x0001dd5c   Section        0  ble_srv_common.o(i.set_security_req)
    set_security_req                         0x0001dd5d   Thumb Code    48  ble_srv_common.o(i.set_security_req)
    i.sleep_mode_enter                       0x0001dd8c   Section        0  main.o(i.sleep_mode_enter)
    sleep_mode_enter                         0x0001dd8d   Thumb Code    40  main.o(i.sleep_mode_enter)
    i.soc_evt_handler                        0x0001ddb4   Section        0  nrf_drv_clock.o(i.soc_evt_handler)
    soc_evt_handler                          0x0001ddb5   Thumb Code    18  nrf_drv_clock.o(i.soc_evt_handler)
    i.softdevices_evt_irq_enable             0x0001ddcc   Section        0  nrf_sdh.o(i.softdevices_evt_irq_enable)
    softdevices_evt_irq_enable               0x0001ddcd   Thumb Code    80  nrf_sdh.o(i.softdevices_evt_irq_enable)
    i.std_n                                  0x0001de24   Section        0  nrf_log_frontend.o(i.std_n)
    std_n                                    0x0001de25   Thumb Code   136  nrf_log_frontend.o(i.std_n)
    i.timer_list_handler                     0x0001deb0   Section        0  app_timer.o(i.timer_list_handler)
    timer_list_handler                       0x0001deb1   Thumb Code   122  app_timer.o(i.timer_list_handler)
    i.timer_list_insert                      0x0001df30   Section        0  app_timer.o(i.timer_list_insert)
    timer_list_insert                        0x0001df31   Thumb Code    56  app_timer.o(i.timer_list_insert)
    i.timer_list_remove                      0x0001df6c   Section        0  app_timer.o(i.timer_list_remove)
    timer_list_remove                        0x0001df6d   Thumb Code    88  app_timer.o(i.timer_list_remove)
    i.timer_stop_op_schedule                 0x0001dfcc   Section        0  app_timer.o(i.timer_stop_op_schedule)
    timer_stop_op_schedule                   0x0001dfcd   Thumb Code    68  app_timer.o(i.timer_stop_op_schedule)
    i.timer_timeouts_check                   0x0001e014   Section        0  app_timer.o(i.timer_timeouts_check)
    timer_timeouts_check                     0x0001e015   Thumb Code   106  app_timer.o(i.timer_timeouts_check)
    i.twi_clear_bus                          0x0001e088   Section        0  nrf_drv_twi.o(i.twi_clear_bus)
    twi_clear_bus                            0x0001e089   Thumb Code   170  nrf_drv_twi.o(i.twi_clear_bus)
    i.twi_handler                            0x0001e134   Section        0  main.o(i.twi_handler)
    i.twi_init                               0x0001e25c   Section        0  main.o(i.twi_init)
    i.twim_evt_handler                       0x0001e28c   Section        0  nrf_drv_twi.o(i.twim_evt_handler)
    twim_evt_handler                         0x0001e28d   Thumb Code    60  nrf_drv_twi.o(i.twim_evt_handler)
    i.twim_irq_handler                       0x0001e2cc   Section        0  nrfx_twim.o(i.twim_irq_handler)
    twim_irq_handler                         0x0001e2cd   Thumb Code   328  nrfx_twim.o(i.twim_irq_handler)
    i.twim_xfer                              0x0001e418   Section        0  nrfx_twim.o(i.twim_xfer)
    twim_xfer                                0x0001e419   Thumb Code   558  nrfx_twim.o(i.twim_xfer)
    i.uart_event_handle                      0x0001e650   Section        0  main.o(i.uart_event_handle)
    i.uart_event_handler                     0x0001e6b8   Section        0  app_uart_fifo.o(i.uart_event_handler)
    uart_event_handler                       0x0001e6b9   Thumb Code   152  app_uart_fifo.o(i.uart_event_handler)
    i.uarte_evt_handler                      0x0001e758   Section        0  nrf_drv_uart.o(i.uarte_evt_handler)
    uarte_evt_handler                        0x0001e759   Thumb Code    42  nrf_drv_uart.o(i.uarte_evt_handler)
    i.uarte_irq_handler                      0x0001e788   Section        0  nrfx_uarte.o(i.uarte_irq_handler)
    uarte_irq_handler                        0x0001e789   Thumb Code   244  nrfx_uarte.o(i.uarte_irq_handler)
    i.uint16_encode                          0x0001e87c   Section        0  ble_advdata.o(i.uint16_encode)
    uint16_encode                            0x0001e87d   Thumb Code    10  ble_advdata.o(i.uint16_encode)
    i.unsigned_print                         0x0001e888   Section        0  nrf_fprintf_format.o(i.unsigned_print)
    unsigned_print                           0x0001e889   Thumb Code   176  nrf_fprintf_format.o(i.unsigned_print)
    i.update_timeout_handler                 0x0001e93c   Section        0  ble_conn_params.o(i.update_timeout_handler)
    update_timeout_handler                   0x0001e93d   Thumb Code    98  ble_conn_params.o(i.update_timeout_handler)
    i.use_whitelist                          0x0001e9a4   Section        0  ble_advertising.o(i.use_whitelist)
    use_whitelist                            0x0001e9a5   Thumb Code    24  ble_advertising.o(i.use_whitelist)
    i.user_mem_reply                         0x0001e9bc   Section        0  nrf_ble_qwr.o(i.user_mem_reply)
    user_mem_reply                           0x0001e9bd   Thumb Code    36  nrf_ble_qwr.o(i.user_mem_reply)
    i.user_op_alloc                          0x0001e9e0   Section        0  app_timer.o(i.user_op_alloc)
    user_op_alloc                            0x0001e9e1   Thumb Code    42  app_timer.o(i.user_op_alloc)
    i.uuid_list_encode                       0x0001ea10   Section        0  ble_advdata.o(i.uuid_list_encode)
    uuid_list_encode                         0x0001ea11   Thumb Code    48  ble_advdata.o(i.uuid_list_encode)
    i.uuid_list_sized_encode                 0x0001ea40   Section        0  ble_advdata.o(i.uuid_list_sized_encode)
    uuid_list_sized_encode                   0x0001ea41   Thumb Code   158  ble_advdata.o(i.uuid_list_sized_encode)
    i.wakeup_button_cfg                      0x0001eade   Section        0  bsp.o(i.wakeup_button_cfg)
    wakeup_button_cfg                        0x0001eadf   Thumb Code    58  bsp.o(i.wakeup_button_cfg)
    .constdata                               0x0001eb18   Section       68  main.o(.constdata)
    m_heart_rate_timer_id                    0x0001eb18   Data           4  main.o(.constdata)
    delay_bytecode                           0x0001eb1c   Data           6  main.o(.constdata)
    m_twi                                    0x0001eb24   Data          16  main.o(.constdata)
    .constdata                               0x0001eb5c   Section        8  boards.o(.constdata)
    m_board_led_list                         0x0001eb5c   Data           4  boards.o(.constdata)
    m_board_btn_list                         0x0001eb60   Data           4  boards.o(.constdata)
    .constdata                               0x0001eb64   Section       44  bsp.o(.constdata)
    m_bsp_leds_tmr                           0x0001eb64   Data           4  bsp.o(.constdata)
    m_bsp_alert_tmr                          0x0001eb68   Data           4  bsp.o(.constdata)
    m_bsp_button_tmr                         0x0001eb6c   Data           4  bsp.o(.constdata)
    app_buttons                              0x0001eb70   Data          32  bsp.o(.constdata)
    .constdata                               0x0001eb90   Section       14  nrf_ble_gatt.o(.constdata)
    .constdata                               0x0001eba0   Section       16  ble_nus.o(.constdata)
    .constdata                               0x0001ebb0   Section        4  nrfx_gpiote.o(.constdata)
    .constdata                               0x0001ebb4   Section        4  nrfx_uarte.o(.constdata)
    irq_handlers                             0x0001ebb4   Data           4  nrfx_uarte.o(.constdata)
    .constdata                               0x0001ebb8   Section       24  nrfx_twim.o(.constdata)
    irq_handlers                             0x0001ebb8   Data           4  nrfx_twim.o(.constdata)
    .constdata                               0x0001ebd0   Section        6  nrf_drv_twi.o(.constdata)
    delay_bytecode                           0x0001ebd0   Data           6  nrf_drv_twi.o(.constdata)
    .constdata                               0x0001ebd6   Section        6  app_timer.o(.constdata)
    delay_bytecode                           0x0001ebd6   Data           6  app_timer.o(.constdata)
    .constdata                               0x0001ebdc   Section       32  app_uart_fifo.o(.constdata)
    .constdata                               0x0001ebfc   Section       16  nrf_fprintf_format.o(.constdata)
    _aV2C                                    0x0001ebfc   Data          16  nrf_fprintf_format.o(.constdata)
    .constdata                               0x0001ec0c   Section       24  nrf_pwr_mgmt.o(.constdata)
    pwr_mgmt_data_array                      0x0001ec0c   Data          24  nrf_pwr_mgmt.o(.constdata)
    .constdata                               0x0001ec24   Section       12  nrf_pwr_mgmt.o(.constdata)
    pwr_mgmt_data                            0x0001ec24   Data          12  nrf_pwr_mgmt.o(.constdata)
    .constdata                               0x0001ec30   Section      316  nrf_strerror.o(.constdata)
    m_unknown_str                            0x0001ec30   Data          19  nrf_strerror.o(.constdata)
    nrf_strerror_array                       0x0001ec44   Data         296  nrf_strerror.o(.constdata)
    .constdata                               0x0001ed6c   Section       12  nrf_log_backend_rtt.o(.constdata)
    .constdata                               0x0001ed78   Section        6  nrf_log_backend_rtt.o(.constdata)
    delay_bytecode                           0x0001ed78   Data           6  nrf_log_backend_rtt.o(.constdata)
    .constdata                               0x0001ed80   Section       12  nrf_log_frontend.o(.constdata)
    m_log_push_ringbuf                       0x0001ed80   Data          12  nrf_log_frontend.o(.constdata)
    .constdata                               0x0001ed8c   Section       16  nrf_sdh.o(.constdata)
    sdh_req_observers_array                  0x0001ed8c   Data          16  nrf_sdh.o(.constdata)
    .constdata                               0x0001ed9c   Section       40  nrf_sdh.o(.constdata)
    sdh_req_observers                        0x0001eda0   Data          12  nrf_sdh.o(.constdata)
    sdh_state_observers                      0x0001edac   Data          12  nrf_sdh.o(.constdata)
    sdh_stack_observers                      0x0001edb8   Data          12  nrf_sdh.o(.constdata)
    .constdata                               0x0001edc4   Section       16  nrf_sdh.o(.constdata)
    sdh_state_observers_array                0x0001edc4   Data          16  nrf_sdh.o(.constdata)
    .constdata                               0x0001edd4   Section       16  nrf_sdh.o(.constdata)
    sdh_stack_observers_array                0x0001edd4   Data          16  nrf_sdh.o(.constdata)
    .constdata                               0x0001ede4   Section       32  nrf_sdh_ble.o(.constdata)
    sdh_ble_observers_array                  0x0001ede4   Data          32  nrf_sdh_ble.o(.constdata)
    .constdata                               0x0001ee04   Section       16  nrf_sdh_ble.o(.constdata)
    sdh_ble_observers                        0x0001ee08   Data          12  nrf_sdh_ble.o(.constdata)
    .constdata                               0x0001ee14   Section       16  nrf_sdh_soc.o(.constdata)
    sdh_soc_observers_array                  0x0001ee14   Data          16  nrf_sdh_soc.o(.constdata)
    .constdata                               0x0001ee24   Section       12  nrf_sdh_soc.o(.constdata)
    sdh_soc_observers                        0x0001ee24   Data          12  nrf_sdh_soc.o(.constdata)
    .constdata                               0x0001ee30   Section      129  ctype_o.o(.constdata)
    .constdata                               0x0001eeb4   Section        4  ctype_o.o(.constdata)
    table                                    0x0001eeb4   Data           4  ctype_o.o(.constdata)
    .conststring                             0x0001eeb8   Section     1003  nrf_strerror.o(.conststring)
    .conststring                             0x0001f2a4   Section      102  nrf_log_str_formatter.o(.conststring)
    .conststring                             0x0001f30c   Section      463  nrf_sdh_ble.o(.conststring)
    .conststrlit                             0x0001f4dc   Section       13  nrf_ble_gatt.o(.conststrlit)
    .conststrlit                             0x0001f4ec   Section        8  ble_nus.o(.conststrlit)
    .conststrlit                             0x0001f4f4   Section        6  nrf_drv_clock.o(.conststrlit)
    .conststrlit                             0x0001f4fc   Section        6  nrfx_clock.o(.conststrlit)
    .conststrlit                             0x0001f504   Section        7  nrfx_gpiote.o(.conststrlit)
    .conststrlit                             0x0001f50c   Section        4  nrfx_prs.o(.conststrlit)
    .conststrlit                             0x0001f510   Section        6  nrfx_uarte.o(.conststrlit)
    .conststrlit                             0x0001f518   Section        5  nrfx_twim.o(.conststrlit)
    .conststrlit                             0x0001f520   Section        9  nrf_pwr_mgmt.o(.conststrlit)
    .conststrlit                             0x0001f52c   Section       16  nrf_log_default_backends.o(.conststrlit)
    .conststrlit                             0x0001f53c   Section        4  nrf_log_frontend.o(.conststrlit)
    .conststrlit                             0x0001f540   Section        8  nrf_sdh.o(.conststrlit)
    .conststrlit                             0x0001f548   Section       12  nrf_sdh_ble.o(.conststrlit)
    .conststrlit                             0x0001f554   Section       12  nrf_sdh_soc.o(.conststrlit)
    log_backends                             0x0001f580   Section       16  nrf_log_default_backends.o(log_backends)
    __tagsym$$used                           0x0001f580   Number         0  nrf_log_default_backends.o(log_backends)
    rtt_log_backend                          0x0001f580   Data          16  nrf_log_default_backends.o(log_backends)
    log_const_data                           0x0001f590   Section        8  nrf_ble_gatt.o(log_const_data)
    __tagsym$$used                           0x0001f590   Number         0  nrf_ble_gatt.o(log_const_data)
    log_const_data                           0x0001f598   Section        8  ble_nus.o(log_const_data)
    __tagsym$$used                           0x0001f598   Number         0  ble_nus.o(log_const_data)
    log_const_data                           0x0001f5a0   Section        8  nrf_drv_clock.o(log_const_data)
    __tagsym$$used                           0x0001f5a0   Number         0  nrf_drv_clock.o(log_const_data)
    log_const_data                           0x0001f5a8   Section        8  nrfx_clock.o(log_const_data)
    __tagsym$$used                           0x0001f5a8   Number         0  nrfx_clock.o(log_const_data)
    log_const_data                           0x0001f5b0   Section        8  nrfx_gpiote.o(log_const_data)
    __tagsym$$used                           0x0001f5b0   Number         0  nrfx_gpiote.o(log_const_data)
    log_const_data                           0x0001f5b8   Section        8  nrfx_prs.o(log_const_data)
    __tagsym$$used                           0x0001f5b8   Number         0  nrfx_prs.o(log_const_data)
    log_const_data                           0x0001f5c0   Section        8  nrfx_uarte.o(log_const_data)
    __tagsym$$used                           0x0001f5c0   Number         0  nrfx_uarte.o(log_const_data)
    log_const_data                           0x0001f5c8   Section        8  nrfx_twim.o(log_const_data)
    __tagsym$$used                           0x0001f5c8   Number         0  nrfx_twim.o(log_const_data)
    log_const_data                           0x0001f5d0   Section        8  nrf_pwr_mgmt.o(log_const_data)
    __tagsym$$used                           0x0001f5d0   Number         0  nrf_pwr_mgmt.o(log_const_data)
    log_const_data                           0x0001f5d8   Section        8  nrf_log_frontend.o(log_const_data)
    __tagsym$$used                           0x0001f5d8   Number         0  nrf_log_frontend.o(log_const_data)
    log_const_data                           0x0001f5e0   Section        8  nrf_sdh.o(log_const_data)
    __tagsym$$used                           0x0001f5e0   Number         0  nrf_sdh.o(log_const_data)
    log_const_data                           0x0001f5e8   Section        8  nrf_sdh_ble.o(log_const_data)
    __tagsym$$used                           0x0001f5e8   Number         0  nrf_sdh_ble.o(log_const_data)
    log_const_data                           0x0001f5f0   Section        8  nrf_sdh_soc.o(log_const_data)
    __tagsym$$used                           0x0001f5f0   Number         0  nrf_sdh_soc.o(log_const_data)
    nrf_balloc                               0x0001f5f8   Section       20  nrf_log_frontend.o(nrf_balloc)
    __tagsym$$used                           0x0001f5f8   Number         0  nrf_log_frontend.o(nrf_balloc)
    sdh_ble_observers0                       0x0001f60c   Section        8  ble_conn_state.o(sdh_ble_observers0)
    __tagsym$$used                           0x0001f60c   Number         0  ble_conn_state.o(sdh_ble_observers0)
    m_ble_evt_observer                       0x0001f60c   Data           8  ble_conn_state.o(sdh_ble_observers0)
    sdh_ble_observers1                       0x0001f614   Section       16  main.o(sdh_ble_observers1)
    __tagsym$$used                           0x0001f614   Number         0  main.o(sdh_ble_observers1)
    m_gatt_obs                               0x0001f614   Data           8  main.o(sdh_ble_observers1)
    __tagsym$$used                           0x0001f61c   Number         0  main.o(sdh_ble_observers1)
    m_advertising_ble_obs                    0x0001f61c   Data           8  main.o(sdh_ble_observers1)
    sdh_ble_observers1                       0x0001f624   Section        8  bsp_btn_ble.o(sdh_ble_observers1)
    __tagsym$$used                           0x0001f624   Number         0  bsp_btn_ble.o(sdh_ble_observers1)
    m_ble_observer                           0x0001f624   Data           8  bsp_btn_ble.o(sdh_ble_observers1)
    sdh_ble_observers1                       0x0001f62c   Section        8  ble_conn_params.o(sdh_ble_observers1)
    __tagsym$$used                           0x0001f62c   Number         0  ble_conn_params.o(sdh_ble_observers1)
    m_ble_observer                           0x0001f62c   Data           8  ble_conn_params.o(sdh_ble_observers1)
    sdh_ble_observers2                       0x0001f634   Section       16  main.o(sdh_ble_observers2)
    __tagsym$$used                           0x0001f634   Number         0  main.o(sdh_ble_observers2)
    m_nus_obs                                0x0001f634   Data           8  main.o(sdh_ble_observers2)
    __tagsym$$used                           0x0001f63c   Number         0  main.o(sdh_ble_observers2)
    m_qwr_obs                                0x0001f63c   Data           8  main.o(sdh_ble_observers2)
    sdh_ble_observers3                       0x0001f644   Section        8  main.o(sdh_ble_observers3)
    __tagsym$$used                           0x0001f644   Number         0  main.o(sdh_ble_observers3)
    m_ble_observer                           0x0001f644   Data           8  main.o(sdh_ble_observers3)
    sdh_soc_observers0                       0x0001f64c   Section        8  nrf_drv_clock.o(sdh_soc_observers0)
    __tagsym$$used                           0x0001f64c   Number         0  nrf_drv_clock.o(sdh_soc_observers0)
    m_soc_evt_observer                       0x0001f64c   Data           8  nrf_drv_clock.o(sdh_soc_observers0)
    sdh_soc_observers1                       0x0001f654   Section        8  main.o(sdh_soc_observers1)
    __tagsym$$used                           0x0001f654   Number         0  main.o(sdh_soc_observers1)
    m_advertising_soc_obs                    0x0001f654   Data           8  main.o(sdh_soc_observers1)
    sdh_stack_observers0                     0x0001f65c   Section        8  nrf_sdh_ble.o(sdh_stack_observers0)
    __tagsym$$used                           0x0001f65c   Number         0  nrf_sdh_ble.o(sdh_stack_observers0)
    m_nrf_sdh_ble_evts_poll                  0x0001f65c   Data           8  nrf_sdh_ble.o(sdh_stack_observers0)
    sdh_stack_observers0                     0x0001f664   Section        8  nrf_sdh_soc.o(sdh_stack_observers0)
    __tagsym$$used                           0x0001f664   Number         0  nrf_sdh_soc.o(sdh_stack_observers0)
    m_nrf_sdh_soc_evts_poll                  0x0001f664   Data           8  nrf_sdh_soc.o(sdh_stack_observers0)
    sdh_state_observers0                     0x0001f66c   Section        8  nrf_drv_clock.o(sdh_state_observers0)
    __tagsym$$used                           0x0001f66c   Number         0  nrf_drv_clock.o(sdh_state_observers0)
    m_sd_state_observer                      0x0001f66c   Data           8  nrf_drv_clock.o(sdh_state_observers0)
    .data                                    0x20002500   Section        8  main.o(.data)
    m_nus_link_ctx_storage                   0x20002500   Data           8  main.o(.data)
    .data                                    0x20002508   Section       52  main.o(.data)
    m_xfer_done                              0x20002508   Data           1  main.o(.data)
    twi_status                               0x20002509   Data           1  main.o(.data)
    index                                    0x2000250a   Data           1  main.o(.data)
    m_sample                                 0x2000250b   Data           1  main.o(.data)
    sensor_temp                              0x2000250c   Data           1  main.o(.data)
    sensor_humi                              0x2000250d   Data           1  main.o(.data)
    m_conn_handle                            0x2000250e   Data           2  main.o(.data)
    m_ble_nus_max_data_len                   0x20002510   Data           2  main.o(.data)
    m_adv_uuids                              0x20002512   Data           4  main.o(.data)
    device_id                                0x20002516   Data           4  main.o(.data)
    ens210_buf                               0x2000251a   Data           6  main.o(.data)
    m_nus                                    0x20002520   Data          28  main.o(.data)
    .data                                    0x2000253c   Section        4  main.o(.data)
    m_nus_link_ctx_storage_ctx_data_pool     0x2000253c   Data           4  main.o(.data)
    .data                                    0x20002540   Section       16  bsp.o(.data)
    m_stable_state                           0x20002540   Data           1  bsp.o(.data)
    m_leds_clear                             0x20002541   Data           1  bsp.o(.data)
    m_alert_on                               0x20002542   Data           1  bsp.o(.data)
    current_long_push_pin_no                 0x20002543   Data           1  bsp.o(.data)
    m_indication_type                        0x20002544   Data           4  bsp.o(.data)
    m_registered_callback                    0x20002548   Data           4  bsp.o(.data)
    release_event_at_push                    0x2000254c   Data           4  bsp.o(.data)
    .data                                    0x20002550   Section        8  bsp_btn_ble.o(.data)
    m_error_handler                          0x20002550   Data           4  bsp_btn_ble.o(.data)
    m_num_connections                        0x20002554   Data           4  bsp_btn_ble.o(.data)
    .data                                    0x20002558   Section        8  ble_conn_params.o(.data)
    m_preferred_conn_params                  0x20002558   Data           8  ble_conn_params.o(.data)
    .data                                    0x20002560   Section        8  nrf_drv_uart.o(.data)
    m_handlers                               0x20002560   Data           4  nrf_drv_uart.o(.data)
    m_contexts                               0x20002564   Data           4  nrf_drv_uart.o(.data)
    .data                                    0x20002568   Section        8  nrfx_clock.o(.data)
    m_clock_cb                               0x20002568   Data           8  nrfx_clock.o(.data)
    .data                                    0x20002570   Section        8  nrf_drv_twi.o(.data)
    m_handlers                               0x20002570   Data           4  nrf_drv_twi.o(.data)
    m_contexts                               0x20002574   Data           4  nrf_drv_twi.o(.data)
    .data                                    0x20002578   Section       20  app_timer.o(.data)
    m_ticks_elapsed_q_read_ind               0x20002578   Data           1  app_timer.o(.data)
    m_ticks_elapsed_q_write_ind              0x20002579   Data           1  app_timer.o(.data)
    m_rtc1_running                           0x2000257a   Data           1  app_timer.o(.data)
    m_rtc1_reset                             0x2000257b   Data           1  app_timer.o(.data)
    mp_timer_id_head                         0x2000257c   Data           4  app_timer.o(.data)
    m_ticks_latest                           0x20002580   Data           4  app_timer.o(.data)
    m_ticks_elapsed                          0x20002584   Data           8  app_timer.o(.data)
    .data                                    0x2000258c   Section       20  app_uart_fifo.o(.data)
    tx_buffer                                0x2000258c   Data           1  app_uart_fifo.o(.data)
    rx_buffer                                0x2000258d   Data           1  app_uart_fifo.o(.data)
    m_rx_ovf                                 0x2000258e   Data           1  app_uart_fifo.o(.data)
    m_event_handler                          0x20002590   Data           4  app_uart_fifo.o(.data)
    app_uart_inst                            0x20002594   Data          12  app_uart_fifo.o(.data)
    .data                                    0x200025a0   Section        8  nrf_pwr_mgmt.o(.data)
    m_pwr_mgmt_evt                           0x200025a0   Data           1  nrf_pwr_mgmt.o(.data)
    m_shutdown_started                       0x200025a1   Data           1  nrf_pwr_mgmt.o(.data)
    m_sysoff_mtx                             0x200025a4   Data           4  nrf_pwr_mgmt.o(.data)
    .data                                    0x200025a8   Section        1  nrf_log_backend_rtt.o(.data)
    m_host_present                           0x200025a8   Data           1  nrf_log_backend_rtt.o(.data)
    .data                                    0x200025ac   Section        8  nrf_log_default_backends.o(.data)
    log_backend_cb_rtt_log_backend           0x200025ac   Data           8  nrf_log_default_backends.o(.data)
    .data                                    0x200025b4   Section        8  nrf_log_frontend.o(.data)
    log_mempool_nrf_balloc_pool_stack        0x200025b4   Data           8  nrf_log_frontend.o(.data)
    .data                                    0x200025bc   Section        8  nrf_log_frontend.o(.data)
    log_mempool_nrf_balloc_cb                0x200025bc   Data           8  nrf_log_frontend.o(.data)
    .data                                    0x200025c4   Section       64  nrf_log_str_formatter.o(.data)
    m_freq                                   0x200025c4   Data           4  nrf_log_str_formatter.o(.data)
    m_timestamp_div                          0x200025c8   Data           4  nrf_log_str_formatter.o(.data)
    severity_names                           0x200025cc   Data          20  nrf_log_str_formatter.o(.data)
    m_colors                                 0x200025e0   Data          36  nrf_log_str_formatter.o(.data)
    .data                                    0x20002604   Section        3  nrf_sdh.o(.data)
    m_nrf_sdh_enabled                        0x20002604   Data           1  nrf_sdh.o(.data)
    m_nrf_sdh_suspended                      0x20002605   Data           1  nrf_sdh.o(.data)
    m_nrf_sdh_continue                       0x20002606   Data           1  nrf_sdh.o(.data)
    .data                                    0x20002607   Section        1  nrf_sdh_ble.o(.data)
    m_stack_is_enabled                       0x20002607   Data           1  nrf_sdh_ble.o(.data)
    .data                                    0x20002608   Section        4  system_nrf52810.o(.data)
    __tagsym$$used                           0x20002608   Number         0  system_nrf52810.o(.data)
    .data                                    0x2000260c   Section        4  mvars.o(.data)
    .data                                    0x20002610   Section        4  mvars.o(.data)
    .bss                                     0x20002614   Section       32  main.o(.bss)
    m_heart_rate_timer_id_data               0x20002614   Data          32  main.o(.bss)
    .bss                                     0x20002634   Section      968  main.o(.bss)
    data_array                               0x20002634   Data         244  main.o(.bss)
    rx_buf                                   0x20002728   Data         256  main.o(.bss)
    tx_buf                                   0x20002828   Data         256  main.o(.bss)
    m_gatt                                   0x20002928   Data          16  main.o(.bss)
    m_qwr                                    0x20002938   Data          12  main.o(.bss)
    m_advertising                            0x20002944   Data         184  main.o(.bss)
    .bss                                     0x200029fc   Section       32  bsp.o(.bss)
    m_bsp_leds_tmr_data                      0x200029fc   Data          32  bsp.o(.bss)
    .bss                                     0x20002a1c   Section       32  bsp.o(.bss)
    m_bsp_alert_tmr_data                     0x20002a1c   Data          32  bsp.o(.bss)
    .bss                                     0x20002a3c   Section       12  bsp.o(.bss)
    m_events_list                            0x20002a3c   Data          12  bsp.o(.bss)
    .bss                                     0x20002a48   Section       32  bsp.o(.bss)
    m_bsp_button_tmr_data                    0x20002a48   Data          32  bsp.o(.bss)
    .bss                                     0x20002a68   Section       80  ble_conn_params.o(.bss)
    m_timer_data                             0x20002a68   Data          32  ble_conn_params.o(.bss)
    m_conn_params_instances                  0x20002a88   Data          20  ble_conn_params.o(.bss)
    m_conn_params_config                     0x20002a9c   Data          28  ble_conn_params.o(.bss)
    .bss                                     0x20002ab8   Section      120  ble_conn_state.o(.bss)
    m_bcs                                    0x20002ab8   Data         120  ble_conn_state.o(.bss)
    .bss                                     0x20002b30   Section       20  nrf_drv_clock.o(.bss)
    m_clock_cb                               0x20002b30   Data          20  nrf_drv_clock.o(.bss)
    .bss                                     0x20002b44   Section       92  nrfx_gpiote.o(.bss)
    m_cb                                     0x20002b44   Data          92  nrfx_gpiote.o(.bss)
    .bss                                     0x20002ba0   Section       36  nrfx_uarte.o(.bss)
    m_cb                                     0x20002ba0   Data          36  nrfx_uarte.o(.bss)
    .bss                                     0x20002bc4   Section       52  nrfx_twim.o(.bss)
    m_cb                                     0x20002bc4   Data          52  nrfx_twim.o(.bss)
    .bss                                     0x20002bf8   Section      268  app_timer.o(.bss)
    m_op_queue                               0x20002bf8   Data         268  app_timer.o(.bss)
    .bss                                     0x20002d04   Section       32  app_uart_fifo.o(.bss)
    m_rx_fifo                                0x20002d04   Data          16  app_uart_fifo.o(.bss)
    m_tx_fifo                                0x20002d14   Data          16  app_uart_fifo.o(.bss)
    .bss                                     0x20002d24   Section       12  app_util_platform.o(.bss)
    .bss                                     0x20002d30   Section       12  nrf_pwr_mgmt.o(.bss)
    m_handlers_iter                          0x20002d30   Data          12  nrf_pwr_mgmt.o(.bss)
    .bss                                     0x20002d3c   Section       64  nrf_log_backend_rtt.o(.bss)
    m_string_buff                            0x20002d3c   Data          64  nrf_log_backend_rtt.o(.bss)
    .bss                                     0x20002d7c   Section      192  nrf_log_frontend.o(.bss)
    log_mempool_nrf_balloc_pool_mem          0x20002d7c   Data         192  nrf_log_frontend.o(.bss)
    .bss                                     0x20002e3c   Section      128  nrf_log_frontend.o(.bss)
    m_log_push_ringbuf_buf                   0x20002e3c   Data         128  nrf_log_frontend.o(.bss)
    .bss                                     0x20002ebc   Section       24  nrf_log_frontend.o(.bss)
    m_log_push_ringbuf_cb                    0x20002ebc   Data          24  nrf_log_frontend.o(.bss)
    .bss                                     0x20002ed4   Section     1060  nrf_log_frontend.o(.bss)
    m_log_data                               0x20002ed4   Data        1060  nrf_log_frontend.o(.bss)
    .bss                                     0x200032f8   Section      648  segger_rtt.o(.bss)
    _acUpBuffer                              0x20003370   Data         512  segger_rtt.o(.bss)
    _acDownBuffer                            0x20003570   Data          16  segger_rtt.o(.bss)
    HEAP                                     0x20003580   Section     2048  arm_startup_nrf52810.o(HEAP)
    STACK                                    0x20003d80   Section     2048  arm_startup_nrf52810.o(STACK)

    Global Symbols

    Symbol Name                              Value     Ov Type        Size  Object(Section)

    BuildAttributes$$THM_ISAv4$E$P$D$K$B$S$7EM$PE$A:L22UL41UL21$X:L11$S22US41US21$IEEE1$IW$USESV6$~STKCKD$USESV7$~SHL$OTIME$ROPI$EBA8$MICROLIB$REQ8$EABIv2 0x00000000   Number         0  anon$$obj.o ABSOLUTE
    __ARM_use_no_argv                        0x00000000   Number         0  main.o ABSOLUTE
    __cpp_initialize__aeabi_                  - Undefined Weak Reference
    __cxa_finalize                            - Undefined Weak Reference
    __decompress                              - Undefined Weak Reference
    _clock_init                               - Undefined Weak Reference
    _microlib_exit                            - Undefined Weak Reference
    log_dynamic_data$$Base                    - Undefined Reference
    pwr_mgmt_data0$$Base                      - Undefined Reference
    pwr_mgmt_data0$$Limit                     - Undefined Reference
    pwr_mgmt_data1$$Base                      - Undefined Reference
    pwr_mgmt_data1$$Limit                     - Undefined Reference
    pwr_mgmt_data2$$Base                      - Undefined Reference
    pwr_mgmt_data2$$Limit                     - Undefined Reference
    sdh_req_observers0$$Base                  - Undefined Reference
    sdh_req_observers0$$Limit                 - Undefined Reference
    sdh_req_observers1$$Base                  - Undefined Reference
    sdh_req_observers1$$Limit                 - Undefined Reference
    sdh_stack_observers1$$Base                - Undefined Reference
    sdh_stack_observers1$$Limit               - Undefined Reference
    sdh_state_observers1$$Base                - Undefined Reference
    sdh_state_observers1$$Limit               - Undefined Reference
    __Vectors_Size                           0x00000200   Number         0  arm_startup_nrf52810.o ABSOLUTE
    __Vectors                                0x00019000   Data           4  arm_startup_nrf52810.o(RESET)
    __Vectors_End                            0x00019200   Data           0  arm_startup_nrf52810.o(RESET)
    __main                                   0x00019201   Thumb Code     0  entry.o(.ARM.Collect$$$$00000000)
    _main_stk                                0x00019201   Thumb Code     0  entry2.o(.ARM.Collect$$$$00000001)
    _main_scatterload                        0x00019205   Thumb Code     0  entry5.o(.ARM.Collect$$$$00000004)
    __main_after_scatterload                 0x00019209   Thumb Code     0  entry5.o(.ARM.Collect$$$$00000004)
    _main_clock                              0x00019209   Thumb Code     0  entry7b.o(.ARM.Collect$$$$00000008)
    _main_cpp_init                           0x00019209   Thumb Code     0  entry8b.o(.ARM.Collect$$$$0000000A)
    _main_init                               0x00019209   Thumb Code     0  entry9a.o(.ARM.Collect$$$$0000000B)
    __rt_final_cpp                           0x00019211   Thumb Code     0  entry10a.o(.ARM.Collect$$$$0000000D)
    __rt_final_exit                          0x00019211   Thumb Code     0  entry11a.o(.ARM.Collect$$$$0000000F)
    __asm___12_nrf_atomic_c_85ca2469__nrf_atomic_internal_mov 0x00019215   Thumb Code    24  nrf_atomic.o(.emb_text)
    __asm___12_nrf_atomic_c_85ca2469__nrf_atomic_internal_orr 0x0001922d   Thumb Code    26  nrf_atomic.o(.emb_text)
    __asm___12_nrf_atomic_c_85ca2469__nrf_atomic_internal_and 0x00019247   Thumb Code    26  nrf_atomic.o(.emb_text)
    __asm___12_nrf_atomic_c_85ca2469__nrf_atomic_internal_eor 0x00019261   Thumb Code    26  nrf_atomic.o(.emb_text)
    __asm___12_nrf_atomic_c_85ca2469__nrf_atomic_internal_add 0x0001927b   Thumb Code    26  nrf_atomic.o(.emb_text)
    __asm___12_nrf_atomic_c_85ca2469__nrf_atomic_internal_sub 0x00019295   Thumb Code    26  nrf_atomic.o(.emb_text)
    __asm___12_nrf_atomic_c_85ca2469__nrf_atomic_internal_cmp_exch 0x000192af   Thumb Code    42  nrf_atomic.o(.emb_text)
    __asm___12_nrf_atomic_c_85ca2469__nrf_atomic_internal_sub_hs 0x000192d9   Thumb Code    30  nrf_atomic.o(.emb_text)
    Reset_Handler                            0x000192f9   Thumb Code     8  arm_startup_nrf52810.o(.text)
    NMI_Handler                              0x00019301   Thumb Code     2  arm_startup_nrf52810.o(.text)
    HardFault_Handler                        0x00019303   Thumb Code     2  arm_startup_nrf52810.o(.text)
    MemoryManagement_Handler                 0x00019305   Thumb Code     2  arm_startup_nrf52810.o(.text)
    BusFault_Handler                         0x00019307   Thumb Code     2  arm_startup_nrf52810.o(.text)
    UsageFault_Handler                       0x00019309   Thumb Code     2  arm_startup_nrf52810.o(.text)
    SVC_Handler                              0x0001930b   Thumb Code     2  arm_startup_nrf52810.o(.text)
    DebugMon_Handler                         0x0001930d   Thumb Code     2  arm_startup_nrf52810.o(.text)
    PendSV_Handler                           0x0001930f   Thumb Code     2  arm_startup_nrf52810.o(.text)
    SysTick_Handler                          0x00019311   Thumb Code     2  arm_startup_nrf52810.o(.text)
    CCM_AAR_IRQHandler                       0x00019313   Thumb Code     0  arm_startup_nrf52810.o(.text)
    COMP_IRQHandler                          0x00019313   Thumb Code     0  arm_startup_nrf52810.o(.text)
    ECB_IRQHandler                           0x00019313   Thumb Code     0  arm_startup_nrf52810.o(.text)
    PDM_IRQHandler                           0x00019313   Thumb Code     0  arm_startup_nrf52810.o(.text)
    PWM0_IRQHandler                          0x00019313   Thumb Code     0  arm_startup_nrf52810.o(.text)
    QDEC_IRQHandler                          0x00019313   Thumb Code     0  arm_startup_nrf52810.o(.text)
    RADIO_IRQHandler                         0x00019313   Thumb Code     0  arm_startup_nrf52810.o(.text)
    RNG_IRQHandler                           0x00019313   Thumb Code     0  arm_startup_nrf52810.o(.text)
    RTC0_IRQHandler                          0x00019313   Thumb Code     0  arm_startup_nrf52810.o(.text)
    SAADC_IRQHandler                         0x00019313   Thumb Code     0  arm_startup_nrf52810.o(.text)
    SPIM0_SPIS0_IRQHandler                   0x00019313   Thumb Code     0  arm_startup_nrf52810.o(.text)
    SWI1_EGU1_IRQHandler                     0x00019313   Thumb Code     0  arm_startup_nrf52810.o(.text)
    SWI3_IRQHandler                          0x00019313   Thumb Code     0  arm_startup_nrf52810.o(.text)
    SWI4_IRQHandler                          0x00019313   Thumb Code     0  arm_startup_nrf52810.o(.text)
    SWI5_IRQHandler                          0x00019313   Thumb Code     0  arm_startup_nrf52810.o(.text)
    TEMP_IRQHandler                          0x00019313   Thumb Code     0  arm_startup_nrf52810.o(.text)
    TIMER0_IRQHandler                        0x00019313   Thumb Code     0  arm_startup_nrf52810.o(.text)
    TIMER1_IRQHandler                        0x00019313   Thumb Code     0  arm_startup_nrf52810.o(.text)
    TIMER2_IRQHandler                        0x00019313   Thumb Code     0  arm_startup_nrf52810.o(.text)
    WDT_IRQHandler                           0x00019313   Thumb Code     0  arm_startup_nrf52810.o(.text)
    __aeabi_uldivmod                         0x0001931d   Thumb Code    98  uldiv.o(.text)
    __aeabi_llsl                             0x0001937f   Thumb Code    30  llshl.o(.text)
    _ll_shift_l                              0x0001937f   Thumb Code     0  llshl.o(.text)
    __rt_ctype_table                         0x0001939d   Thumb Code     4  ctype_o.o(.text)
    __aeabi_memcpy                           0x000193a5   Thumb Code    36  memcpya.o(.text)
    __aeabi_memcpy4                          0x000193a5   Thumb Code     0  memcpya.o(.text)
    __aeabi_memcpy8                          0x000193a5   Thumb Code     0  memcpya.o(.text)
    __aeabi_memset                           0x000193c9   Thumb Code    14  memseta.o(.text)
    __aeabi_memset4                          0x000193c9   Thumb Code     0  memseta.o(.text)
    __aeabi_memset8                          0x000193c9   Thumb Code     0  memseta.o(.text)
    __aeabi_memclr                           0x000193d7   Thumb Code     4  memseta.o(.text)
    __aeabi_memclr4                          0x000193d7   Thumb Code     0  memseta.o(.text)
    __aeabi_memclr8                          0x000193d7   Thumb Code     0  memseta.o(.text)
    _memset$wrapper                          0x000193db   Thumb Code    18  memseta.o(.text)
    strlen                                   0x000193ed   Thumb Code    14  strlen.o(.text)
    strcpy                                   0x000193fb   Thumb Code    18  strcpy.o(.text)
    __aeabi_fadd                             0x0001940d   Thumb Code   164  fadd.o(.text)
    __aeabi_fsub                             0x000194b1   Thumb Code     6  fadd.o(.text)
    __aeabi_frsub                            0x000194b7   Thumb Code     6  fadd.o(.text)
    __ARM_scalbnf                            0x000194bd   Thumb Code    24  fscalb.o(.text)
    scalbnf                                  0x000194bd   Thumb Code     0  fscalb.o(.text)
    __aeabi_ui2f                             0x000194d5   Thumb Code    10  ffltui.o(.text)
    __aeabi_f2uiz                            0x000194df   Thumb Code    40  ffixui.o(.text)
    __aeabi_llsr                             0x00019507   Thumb Code    32  llushr.o(.text)
    _ll_ushift_r                             0x00019507   Thumb Code     0  llushr.o(.text)
    __I$use$fp                               0x00019527   Thumb Code     0  iusefp.o(.text)
    _float_round                             0x00019527   Thumb Code    18  fepilogue.o(.text)
    _float_epilogue                          0x00019539   Thumb Code    92  fepilogue.o(.text)
    __scatterload                            0x00019595   Thumb Code    28  init.o(.text)
    __scatterload_rt2                        0x00019595   Thumb Code     0  init.o(.text)
    ENS210_set_mode                          0x000195b9   Thumb Code   206  main.o(i.ENS210_set_mode)
    GPIOTE_IRQHandler                        0x0001969d   Thumb Code   346  nrfx_gpiote.o(i.GPIOTE_IRQHandler)
    POWER_CLOCK_IRQHandler                   0x00019865   Thumb Code    82  nrfx_clock.o(i.POWER_CLOCK_IRQHandler)
    RTC1_IRQHandler                          0x000198bd   Thumb Code    32  app_timer.o(i.RTC1_IRQHandler)
    SEGGER_RTT_Init                          0x000198e1   Thumb Code     4  segger_rtt.o(i.SEGGER_RTT_Init)
    SEGGER_RTT_WriteNoLock                   0x000198e5   Thumb Code    86  segger_rtt.o(i.SEGGER_RTT_WriteNoLock)
    SWI0_EGU0_IRQHandler                     0x00019941   Thumb Code     4  app_timer.o(i.SWI0_EGU0_IRQHandler)
    SWI2_IRQHandler                          0x00019945   Thumb Code     4  nrf_sdh.o(i.SWI2_IRQHandler)
    SystemInit                               0x00019949   Thumb Code   676  system_nrf52810.o(i.SystemInit)
    TWIM0_TWIS0_IRQHandler                   0x00019c35   Thumb Code     8  nrfx_twim.o(i.TWIM0_TWIS0_IRQHandler)
    UARTE0_IRQHandler                        0x00019c45   Thumb Code     8  nrfx_uarte.o(i.UARTE0_IRQHandler)
    __scatterload_copy                       0x00019d6f   Thumb Code    14  handlers.o(i.__scatterload_copy)
    __scatterload_null                       0x00019d7d   Thumb Code     2  handlers.o(i.__scatterload_null)
    __scatterload_zeroinit                   0x00019d7f   Thumb Code    14  handlers.o(i.__scatterload_zeroinit)
    app_error_fault_handler                  0x00019de9   Thumb Code    86  app_error_weak.o(i.app_error_fault_handler)
    app_error_handler_bare                   0x00019e6d   Thumb Code    22  app_error.o(i.app_error_handler_bare)
    app_fifo_get                             0x00019e83   Thumb Code    22  app_fifo.o(i.app_fifo_get)
    app_fifo_init                            0x00019e99   Thumb Code    32  app_fifo.o(i.app_fifo_init)
    app_fifo_put                             0x00019eb9   Thumb Code    26  app_fifo.o(i.app_fifo_put)
    app_timer_create                         0x00019ed5   Thumb Code    32  app_timer.o(i.app_timer_create)
    app_timer_init                           0x00019ef9   Thumb Code    70  app_timer.o(i.app_timer_init)
    app_timer_start                          0x00019f4d   Thumb Code   128  app_timer.o(i.app_timer_start)
    app_timer_stop                           0x00019fd5   Thumb Code    26  app_timer.o(i.app_timer_stop)
    app_uart_get                             0x00019ff5   Thumb Code    42  app_uart_fifo.o(i.app_uart_get)
    app_uart_init                            0x0001a029   Thumb Code   148  app_uart_fifo.o(i.app_uart_init)
    app_util_critical_region_enter           0x0001a0cd   Thumb Code    64  app_util_platform.o(i.app_util_critical_region_enter)
    app_util_critical_region_exit            0x0001a115   Thumb Code    46  app_util_platform.o(i.app_util_critical_region_exit)
    blcm_link_ctx_get                        0x0001a1d1   Thumb Code    72  ble_link_ctx_manager.o(i.blcm_link_ctx_get)
    ble_advdata_encode                       0x0001a219   Thumb Code   386  ble_advdata.o(i.ble_advdata_encode)
    ble_advdata_parse                        0x0001a39b   Thumb Code    32  ble_advdata.o(i.ble_advdata_parse)
    ble_advdata_search                       0x0001a3bb   Thumb Code    56  ble_advdata.o(i.ble_advdata_search)
    ble_advertising_conn_cfg_tag_set         0x0001a3f3   Thumb Code     6  ble_advertising.o(i.ble_advertising_conn_cfg_tag_set)
    ble_advertising_init                     0x0001a3f9   Thumb Code   250  ble_advertising.o(i.ble_advertising_init)
    ble_advertising_on_ble_evt               0x0001a4f3   Thumb Code   106  ble_advertising.o(i.ble_advertising_on_ble_evt)
    ble_advertising_on_sys_evt               0x0001a55d   Thumb Code     2  ble_advertising.o(i.ble_advertising_on_sys_evt)
    ble_advertising_start                    0x0001a55f   Thumb Code   514  ble_advertising.o(i.ble_advertising_start)
    ble_conn_params_init                     0x0001a761   Thumb Code    90  ble_conn_params.o(i.ble_conn_params_init)
    ble_conn_state_conn_idx                  0x0001a7c9   Thumb Code    18  ble_conn_state.o(i.ble_conn_state_conn_idx)
    ble_conn_state_valid                     0x0001a7dd   Thumb Code    16  ble_conn_state.o(i.ble_conn_state_valid)
    ble_nus_data_send                        0x0001ab8d   Thumb Code   102  ble_nus.o(i.ble_nus_data_send)
    ble_nus_init                             0x0001abf5   Thumb Code   206  ble_nus.o(i.ble_nus_init)
    ble_nus_on_ble_evt                       0x0001acc9   Thumb Code   112  ble_nus.o(i.ble_nus_on_ble_evt)
    ble_srv_is_notification_enabled          0x0001ad39   Thumb Code     8  ble_srv_common.o(i.ble_srv_is_notification_enabled)
    bsp_board_button_idx_to_pin              0x0001ad41   Thumb Code     6  boards.o(i.bsp_board_button_idx_to_pin)
    bsp_board_led_invert                     0x0001ad4d   Thumb Code    32  boards.o(i.bsp_board_led_invert)
    bsp_board_led_off                        0x0001ad71   Thumb Code    10  boards.o(i.bsp_board_led_off)
    bsp_board_led_on                         0x0001ad81   Thumb Code    10  boards.o(i.bsp_board_led_on)
    bsp_board_led_state_get                  0x0001ad91   Thumb Code    28  boards.o(i.bsp_board_led_state_get)
    bsp_board_leds_off                       0x0001adb1   Thumb Code    18  boards.o(i.bsp_board_leds_off)
    bsp_board_leds_on                        0x0001adc3   Thumb Code    18  boards.o(i.bsp_board_leds_on)
    bsp_board_pin_to_button_idx              0x0001add5   Thumb Code    30  boards.o(i.bsp_board_pin_to_button_idx)
    bsp_btn_ble_sleep_mode_prepare           0x0001adf9   Thumb Code    30  bsp_btn_ble.o(i.bsp_btn_ble_sleep_mode_prepare)
    bsp_event_to_button_action_assign        0x0001aea9   Thumb Code    64  bsp.o(i.bsp_event_to_button_action_assign)
    bsp_indication_set                       0x0001aeed   Thumb Code    20  bsp.o(i.bsp_indication_set)
    bsp_wakeup_button_enable                 0x0001b0cd   Thumb Code     6  bsp.o(i.bsp_wakeup_button_enable)
    buffer_is_empty                          0x0001b185   Thumb Code    16  nrf_log_frontend.o(i.buffer_is_empty)
    characteristic_add                       0x0001b231   Thumb Code   400  ble_srv_common.o(i.characteristic_add)
    conn_handle_list_get                     0x0001b4b1   Thumb Code    62  ble_conn_state.o(i.conn_handle_list_get)
    free                                     0x0001b669   Thumb Code    76  malloc.o(i.free)
    gatt_evt_handler                         0x0001b6b9   Thumb Code    52  main.o(i.gatt_evt_handler)
    gatt_init                                0x0001b715   Thumb Code    38  main.o(i.gatt_init)
    main                                     0x0001bb49   Thumb Code   482  main.o(i.main)
    malloc                                   0x0001bd9d   Thumb Code    92  malloc.o(i.malloc)
    nrf_atflags_clear                        0x0001bfc3   Thumb Code    22  nrf_atflags.o(i.nrf_atflags_clear)
    nrf_atflags_get                          0x0001bfd9   Thumb Code    22  nrf_atflags.o(i.nrf_atflags_get)
    nrf_atflags_set                          0x0001bfef   Thumb Code    20  nrf_atflags.o(i.nrf_atflags_set)
    nrf_atomic_flag_clear_fetch              0x0001c003   Thumb Code     6  nrf_atomic.o(i.nrf_atomic_flag_clear_fetch)
    nrf_atomic_flag_set                      0x0001c009   Thumb Code     6  nrf_atomic.o(i.nrf_atomic_flag_set)
    nrf_atomic_u32_add                       0x0001c00f   Thumb Code    12  nrf_atomic.o(i.nrf_atomic_u32_add)
    nrf_atomic_u32_and                       0x0001c01b   Thumb Code    12  nrf_atomic.o(i.nrf_atomic_u32_and)
    nrf_atomic_u32_fetch_and                 0x0001c027   Thumb Code    10  nrf_atomic.o(i.nrf_atomic_u32_fetch_and)
    nrf_atomic_u32_fetch_store               0x0001c031   Thumb Code    10  nrf_atomic.o(i.nrf_atomic_u32_fetch_store)
    nrf_atomic_u32_or                        0x0001c03b   Thumb Code    12  nrf_atomic.o(i.nrf_atomic_u32_or)
    nrf_atomic_u32_sub                       0x0001c047   Thumb Code    12  nrf_atomic.o(i.nrf_atomic_u32_sub)
    nrf_balloc_alloc                         0x0001c053   Thumb Code    68  nrf_balloc.o(i.nrf_balloc_alloc)
    nrf_balloc_free                          0x0001c097   Thumb Code    48  nrf_balloc.o(i.nrf_balloc_free)
    nrf_balloc_init                          0x0001c0c7   Thumb Code    48  nrf_balloc.o(i.nrf_balloc_init)
    nrf_ble_gatt_att_mtu_periph_set          0x0001c11b   Thumb Code    24  nrf_ble_gatt.o(i.nrf_ble_gatt_att_mtu_periph_set)
    nrf_ble_gatt_init                        0x0001c133   Thumb Code    34  nrf_ble_gatt.o(i.nrf_ble_gatt_init)
    nrf_ble_gatt_on_ble_evt                  0x0001c155   Thumb Code   180  nrf_ble_gatt.o(i.nrf_ble_gatt_on_ble_evt)
    nrf_ble_qwr_init                         0x0001c249   Thumb Code    36  nrf_ble_qwr.o(i.nrf_ble_qwr_init)
    nrf_ble_qwr_on_ble_evt                   0x0001c26d   Thumb Code   182  nrf_ble_qwr.o(i.nrf_ble_qwr_on_ble_evt)
    nrf_drv_clock_init                       0x0001c361   Thumb Code    48  nrf_drv_clock.o(i.nrf_drv_clock_init)
    nrf_drv_clock_lfclk_release              0x0001c399   Thumb Code    42  nrf_drv_clock.o(i.nrf_drv_clock_lfclk_release)
    nrf_drv_twi_init                         0x0001c3c9   Thumb Code    56  nrf_drv_twi.o(i.nrf_drv_twi_init)
    nrf_drv_uart_init                        0x0001c41d   Thumb Code    56  nrf_drv_uart.o(i.nrf_drv_uart_init)
    nrf_fprintf                              0x0001c469   Thumb Code    26  nrf_fprintf.o(i.nrf_fprintf)
    nrf_fprintf_buffer_flush                 0x0001c483   Thumb Code    24  nrf_fprintf.o(i.nrf_fprintf_buffer_flush)
    nrf_fprintf_fmt                          0x0001c49b   Thumb Code   474  nrf_fprintf_format.o(i.nrf_fprintf_fmt)
    nrf_log_backend_add                      0x0001c7a1   Thumb Code    86  nrf_log_frontend.o(i.nrf_log_backend_add)
    nrf_log_backend_rtt_init                 0x0001c7ff   Thumb Code     4  nrf_log_backend_rtt.o(i.nrf_log_backend_rtt_init)
    nrf_log_backend_serial_put               0x0001c81d   Thumb Code   200  nrf_log_backend_serial.o(i.nrf_log_backend_serial_put)
    nrf_log_color_id_get                     0x0001c8e5   Thumb Code    42  nrf_log_frontend.o(i.nrf_log_color_id_get)
    nrf_log_default_backends_init            0x0001c915   Thumb Code    24  nrf_log_default_backends.o(i.nrf_log_default_backends_init)
    nrf_log_frontend_dequeue                 0x0001c931   Thumb Code   528  nrf_log_frontend.o(i.nrf_log_frontend_dequeue)
    nrf_log_frontend_std_0                   0x0001cb65   Thumb Code     8  nrf_log_frontend.o(i.nrf_log_frontend_std_0)
    nrf_log_frontend_std_1                   0x0001cb6d   Thumb Code    14  nrf_log_frontend.o(i.nrf_log_frontend_std_1)
    nrf_log_frontend_std_2                   0x0001cb7b   Thumb Code    16  nrf_log_frontend.o(i.nrf_log_frontend_std_2)
    nrf_log_hexdump_entry_process            0x0001cb8d   Thumb Code   146  nrf_log_str_formatter.o(i.nrf_log_hexdump_entry_process)
    nrf_log_init                             0x0001cc39   Thumb Code    46  nrf_log_frontend.o(i.nrf_log_init)
    nrf_log_module_cnt_get                   0x0001cc75   Thumb Code    10  nrf_log_frontend.o(i.nrf_log_module_cnt_get)
    nrf_log_module_name_get                  0x0001cc89   Thumb Code    24  nrf_log_frontend.o(i.nrf_log_module_name_get)
    nrf_log_panic                            0x0001cca5   Thumb Code    38  nrf_log_frontend.o(i.nrf_log_panic)
    nrf_log_std_entry_process                0x0001ccd1   Thumb Code   182  nrf_log_str_formatter.o(i.nrf_log_std_entry_process)
    nrf_memobj_alloc                         0x0001cd87   Thumb Code    96  nrf_memobj.o(i.nrf_memobj_alloc)
    nrf_memobj_free                          0x0001cde7   Thumb Code    50  nrf_memobj.o(i.nrf_memobj_free)
    nrf_memobj_get                           0x0001ce19   Thumb Code     8  nrf_memobj.o(i.nrf_memobj_get)
    nrf_memobj_pool_init                     0x0001ce21   Thumb Code     4  nrf_memobj.o(i.nrf_memobj_pool_init)
    nrf_memobj_put                           0x0001ce25   Thumb Code    30  nrf_memobj.o(i.nrf_memobj_put)
    nrf_memobj_read                          0x0001ce43   Thumb Code    16  nrf_memobj.o(i.nrf_memobj_read)
    nrf_memobj_write                         0x0001ce53   Thumb Code    16  nrf_memobj.o(i.nrf_memobj_write)
    nrf_pwr_mgmt_init                        0x0001ce65   Thumb Code    28  nrf_pwr_mgmt.o(i.nrf_pwr_mgmt_init)
    nrf_pwr_mgmt_run                         0x0001ce8d   Thumb Code    20  nrf_pwr_mgmt.o(i.nrf_pwr_mgmt_run)
    nrf_ringbuf_init                         0x0001cea5   Thumb Code    28  nrf_ringbuf.o(i.nrf_ringbuf_init)
    nrf_sdh_ble_app_ram_start_get            0x0001cec1   Thumb Code    16  nrf_sdh_ble.o(i.nrf_sdh_ble_app_ram_start_get)
    nrf_sdh_ble_default_cfg_set              0x0001ced5   Thumb Code   264  nrf_sdh_ble.o(i.nrf_sdh_ble_default_cfg_set)
    nrf_sdh_ble_enable                       0x0001cffd   Thumb Code   116  nrf_sdh_ble.o(i.nrf_sdh_ble_enable)
    nrf_sdh_enable_request                   0x0001d18d   Thumb Code   102  nrf_sdh.o(i.nrf_sdh_enable_request)
    nrf_sdh_evts_poll                        0x0001d201   Thumb Code    32  nrf_sdh.o(i.nrf_sdh_evts_poll)
    nrf_sdh_is_enabled                       0x0001d225   Thumb Code     6  nrf_sdh.o(i.nrf_sdh_is_enabled)
    nrf_section_iter_init                    0x0001d26d   Thumb Code    10  nrf_section_iter.o(i.nrf_section_iter_init)
    nrf_section_iter_next                    0x0001d29b   Thumb Code    32  nrf_section_iter.o(i.nrf_section_iter_next)
    nrf_strerror_find                        0x0001d2bd   Thumb Code    52  nrf_strerror.o(i.nrf_strerror_find)
    nrf_strerror_get                         0x0001d2f5   Thumb Code    14  nrf_strerror.o(i.nrf_strerror_get)
    nrfx_clock_enable                        0x0001d335   Thumb Code    38  nrfx_clock.o(i.nrfx_clock_enable)
    nrfx_clock_init                          0x0001d365   Thumb Code    26  nrfx_clock.o(i.nrfx_clock_init)
    nrfx_clock_lfclk_stop                    0x0001d385   Thumb Code    20  nrfx_clock.o(i.nrfx_clock_lfclk_stop)
    nrfx_prs_acquire                         0x0001d3e1   Thumb Code     4  nrfx_prs.o(i.nrfx_prs_acquire)
    nrfx_twim_enable                         0x0001d3e5   Thumb Code    32  nrfx_twim.o(i.nrfx_twim_enable)
    nrfx_twim_init                           0x0001d409   Thumb Code   218  nrfx_twim.o(i.nrfx_twim_init)
    nrfx_twim_rx                             0x0001d4ed   Thumb Code    44  nrfx_twim.o(i.nrfx_twim_rx)
    nrfx_twim_tx                             0x0001d51d   Thumb Code    54  nrfx_twim.o(i.nrfx_twim_tx)
    nrfx_twim_xfer                           0x0001d555   Thumb Code    34  nrfx_twim.o(i.nrfx_twim_xfer)
    nrfx_uarte_init                          0x0001d57d   Thumb Code   100  nrfx_uarte.o(i.nrfx_uarte_init)
    nrfx_uarte_rx                            0x0001d5e9   Thumb Code   256  nrfx_uarte.o(i.nrfx_uarte_rx)
    nrfx_uarte_tx                            0x0001d6ed   Thumb Code   138  nrfx_uarte.o(i.nrfx_uarte_tx)
    nrfx_uarte_tx_in_progress                0x0001d77d   Thumb Code    22  nrfx_uarte.o(i.nrfx_uarte_tx_in_progress)
    twi_handler                              0x0001e135   Thumb Code   198  main.o(i.twi_handler)
    twi_init                                 0x0001e25d   Thumb Code    40  main.o(i.twi_init)
    uart_event_handle                        0x0001e651   Thumb Code    96  main.o(i.uart_event_handle)
    nrf_log_backend_rtt_api                  0x0001ed6c   Data          12  nrf_log_backend_rtt.o(.constdata)
    m_ram_start                              0x0001ee04   Data           4  nrf_sdh_ble.o(.constdata)
    __ctype_table                            0x0001ee30   Data         129  ctype_o.o(.constdata)
    Region$$Table$$Base                      0x0001f560   Number         0  anon$$obj.o(Region$$Table)
    Region$$Table$$Limit                     0x0001f580   Number         0  anon$$obj.o(Region$$Table)
    log_const_data$$Base                     0x0001f590   Number         0  nrf_ble_gatt.o(log_const_data)
    m_nrf_log_nrf_ble_gatt_logs_data_const   0x0001f590   Data           8  nrf_ble_gatt.o(log_const_data)
    m_nrf_log_ble_nus_logs_data_const        0x0001f598   Data           8  ble_nus.o(log_const_data)
    m_nrf_log_clock_logs_data_const          0x0001f5a0   Data           8  nrf_drv_clock.o(log_const_data)
    m_nrf_log_CLOCK_logs_data_const          0x0001f5a8   Data           8  nrfx_clock.o(log_const_data)
    m_nrf_log_GPIOTE_logs_data_const         0x0001f5b0   Data           8  nrfx_gpiote.o(log_const_data)
    m_nrf_log_PRS_logs_data_const            0x0001f5b8   Data           8  nrfx_prs.o(log_const_data)
    m_nrf_log_UARTE_logs_data_const          0x0001f5c0   Data           8  nrfx_uarte.o(log_const_data)
    m_nrf_log_TWIM_logs_data_const           0x0001f5c8   Data           8  nrfx_twim.o(log_const_data)
    m_nrf_log_pwr_mgmt_logs_data_const       0x0001f5d0   Data           8  nrf_pwr_mgmt.o(log_const_data)
    m_nrf_log_app_logs_data_const            0x0001f5d8   Data           8  nrf_log_frontend.o(log_const_data)
    m_nrf_log_nrf_sdh_logs_data_const        0x0001f5e0   Data           8  nrf_sdh.o(log_const_data)
    m_nrf_log_nrf_sdh_ble_logs_data_const    0x0001f5e8   Data           8  nrf_sdh_ble.o(log_const_data)
    m_nrf_log_nrf_sdh_soc_logs_data_const    0x0001f5f0   Data           8  nrf_sdh_soc.o(log_const_data)
    log_const_data$$Limit                    0x0001f5f8   Number         0  nrf_sdh_soc.o(log_const_data)
    log_mempool                              0x0001f5f8   Data          20  nrf_log_frontend.o(nrf_balloc)
    sdh_ble_observers0$$Base                 0x0001f60c   Number         0  ble_conn_state.o(sdh_ble_observers0)
    sdh_ble_observers0$$Limit                0x0001f614   Number         0  ble_conn_state.o(sdh_ble_observers0)
    sdh_ble_observers1$$Base                 0x0001f614   Number         0  main.o(sdh_ble_observers1)
    sdh_ble_observers1$$Limit                0x0001f634   Number         0  ble_conn_params.o(sdh_ble_observers1)
    sdh_ble_observers2$$Base                 0x0001f634   Number         0  main.o(sdh_ble_observers2)
    sdh_ble_observers2$$Limit                0x0001f644   Number         0  main.o(sdh_ble_observers2)
    sdh_ble_observers3$$Base                 0x0001f644   Number         0  main.o(sdh_ble_observers3)
    sdh_ble_observers3$$Limit                0x0001f64c   Number         0  main.o(sdh_ble_observers3)
    sdh_soc_observers0$$Base                 0x0001f64c   Number         0  nrf_drv_clock.o(sdh_soc_observers0)
    sdh_soc_observers0$$Limit                0x0001f654   Number         0  nrf_drv_clock.o(sdh_soc_observers0)
    sdh_soc_observers1$$Base                 0x0001f654   Number         0  main.o(sdh_soc_observers1)
    sdh_soc_observers1$$Limit                0x0001f65c   Number         0  main.o(sdh_soc_observers1)
    sdh_stack_observers0$$Base               0x0001f65c   Number         0  nrf_sdh_ble.o(sdh_stack_observers0)
    sdh_stack_observers0$$Limit              0x0001f66c   Number         0  nrf_sdh_soc.o(sdh_stack_observers0)
    sdh_state_observers0$$Base               0x0001f66c   Number         0  nrf_drv_clock.o(sdh_state_observers0)
    sdh_state_observers0$$Limit              0x0001f674   Number         0  nrf_drv_clock.o(sdh_state_observers0)
    Image$$RW_IRAM1$$Base                    0x20002500   Number         0  anon$$obj.o ABSOLUTE
    SystemCoreClock                          0x20002608   Data           4  system_nrf52810.o(.data)
    __microlib_freelist                      0x2000260c   Data           4  mvars.o(.data)
    __microlib_freelist_initialised          0x20002610   Data           4  mvars.o(.data)
    nrf_nvic_state                           0x20002d24   Data          12  app_util_platform.o(.bss)
    _SEGGER_RTT                              0x200032f8   Data         120  segger_rtt.o(.bss)
    __heap_base                              0x20003580   Data           0  arm_startup_nrf52810.o(HEAP)
    __heap_limit                             0x20003d80   Data           0  arm_startup_nrf52810.o(HEAP)
    __initial_sp                             0x20004580   Data           0  arm_startup_nrf52810.o(STACK)



==============================================================================

Memory Map of the image

  Image Entry point : 0x00019201

  Load Region LR_IROM1 (Base: 0x00019000, Size: 0x00006788, Max: 0x00017000, ABSOLUTE)

    Execution Region ER_IROM1 (Base: 0x00019000, Size: 0x00006674, Max: 0x00017000, ABSOLUTE)

    Base Addr    Size         Type   Attr      Idx    E Section Name        Object

    0x00019000   0x00000200   Data   RO         4818    RESET               arm_startup_nrf52810.o
    0x00019200   0x00000000   Code   RO         4859  * .ARM.Collect$$$$00000000  mc_w.l(entry.o)
    0x00019200   0x00000004   Code   RO         4942    .ARM.Collect$$$$00000001  mc_w.l(entry2.o)
    0x00019204   0x00000004   Code   RO         4945    .ARM.Collect$$$$00000004  mc_w.l(entry5.o)
    0x00019208   0x00000000   Code   RO         4947    .ARM.Collect$$$$00000008  mc_w.l(entry7b.o)
    0x00019208   0x00000000   Code   RO         4949    .ARM.Collect$$$$0000000A  mc_w.l(entry8b.o)
    0x00019208   0x00000008   Code   RO         4950    .ARM.Collect$$$$0000000B  mc_w.l(entry9a.o)
    0x00019210   0x00000000   Code   RO         4952    .ARM.Collect$$$$0000000D  mc_w.l(entry10a.o)
    0x00019210   0x00000000   Code   RO         4954    .ARM.Collect$$$$0000000F  mc_w.l(entry11a.o)
    0x00019210   0x00000004   Code   RO         4943    .ARM.Collect$$$$00002712  mc_w.l(entry2.o)
    0x00019214   0x000000e2   Code   RO         3408    .emb_text           nrf_atomic.o
    0x000192f6   0x00000002   PAD
    0x000192f8   0x00000024   Code   RO         4819    .text               arm_startup_nrf52810.o
    0x0001931c   0x00000062   Code   RO         4862    .text               mc_w.l(uldiv.o)
    0x0001937e   0x0000001e   Code   RO         4864    .text               mc_w.l(llshl.o)
    0x0001939c   0x00000008   Code   RO         4866    .text               mc_w.l(ctype_o.o)
    0x000193a4   0x00000024   Code   RO         4894    .text               mc_w.l(memcpya.o)
    0x000193c8   0x00000024   Code   RO         4896    .text               mc_w.l(memseta.o)
    0x000193ec   0x0000000e   Code   RO         4898    .text               mc_w.l(strlen.o)
    0x000193fa   0x00000012   Code   RO         4902    .text               mc_w.l(strcpy.o)
    0x0001940c   0x000000b0   Code   RO         4934    .text               mf_w.l(fadd.o)
    0x000194bc   0x00000018   Code   RO         4936    .text               mf_w.l(fscalb.o)
    0x000194d4   0x0000000a   Code   RO         4938    .text               mf_w.l(ffltui.o)
    0x000194de   0x00000028   Code   RO         4940    .text               mf_w.l(ffixui.o)
    0x00019506   0x00000020   Code   RO         4956    .text               mc_w.l(llushr.o)
    0x00019526   0x00000000   Code   RO         4960    .text               mc_w.l(iusefp.o)
    0x00019526   0x0000006e   Code   RO         4961    .text               mf_w.l(fepilogue.o)
    0x00019594   0x00000024   Code   RO         4963    .text               mc_w.l(init.o)
    0x000195b8   0x000000e4   Code   RO            4    i.ENS210_set_mode   main.o
    0x0001969c   0x00000164   Code   RO         1899    i.GPIOTE_IRQHandler  nrfx_gpiote.o
    0x00019800   0x00000016   Code   RO         2913    i.NVIC_ClearPendingIRQ  app_timer.o
    0x00019816   0x00000016   Code   RO         2914    i.NVIC_EnableIRQ    app_timer.o
    0x0001982c   0x00000016   Code   RO         2915    i.NVIC_SetPendingIRQ  app_timer.o
    0x00019842   0x00000020   Code   RO         2916    i.NVIC_SetPriority  app_timer.o
    0x00019862   0x00000002   PAD
    0x00019864   0x00000058   Code   RO         1764    i.POWER_CLOCK_IRQHandler  nrfx_clock.o
    0x000198bc   0x00000024   Code   RO         2917    i.RTC1_IRQHandler   app_timer.o
    0x000198e0   0x00000004   Code   RO         4358    i.SEGGER_RTT_Init   segger_rtt.o
    0x000198e4   0x0000005c   Code   RO         4372    i.SEGGER_RTT_WriteNoLock  segger_rtt.o
    0x00019940   0x00000004   Code   RO         2918    i.SWI0_EGU0_IRQHandler  app_timer.o
    0x00019944   0x00000004   Code   RO         4609    i.SWI2_IRQHandler   nrf_sdh.o
    0x00019948   0x000002ec   Code   RO         4827    i.SystemInit        system_nrf52810.o
    0x00019c34   0x00000010   Code   RO         2416    i.TWIM0_TWIS0_IRQHandler  nrfx_twim.o
    0x00019c44   0x00000010   Code   RO         2234    i.UARTE0_IRQHandler  nrfx_uarte.o
    0x00019c54   0x00000068   Code   RO         4376    i._DoInit           segger_rtt.o
    0x00019cbc   0x00000016   Code   RO         4377    i._GetAvailWriteSpace  segger_rtt.o
    0x00019cd2   0x0000005a   Code   RO         4379    i._WriteBlocking    segger_rtt.o
    0x00019d2c   0x00000042   Code   RO         4380    i._WriteNoCheck     segger_rtt.o
    0x00019d6e   0x0000000e   Code   RO         4967    i.__scatterload_copy  mc_w.l(handlers.o)
    0x00019d7c   0x00000002   Code   RO         4968    i.__scatterload_null  mc_w.l(handlers.o)
    0x00019d7e   0x0000000e   Code   RO         4969    i.__scatterload_zeroinit  mc_w.l(handlers.o)
    0x00019d8c   0x00000024   Code   RO         4610    i.__sd_nvic_app_accessible_irq  nrf_sdh.o
    0x00019db0   0x00000036   Code   RO          773    i.advertising_buttons_configure  bsp_btn_ble.o
    0x00019de6   0x00000002   PAD
    0x00019de8   0x00000084   Code   RO         2746    i.app_error_fault_handler  app_error_weak.o
    0x00019e6c   0x00000016   Code   RO         2686    i.app_error_handler_bare  app_error.o
    0x00019e82   0x00000016   Code   RO         2790    i.app_fifo_get      app_fifo.o
    0x00019e98   0x00000020   Code   RO         2791    i.app_fifo_init     app_fifo.o
    0x00019eb8   0x0000001a   Code   RO         2793    i.app_fifo_put      app_fifo.o
    0x00019ed2   0x00000002   PAD
    0x00019ed4   0x00000024   Code   RO         2921    i.app_timer_create  app_timer.o
    0x00019ef8   0x00000054   Code   RO         2922    i.app_timer_init    app_timer.o
    0x00019f4c   0x00000088   Code   RO         2925    i.app_timer_start   app_timer.o
    0x00019fd4   0x00000020   Code   RO         2926    i.app_timer_stop    app_timer.o
    0x00019ff4   0x00000034   Code   RO         3082    i.app_uart_get      app_uart_fifo.o
    0x0001a028   0x000000a4   Code   RO         3083    i.app_uart_init     app_uart_fifo.o
    0x0001a0cc   0x00000048   Code   RO         3156    i.app_util_critical_region_enter  app_util_platform.o
    0x0001a114   0x00000034   Code   RO         3157    i.app_util_critical_region_exit  app_util_platform.o
    0x0001a148   0x00000088   Code   RO         2235    i.apply_config      nrfx_uarte.o
    0x0001a1d0   0x00000048   Code   RO         1318    i.blcm_link_ctx_get  ble_link_ctx_manager.o
    0x0001a218   0x00000182   Code   RO          883    i.ble_advdata_encode  ble_advdata.o
    0x0001a39a   0x00000020   Code   RO          885    i.ble_advdata_parse  ble_advdata.o
    0x0001a3ba   0x00000038   Code   RO          886    i.ble_advdata_search  ble_advdata.o
    0x0001a3f2   0x00000006   Code   RO          990    i.ble_advertising_conn_cfg_tag_set  ble_advertising.o
    0x0001a3f8   0x000000fa   Code   RO          991    i.ble_advertising_init  ble_advertising.o
    0x0001a4f2   0x0000006a   Code   RO          993    i.ble_advertising_on_ble_evt  ble_advertising.o
    0x0001a55c   0x00000002   Code   RO          994    i.ble_advertising_on_sys_evt  ble_advertising.o
    0x0001a55e   0x00000202   Code   RO          997    i.ble_advertising_start  ble_advertising.o
    0x0001a760   0x00000068   Code   RO         1086    i.ble_conn_params_init  ble_conn_params.o
    0x0001a7c8   0x00000012   Code   RO         1161    i.ble_conn_state_conn_idx  ble_conn_state.o
    0x0001a7da   0x00000002   PAD
    0x0001a7dc   0x00000014   Code   RO         1174    i.ble_conn_state_valid  ble_conn_state.o
    0x0001a7f0   0x00000060   Code   RO          889    i.ble_device_addr_encode  ble_advdata.o
    0x0001a850   0x000000cc   Code   RO            6    i.ble_evt_handler   main.o
    0x0001a91c   0x00000070   Code   RO          774    i.ble_evt_handler   bsp_btn_ble.o
    0x0001a98c   0x000000fc   Code   RO         1088    i.ble_evt_handler   ble_conn_params.o
    0x0001aa88   0x00000104   Code   RO         1175    i.ble_evt_handler   ble_conn_state.o
    0x0001ab8c   0x00000066   Code   RO         1520    i.ble_nus_data_send  ble_nus.o
    0x0001abf2   0x00000002   PAD
    0x0001abf4   0x000000d4   Code   RO         1521    i.ble_nus_init      ble_nus.o
    0x0001acc8   0x00000070   Code   RO         1522    i.ble_nus_on_ble_evt  ble_nus.o
    0x0001ad38   0x00000008   Code   RO         1344    i.ble_srv_is_notification_enabled  ble_srv_common.o
    0x0001ad40   0x0000000c   Code   RO          520    i.bsp_board_button_idx_to_pin  boards.o
    0x0001ad4c   0x00000024   Code   RO          524    i.bsp_board_led_invert  boards.o
    0x0001ad70   0x00000010   Code   RO          525    i.bsp_board_led_off  boards.o
    0x0001ad80   0x00000010   Code   RO          526    i.bsp_board_led_on  boards.o
    0x0001ad90   0x00000020   Code   RO          527    i.bsp_board_led_state_get  boards.o
    0x0001adb0   0x00000012   Code   RO          528    i.bsp_board_leds_off  boards.o
    0x0001adc2   0x00000012   Code   RO          529    i.bsp_board_leds_on  boards.o
    0x0001add4   0x00000024   Code   RO          530    i.bsp_board_pin_to_button_idx  boards.o
    0x0001adf8   0x0000001e   Code   RO          776    i.bsp_btn_ble_sleep_mode_prepare  bsp_btn_ble.o
    0x0001ae16   0x00000002   PAD
    0x0001ae18   0x00000090   Code   RO          657    i.bsp_button_event_handler  bsp.o
    0x0001aea8   0x00000044   Code   RO          661    i.bsp_event_to_button_action_assign  bsp.o
    0x0001aeec   0x00000018   Code   RO          662    i.bsp_indication_set  bsp.o
    0x0001af04   0x000001c8   Code   RO          664    i.bsp_led_indication  bsp.o
    0x0001b0cc   0x00000006   Code   RO          666    i.bsp_wakeup_button_enable  bsp.o
    0x0001b0d2   0x00000002   PAD
    0x0001b0d4   0x00000090   Code   RO         4113    i.buf_prealloc      nrf_log_frontend.o
    0x0001b164   0x0000001e   Code   RO         3620    i.buffer_add        nrf_fprintf_format.o
    0x0001b182   0x00000002   PAD
    0x0001b184   0x00000014   Code   RO         4114    i.buffer_is_empty   nrf_log_frontend.o
    0x0001b198   0x00000088   Code   RO            8    i.buttons_leds_init  main.o
    0x0001b220   0x00000010   Code   RO         1902    i.channel_port_get  nrfx_gpiote.o
    0x0001b230   0x00000190   Code   RO         1346    i.characteristic_add  ble_srv_common.o
    0x0001b3c0   0x00000028   Code   RO         1578    i.clock_clk_started_notify  nrf_drv_clock.o
    0x0001b3e8   0x0000001c   Code   RO         1579    i.clock_irq_handler  nrf_drv_clock.o
    0x0001b404   0x000000ac   Code   RO         2928    i.compare_reg_update  app_timer.o
    0x0001b4b0   0x0000003e   Code   RO         1176    i.conn_handle_list_get  ble_conn_state.o
    0x0001b4ee   0x00000088   Code   RO          890    i.conn_int_encode   ble_advdata.o
    0x0001b576   0x00000004   Code   RO            9    i.conn_params_error_handler  main.o
    0x0001b57a   0x00000002   PAD
    0x0001b57c   0x00000048   Code   RO         1089    i.conn_params_negotiation  ble_conn_params.o
    0x0001b5c4   0x00000014   Code   RO         4115    i.dropped_sat16_get  nrf_log_frontend.o
    0x0001b5d8   0x00000040   Code   RO         2929    i.elapsed_ticks_acquire  app_timer.o
    0x0001b618   0x00000014   Code   RO         2796    i.fifo_get          app_fifo.o
    0x0001b62c   0x00000012   Code   RO         2797    i.fifo_put          app_fifo.o
    0x0001b63e   0x00000028   Code   RO          999    i.flags_set         ble_advertising.o
    0x0001b666   0x00000002   PAD
    0x0001b668   0x00000050   Code   RO         4906    i.free              mc_w.l(malloc.o)
    0x0001b6b8   0x0000005c   Code   RO           10    i.gatt_evt_handler  main.o
    0x0001b714   0x00000030   Code   RO           11    i.gatt_init         main.o
    0x0001b744   0x0000007c   Code   RO           12    i.heart_rate_meas_timeout_handler  main.o
    0x0001b7c0   0x00000014   Code   RO         1090    i.instance_get      ble_conn_params.o
    0x0001b7d4   0x000000a6   Code   RO         3621    i.int_print         nrf_fprintf_format.o
    0x0001b87a   0x00000002   PAD
    0x0001b87c   0x00000080   Code   RO         2236    i.interrupts_enable  nrfx_uarte.o
    0x0001b8fc   0x00000034   Code   RO         4116    i.invalid_packets_omit  nrf_log_frontend.o
    0x0001b930   0x00000044   Code   RO         1091    i.is_conn_params_ok  ble_conn_params.o
    0x0001b974   0x00000030   Code   RO          668    i.leds_off          bsp.o
    0x0001b9a4   0x00000010   Code   RO         1404    i.link_init         nrf_ble_gatt.o
    0x0001b9b4   0x000000f8   Code   RO         2930    i.list_insertions_handler  app_timer.o
    0x0001baac   0x0000009c   Code   RO         4117    i.log_skip          nrf_log_frontend.o
    0x0001bb48   0x00000254   Code   RO           13    i.main              main.o
    0x0001bd9c   0x0000006c   Code   RO         4907    i.malloc            mc_w.l(malloc.o)
    0x0001be08   0x00000064   Code   RO          891    i.manuf_specific_data_encode  ble_advdata.o
    0x0001be6c   0x0000007e   Code   RO         3660    i.memobj_op         nrf_memobj.o
    0x0001beea   0x00000002   PAD
    0x0001beec   0x00000030   Code   RO         4118    i.module_idx_get    nrf_log_frontend.o
    0x0001bf1c   0x000000a6   Code   RO          892    i.name_encode       ble_advdata.o
    0x0001bfc2   0x00000016   Code   RO         3342    i.nrf_atflags_clear  nrf_atflags.o
    0x0001bfd8   0x00000016   Code   RO         3347    i.nrf_atflags_get   nrf_atflags.o
    0x0001bfee   0x00000014   Code   RO         3349    i.nrf_atflags_set   nrf_atflags.o
    0x0001c002   0x00000006   Code   RO         3410    i.nrf_atomic_flag_clear_fetch  nrf_atomic.o
    0x0001c008   0x00000006   Code   RO         3411    i.nrf_atomic_flag_set  nrf_atomic.o
    0x0001c00e   0x0000000c   Code   RO         3413    i.nrf_atomic_u32_add  nrf_atomic.o
    0x0001c01a   0x0000000c   Code   RO         3414    i.nrf_atomic_u32_and  nrf_atomic.o
    0x0001c026   0x0000000a   Code   RO         3417    i.nrf_atomic_u32_fetch_and  nrf_atomic.o
    0x0001c030   0x0000000a   Code   RO         3419    i.nrf_atomic_u32_fetch_store  nrf_atomic.o
    0x0001c03a   0x0000000c   Code   RO         3423    i.nrf_atomic_u32_or  nrf_atomic.o
    0x0001c046   0x0000000c   Code   RO         3425    i.nrf_atomic_u32_sub  nrf_atomic.o
    0x0001c052   0x00000044   Code   RO         3544    i.nrf_balloc_alloc  nrf_balloc.o
    0x0001c096   0x00000030   Code   RO         3545    i.nrf_balloc_free   nrf_balloc.o
    0x0001c0c6   0x00000030   Code   RO         3546    i.nrf_balloc_init   nrf_balloc.o
    0x0001c0f6   0x00000010   Code   RO         1903    i.nrf_bitmask_bit_is_set  nrfx_gpiote.o
    0x0001c106   0x00000014   Code   RO         1904    i.nrf_bitmask_bit_set  nrfx_gpiote.o
    0x0001c11a   0x00000018   Code   RO         1406    i.nrf_ble_gatt_att_mtu_periph_set  nrf_ble_gatt.o
    0x0001c132   0x00000022   Code   RO         1408    i.nrf_ble_gatt_init  nrf_ble_gatt.o
    0x0001c154   0x000000f4   Code   RO         1409    i.nrf_ble_gatt_on_ble_evt  nrf_ble_gatt.o
    0x0001c248   0x00000024   Code   RO         1480    i.nrf_ble_qwr_init  nrf_ble_qwr.o
    0x0001c26c   0x000000b6   Code   RO         1481    i.nrf_ble_qwr_on_ble_evt  nrf_ble_qwr.o
    0x0001c322   0x0000000e   Code   RO         1765    i.nrf_clock_event_check  nrfx_clock.o
    0x0001c330   0x00000010   Code   RO         1766    i.nrf_clock_event_clear  nrfx_clock.o
    0x0001c340   0x00000020   Code   RO           14    i.nrf_delay_ms      main.o
    0x0001c360   0x00000038   Code   RO         1586    i.nrf_drv_clock_init  nrf_drv_clock.o
    0x0001c398   0x00000030   Code   RO         1590    i.nrf_drv_clock_lfclk_release  nrf_drv_clock.o
    0x0001c3c8   0x00000040   Code   RO         2556    i.nrf_drv_twi_init  nrf_drv_twi.o
    0x0001c408   0x00000006   Code   RO           15    i.nrf_drv_twi_rx    main.o
    0x0001c40e   0x0000000e   Code   RO           16    i.nrf_drv_twi_tx    main.o
    0x0001c41c   0x00000040   Code   RO         1724    i.nrf_drv_uart_init  nrf_drv_uart.o
    0x0001c45c   0x00000006   Code   RO         3085    i.nrf_drv_uart_rx   app_uart_fifo.o
    0x0001c462   0x00000006   Code   RO         3086    i.nrf_drv_uart_tx   app_uart_fifo.o
    0x0001c468   0x0000001a   Code   RO         3581    i.nrf_fprintf       nrf_fprintf.o
    0x0001c482   0x00000018   Code   RO         3582    i.nrf_fprintf_buffer_flush  nrf_fprintf.o
    0x0001c49a   0x000001da   Code   RO         3622    i.nrf_fprintf_fmt   nrf_fprintf_format.o
    0x0001c674   0x00000024   Code   RO         2237    i.nrf_gpio_cfg      nrfx_uarte.o
    0x0001c698   0x00000024   Code   RO         2417    i.nrf_gpio_cfg      nrfx_twim.o
    0x0001c6bc   0x00000012   Code   RO         2239    i.nrf_gpio_cfg_input  nrfx_uarte.o
    0x0001c6ce   0x00000010   Code   RO           17    i.nrf_gpio_cfg_output  main.o
    0x0001c6de   0x00000014   Code   RO         2240    i.nrf_gpio_cfg_output  nrfx_uarte.o
    0x0001c6f2   0x00000022   Code   RO         1907    i.nrf_gpio_cfg_sense_set  nrfx_gpiote.o
    0x0001c714   0x0000000e   Code   RO           18    i.nrf_gpio_pin_clear  main.o
    0x0001c722   0x0000000e   Code   RO           19    i.nrf_gpio_pin_set  main.o
    0x0001c730   0x0000000e   Code   RO         2557    i.nrf_gpio_pin_set  nrf_drv_twi.o
    0x0001c73e   0x00000016   Code   RO          533    i.nrf_gpio_pin_write  boards.o
    0x0001c754   0x00000028   Code   RO         1908    i.nrf_gpio_ports_read  nrfx_gpiote.o
    0x0001c77c   0x00000014   Code   RO         1909    i.nrf_gpiote_event_clear  nrfx_gpiote.o
    0x0001c790   0x00000010   Code   RO         1910    i.nrf_gpiote_event_is_set  nrfx_gpiote.o
    0x0001c7a0   0x0000005c   Code   RO         4119    i.nrf_log_backend_add  nrf_log_frontend.o
    0x0001c7fc   0x00000002   Code   RO         3977    i.nrf_log_backend_rtt_flush  nrf_log_backend_rtt.o
    0x0001c7fe   0x00000004   Code   RO         3978    i.nrf_log_backend_rtt_init  nrf_log_backend_rtt.o
    0x0001c802   0x00000002   Code   RO         3979    i.nrf_log_backend_rtt_panic_set  nrf_log_backend_rtt.o
    0x0001c804   0x00000018   Code   RO         3980    i.nrf_log_backend_rtt_put  nrf_log_backend_rtt.o
    0x0001c81c   0x000000c8   Code   RO         4043    i.nrf_log_backend_serial_put  nrf_log_backend_serial.o
    0x0001c8e4   0x00000030   Code   RO         4121    i.nrf_log_color_id_get  nrf_log_frontend.o
    0x0001c914   0x0000001c   Code   RO         4077    i.nrf_log_default_backends_init  nrf_log_default_backends.o
    0x0001c930   0x00000234   Code   RO         4122    i.nrf_log_frontend_dequeue  nrf_log_frontend.o
    0x0001cb64   0x00000008   Code   RO         4124    i.nrf_log_frontend_std_0  nrf_log_frontend.o
    0x0001cb6c   0x0000000e   Code   RO         4125    i.nrf_log_frontend_std_1  nrf_log_frontend.o
    0x0001cb7a   0x00000010   Code   RO         4126    i.nrf_log_frontend_std_2  nrf_log_frontend.o
    0x0001cb8a   0x00000002   PAD
    0x0001cb8c   0x000000ac   Code   RO         4299    i.nrf_log_hexdump_entry_process  nrf_log_str_formatter.o
    0x0001cc38   0x0000003c   Code   RO         4131    i.nrf_log_init      nrf_log_frontend.o
    0x0001cc74   0x00000014   Code   RO         4132    i.nrf_log_module_cnt_get  nrf_log_frontend.o
    0x0001cc88   0x0000001c   Code   RO         4135    i.nrf_log_module_name_get  nrf_log_frontend.o
    0x0001cca4   0x0000002c   Code   RO         4136    i.nrf_log_panic     nrf_log_frontend.o
    0x0001ccd0   0x000000b6   Code   RO         4300    i.nrf_log_std_entry_process  nrf_log_str_formatter.o
    0x0001cd86   0x00000060   Code   RO         3661    i.nrf_memobj_alloc  nrf_memobj.o
    0x0001cde6   0x00000032   Code   RO         3662    i.nrf_memobj_free   nrf_memobj.o
    0x0001ce18   0x00000008   Code   RO         3663    i.nrf_memobj_get    nrf_memobj.o
    0x0001ce20   0x00000004   Code   RO         3664    i.nrf_memobj_pool_init  nrf_memobj.o
    0x0001ce24   0x0000001e   Code   RO         3665    i.nrf_memobj_put    nrf_memobj.o
    0x0001ce42   0x00000010   Code   RO         3666    i.nrf_memobj_read   nrf_memobj.o
    0x0001ce52   0x00000010   Code   RO         3667    i.nrf_memobj_write  nrf_memobj.o
    0x0001ce62   0x00000002   PAD
    0x0001ce64   0x00000028   Code   RO         3739    i.nrf_pwr_mgmt_init  nrf_pwr_mgmt.o
    0x0001ce8c   0x00000014   Code   RO         3740    i.nrf_pwr_mgmt_run  nrf_pwr_mgmt.o
    0x0001cea0   0x00000004   Code   RO           20    i.nrf_qwr_error_handler  main.o
    0x0001cea4   0x0000001c   Code   RO         3813    i.nrf_ringbuf_init  nrf_ringbuf.o
    0x0001cec0   0x00000014   Code   RO         4730    i.nrf_sdh_ble_app_ram_start_get  nrf_sdh_ble.o
    0x0001ced4   0x00000128   Code   RO         4731    i.nrf_sdh_ble_default_cfg_set  nrf_sdh_ble.o
    0x0001cffc   0x00000130   Code   RO         4732    i.nrf_sdh_ble_enable  nrf_sdh_ble.o
    0x0001d12c   0x00000060   Code   RO         4733    i.nrf_sdh_ble_evts_poll  nrf_sdh_ble.o
    0x0001d18c   0x00000074   Code   RO         4612    i.nrf_sdh_enable_request  nrf_sdh.o
    0x0001d200   0x00000024   Code   RO         4613    i.nrf_sdh_evts_poll  nrf_sdh.o
    0x0001d224   0x0000000c   Code   RO         4614    i.nrf_sdh_is_enabled  nrf_sdh.o
    0x0001d230   0x0000003c   Code   RO         4784    i.nrf_sdh_soc_evts_poll  nrf_sdh_soc.o
    0x0001d26c   0x0000000a   Code   RO         3871    i.nrf_section_iter_init  nrf_section_iter.o
    0x0001d276   0x00000024   Code   RO         3872    i.nrf_section_iter_item_set  nrf_section_iter.o
    0x0001d29a   0x00000020   Code   RO         3873    i.nrf_section_iter_next  nrf_section_iter.o
    0x0001d2ba   0x00000002   PAD
    0x0001d2bc   0x00000038   Code   RO         3906    i.nrf_strerror_find  nrf_strerror.o
    0x0001d2f4   0x00000014   Code   RO         3907    i.nrf_strerror_get  nrf_strerror.o
    0x0001d308   0x0000000a   Code   RO         2419    i.nrf_twim_event_check  nrfx_twim.o
    0x0001d312   0x0000000c   Code   RO         2420    i.nrf_twim_event_clear  nrfx_twim.o
    0x0001d31e   0x0000000a   Code   RO         2241    i.nrf_uarte_event_check  nrfx_uarte.o
    0x0001d328   0x0000000c   Code   RO         2242    i.nrf_uarte_event_clear  nrfx_uarte.o
    0x0001d334   0x00000030   Code   RO         1771    i.nrfx_clock_enable  nrfx_clock.o
    0x0001d364   0x00000020   Code   RO         1774    i.nrfx_clock_init   nrfx_clock.o
    0x0001d384   0x0000001c   Code   RO         1777    i.nrfx_clock_lfclk_stop  nrfx_clock.o
    0x0001d3a0   0x00000010   Code   RO         2558    i.nrfx_coredep_delay_us  nrf_drv_twi.o
    0x0001d3b0   0x00000010   Code   RO         2931    i.nrfx_coredep_delay_us  app_timer.o
    0x0001d3c0   0x00000010   Code   RO         2243    i.nrfx_is_in_ram    nrfx_uarte.o
    0x0001d3d0   0x00000010   Code   RO         2421    i.nrfx_is_in_ram    nrfx_twim.o
    0x0001d3e0   0x00000004   Code   RO         2192    i.nrfx_prs_acquire  nrfx_prs.o
    0x0001d3e4   0x00000024   Code   RO         2423    i.nrfx_twim_enable  nrfx_twim.o
    0x0001d408   0x000000e4   Code   RO         2424    i.nrfx_twim_init    nrfx_twim.o
    0x0001d4ec   0x00000030   Code   RO         2426    i.nrfx_twim_rx      nrfx_twim.o
    0x0001d51c   0x00000036   Code   RO         2429    i.nrfx_twim_tx      nrfx_twim.o
    0x0001d552   0x00000002   PAD
    0x0001d554   0x00000028   Code   RO         2431    i.nrfx_twim_xfer    nrfx_twim.o
    0x0001d57c   0x0000006c   Code   RO         2245    i.nrfx_uarte_init   nrfx_uarte.o
    0x0001d5e8   0x00000104   Code   RO         2246    i.nrfx_uarte_rx     nrfx_uarte.o
    0x0001d6ec   0x00000090   Code   RO         2249    i.nrfx_uarte_tx     nrfx_uarte.o
    0x0001d77c   0x0000001c   Code   RO         2251    i.nrfx_uarte_tx_in_progress  nrfx_uarte.o
    0x0001d798   0x00000034   Code   RO           21    i.nus_data_handler  main.o
    0x0001d7cc   0x00000024   Code   RO           22    i.on_adv_evt        main.o
    0x0001d7f0   0x0000001c   Code   RO           23    i.on_conn_params_evt  main.o
    0x0001d80c   0x0000006a   Code   RO         1523    i.on_connect        ble_nus.o
    0x0001d876   0x00000002   PAD
    0x0001d878   0x0000008c   Code   RO         1410    i.on_connected_evt  nrf_ble_gatt.o
    0x0001d904   0x000000b0   Code   RO         1411    i.on_exchange_mtu_request_evt  nrf_ble_gatt.o
    0x0001d9b4   0x00000084   Code   RO         1524    i.on_write          ble_nus.o
    0x0001da38   0x00000012   Code   RO         1000    i.phy_is_valid      ble_advertising.o
    0x0001da4a   0x00000002   PAD
    0x0001da4c   0x0000003c   Code   RO         4302    i.postfix_process   nrf_log_str_formatter.o
    0x0001da88   0x00000098   Code   RO         4303    i.prefix_process    nrf_log_str_formatter.o
    0x0001db20   0x00000054   Code   RO           24    i.read_ENS210_sensor_data  main.o
    0x0001db74   0x0000003c   Code   RO         2932    i.rtc1_stop         app_timer.o
    0x0001dbb0   0x00000018   Code   RO         2253    i.rx_done_event     nrfx_uarte.o
    0x0001dbc8   0x00000050   Code   RO         1593    i.sd_state_evt_handler  nrf_drv_clock.o
    0x0001dc18   0x00000030   Code   RO         4619    i.sdh_request_observer_notify  nrf_sdh.o
    0x0001dc48   0x0000002c   Code   RO         4620    i.sdh_state_observer_notify  nrf_sdh.o
    0x0001dc74   0x00000010   Code   RO         1092    i.send_error_evt    ble_conn_params.o
    0x0001dc84   0x00000050   Code   RO         3981    i.serial_tx         nrf_log_backend_rtt.o
    0x0001dcd4   0x00000088   Code   RO          893    i.service_data_encode  ble_advdata.o
    0x0001dd5c   0x00000030   Code   RO         1348    i.set_security_req  ble_srv_common.o
    0x0001dd8c   0x00000028   Code   RO           25    i.sleep_mode_enter  main.o
    0x0001ddb4   0x00000018   Code   RO         1594    i.soc_evt_handler   nrf_drv_clock.o
    0x0001ddcc   0x00000058   Code   RO         4622    i.softdevices_evt_irq_enable  nrf_sdh.o
    0x0001de24   0x0000008c   Code   RO         4138    i.std_n             nrf_log_frontend.o
    0x0001deb0   0x00000080   Code   RO         2933    i.timer_list_handler  app_timer.o
    0x0001df30   0x0000003c   Code   RO         2934    i.timer_list_insert  app_timer.o
    0x0001df6c   0x00000060   Code   RO         2935    i.timer_list_remove  app_timer.o
    0x0001dfcc   0x00000048   Code   RO         2936    i.timer_stop_op_schedule  app_timer.o
    0x0001e014   0x00000074   Code   RO         2937    i.timer_timeouts_check  app_timer.o
    0x0001e088   0x000000aa   Code   RO         2559    i.twi_clear_bus     nrf_drv_twi.o
    0x0001e132   0x00000002   PAD
    0x0001e134   0x00000128   Code   RO           26    i.twi_handler       main.o
    0x0001e25c   0x00000030   Code   RO           27    i.twi_init          main.o
    0x0001e28c   0x00000040   Code   RO         2560    i.twim_evt_handler  nrf_drv_twi.o
    0x0001e2cc   0x0000014c   Code   RO         2432    i.twim_irq_handler  nrfx_twim.o
    0x0001e418   0x00000238   Code   RO         2433    i.twim_xfer         nrfx_twim.o
    0x0001e650   0x00000068   Code   RO           28    i.uart_event_handle  main.o
    0x0001e6b8   0x000000a0   Code   RO         3087    i.uart_event_handler  app_uart_fifo.o
    0x0001e758   0x00000030   Code   RO         1725    i.uarte_evt_handler  nrf_drv_uart.o
    0x0001e788   0x000000f4   Code   RO         2254    i.uarte_irq_handler  nrfx_uarte.o
    0x0001e87c   0x0000000a   Code   RO          894    i.uint16_encode     ble_advdata.o
    0x0001e886   0x00000002   PAD
    0x0001e888   0x000000b4   Code   RO         3623    i.unsigned_print    nrf_fprintf_format.o
    0x0001e93c   0x00000068   Code   RO         1093    i.update_timeout_handler  ble_conn_params.o
    0x0001e9a4   0x00000018   Code   RO         1001    i.use_whitelist     ble_advertising.o
    0x0001e9bc   0x00000024   Code   RO         1482    i.user_mem_reply    nrf_ble_qwr.o
    0x0001e9e0   0x00000030   Code   RO         2938    i.user_op_alloc     app_timer.o
    0x0001ea10   0x00000030   Code   RO          895    i.uuid_list_encode  ble_advdata.o
    0x0001ea40   0x0000009e   Code   RO          896    i.uuid_list_sized_encode  ble_advdata.o
    0x0001eade   0x0000003a   Code   RO          670    i.wakeup_button_cfg  bsp.o
    0x0001eb18   0x00000044   Data   RO           31    .constdata          main.o
    0x0001eb5c   0x00000008   Data   RO          534    .constdata          boards.o
    0x0001eb64   0x0000002c   Data   RO          675    .constdata          bsp.o
    0x0001eb90   0x0000000e   Data   RO         1412    .constdata          nrf_ble_gatt.o
    0x0001eb9e   0x00000002   PAD
    0x0001eba0   0x00000010   Data   RO         1525    .constdata          ble_nus.o
    0x0001ebb0   0x00000004   Data   RO         1939    .constdata          nrfx_gpiote.o
    0x0001ebb4   0x00000004   Data   RO         2257    .constdata          nrfx_uarte.o
    0x0001ebb8   0x00000018   Data   RO         2436    .constdata          nrfx_twim.o
    0x0001ebd0   0x00000006   Data   RO         2561    .constdata          nrf_drv_twi.o
    0x0001ebd6   0x00000006   Data   RO         2940    .constdata          app_timer.o
    0x0001ebdc   0x00000020   Data   RO         3089    .constdata          app_uart_fifo.o
    0x0001ebfc   0x00000010   Data   RO         3624    .constdata          nrf_fprintf_format.o
    0x0001ec0c   0x00000018   Data   RO         3744    .constdata          nrf_pwr_mgmt.o
    0x0001ec24   0x0000000c   Data   RO         3745    .constdata          nrf_pwr_mgmt.o
    0x0001ec30   0x0000013c   Data   RO         3908    .constdata          nrf_strerror.o
    0x0001ed6c   0x0000000c   Data   RO         3983    .constdata          nrf_log_backend_rtt.o
    0x0001ed78   0x00000006   Data   RO         3984    .constdata          nrf_log_backend_rtt.o
    0x0001ed7e   0x00000002   PAD
    0x0001ed80   0x0000000c   Data   RO         4143    .constdata          nrf_log_frontend.o
    0x0001ed8c   0x00000010   Data   RO         4623    .constdata          nrf_sdh.o
    0x0001ed9c   0x00000028   Data   RO         4624    .constdata          nrf_sdh.o
    0x0001edc4   0x00000010   Data   RO         4625    .constdata          nrf_sdh.o
    0x0001edd4   0x00000010   Data   RO         4626    .constdata          nrf_sdh.o
    0x0001ede4   0x00000020   Data   RO         4734    .constdata          nrf_sdh_ble.o
    0x0001ee04   0x00000010   Data   RO         4735    .constdata          nrf_sdh_ble.o
    0x0001ee14   0x00000010   Data   RO         4785    .constdata          nrf_sdh_soc.o
    0x0001ee24   0x0000000c   Data   RO         4786    .constdata          nrf_sdh_soc.o
    0x0001ee30   0x00000081   Data   RO         4867    .constdata          mc_w.l(ctype_o.o)
    0x0001eeb1   0x00000003   PAD
    0x0001eeb4   0x00000004   Data   RO         4868    .constdata          mc_w.l(ctype_o.o)
    0x0001eeb8   0x000003eb   Data   RO         3909    .conststring        nrf_strerror.o
    0x0001f2a3   0x00000001   PAD
    0x0001f2a4   0x00000066   Data   RO         4304    .conststring        nrf_log_str_formatter.o
    0x0001f30a   0x00000002   PAD
    0x0001f30c   0x000001cf   Data   RO         4736    .conststring        nrf_sdh_ble.o
    0x0001f4db   0x00000001   PAD
    0x0001f4dc   0x0000000d   Data   RO         1413    .conststrlit        nrf_ble_gatt.o
    0x0001f4e9   0x00000003   PAD
    0x0001f4ec   0x00000008   Data   RO         1526    .conststrlit        ble_nus.o
    0x0001f4f4   0x00000006   Data   RO         1600    .conststrlit        nrf_drv_clock.o
    0x0001f4fa   0x00000002   PAD
    0x0001f4fc   0x00000006   Data   RO         1781    .conststrlit        nrfx_clock.o
    0x0001f502   0x00000002   PAD
    0x0001f504   0x00000007   Data   RO         1943    .conststrlit        nrfx_gpiote.o
    0x0001f50b   0x00000001   PAD
    0x0001f50c   0x00000004   Data   RO         2195    .conststrlit        nrfx_prs.o
    0x0001f510   0x00000006   Data   RO         2260    .conststrlit        nrfx_uarte.o
    0x0001f516   0x00000002   PAD
    0x0001f518   0x00000005   Data   RO         2439    .conststrlit        nrfx_twim.o
    0x0001f51d   0x00000003   PAD
    0x0001f520   0x00000009   Data   RO         3746    .conststrlit        nrf_pwr_mgmt.o
    0x0001f529   0x00000003   PAD
    0x0001f52c   0x00000010   Data   RO         4078    .conststrlit        nrf_log_default_backends.o
    0x0001f53c   0x00000004   Data   RO         4144    .conststrlit        nrf_log_frontend.o
    0x0001f540   0x00000008   Data   RO         4627    .conststrlit        nrf_sdh.o
    0x0001f548   0x0000000c   Data   RO         4737    .conststrlit        nrf_sdh_ble.o
    0x0001f554   0x0000000c   Data   RO         4787    .conststrlit        nrf_sdh_soc.o
    0x0001f560   0x00000020   Data   RO         4965    Region$$Table       anon$$obj.o
    0x0001f580   0x00000010   Data   RO         4080    log_backends        nrf_log_default_backends.o
    0x0001f590   0x00000008   Data   RO         1414    log_const_data      nrf_ble_gatt.o
    0x0001f598   0x00000008   Data   RO         1527    log_const_data      ble_nus.o
    0x0001f5a0   0x00000008   Data   RO         1601    log_const_data      nrf_drv_clock.o
    0x0001f5a8   0x00000008   Data   RO         1783    log_const_data      nrfx_clock.o
    0x0001f5b0   0x00000008   Data   RO         1944    log_const_data      nrfx_gpiote.o
    0x0001f5b8   0x00000008   Data   RO         2196    log_const_data      nrfx_prs.o
    0x0001f5c0   0x00000008   Data   RO         2261    log_const_data      nrfx_uarte.o
    0x0001f5c8   0x00000008   Data   RO         2440    log_const_data      nrfx_twim.o
    0x0001f5d0   0x00000008   Data   RO         3748    log_const_data      nrf_pwr_mgmt.o
    0x0001f5d8   0x00000008   Data   RO         4147    log_const_data      nrf_log_frontend.o
    0x0001f5e0   0x00000008   Data   RO         4629    log_const_data      nrf_sdh.o
    0x0001f5e8   0x00000008   Data   RO         4739    log_const_data      nrf_sdh_ble.o
    0x0001f5f0   0x00000008   Data   RO         4788    log_const_data      nrf_sdh_soc.o
    0x0001f5f8   0x00000014   Data   RO         4148    nrf_balloc          nrf_log_frontend.o
    0x0001f60c   0x00000008   Data   RO         1180    sdh_ble_observers0  ble_conn_state.o
    0x0001f614   0x00000010   Data   RO           49    sdh_ble_observers1  main.o
    0x0001f624   0x00000008   Data   RO          778    sdh_ble_observers1  bsp_btn_ble.o
    0x0001f62c   0x00000008   Data   RO         1096    sdh_ble_observers1  ble_conn_params.o
    0x0001f634   0x00000010   Data   RO           50    sdh_ble_observers2  main.o
    0x0001f644   0x00000008   Data   RO           51    sdh_ble_observers3  main.o
    0x0001f64c   0x00000008   Data   RO         1602    sdh_soc_observers0  nrf_drv_clock.o
    0x0001f654   0x00000008   Data   RO           52    sdh_soc_observers1  main.o
    0x0001f65c   0x00000008   Data   RO         4740    sdh_stack_observers0  nrf_sdh_ble.o
    0x0001f664   0x00000008   Data   RO         4789    sdh_stack_observers0  nrf_sdh_soc.o
    0x0001f66c   0x00000008   Data   RO         1603    sdh_state_observers0  nrf_drv_clock.o


    Execution Region RW_IRAM1 (Base: 0x20002500, Size: 0x00002080, Max: 0x00003b00, ABSOLUTE)

    Base Addr    Size         Type   Attr      Idx    E Section Name        Object

    0x20002500   0x00000008   Data   RW           46    .data               main.o
    0x20002508   0x00000034   Data   RW           47    .data               main.o
    0x2000253c   0x00000004   Data   RW           48    .data               main.o
    0x20002540   0x00000010   Data   RW          676    .data               bsp.o
    0x20002550   0x00000008   Data   RW          777    .data               bsp_btn_ble.o
    0x20002558   0x00000008   Data   RW         1095    .data               ble_conn_params.o
    0x20002560   0x00000008   Data   RW         1726    .data               nrf_drv_uart.o
    0x20002568   0x00000008   Data   RW         1782    .data               nrfx_clock.o
    0x20002570   0x00000008   Data   RW         2562    .data               nrf_drv_twi.o
    0x20002578   0x00000014   Data   RW         2941    .data               app_timer.o
    0x2000258c   0x00000014   Data   RW         3090    .data               app_uart_fifo.o
    0x200025a0   0x00000008   Data   RW         3747    .data               nrf_pwr_mgmt.o
    0x200025a8   0x00000001   Data   RW         3985    .data               nrf_log_backend_rtt.o
    0x200025a9   0x00000003   PAD
    0x200025ac   0x00000008   Data   RW         4079    .data               nrf_log_default_backends.o
    0x200025b4   0x00000008   Data   RW         4145    .data               nrf_log_frontend.o
    0x200025bc   0x00000008   Data   RW         4146    .data               nrf_log_frontend.o
    0x200025c4   0x00000040   Data   RW         4305    .data               nrf_log_str_formatter.o
    0x20002604   0x00000003   Data   RW         4628    .data               nrf_sdh.o
    0x20002607   0x00000001   Data   RW         4738    .data               nrf_sdh_ble.o
    0x20002608   0x00000004   Data   RW         4828    .data               system_nrf52810.o
    0x2000260c   0x00000004   Data   RW         4958    .data               mc_w.l(mvars.o)
    0x20002610   0x00000004   Data   RW         4959    .data               mc_w.l(mvars.o)
    0x20002614   0x00000020   Zero   RW           29    .bss                main.o
    0x20002634   0x000003c8   Zero   RW           30    .bss                main.o
    0x200029fc   0x00000020   Zero   RW          671    .bss                bsp.o
    0x20002a1c   0x00000020   Zero   RW          672    .bss                bsp.o
    0x20002a3c   0x0000000c   Zero   RW          673    .bss                bsp.o
    0x20002a48   0x00000020   Zero   RW          674    .bss                bsp.o
    0x20002a68   0x00000050   Zero   RW         1094    .bss                ble_conn_params.o
    0x20002ab8   0x00000078   Zero   RW         1179    .bss                ble_conn_state.o
    0x20002b30   0x00000014   Zero   RW         1595    .bss                nrf_drv_clock.o
    0x20002b44   0x0000005c   Zero   RW         1938    .bss                nrfx_gpiote.o
    0x20002ba0   0x00000024   Zero   RW         2255    .bss                nrfx_uarte.o
    0x20002bc4   0x00000034   Zero   RW         2434    .bss                nrfx_twim.o
    0x20002bf8   0x0000010c   Zero   RW         2939    .bss                app_timer.o
    0x20002d04   0x00000020   Zero   RW         3088    .bss                app_uart_fifo.o
    0x20002d24   0x0000000c   Zero   RW         3162    .bss                app_util_platform.o
    0x20002d30   0x0000000c   Zero   RW         3743    .bss                nrf_pwr_mgmt.o
    0x20002d3c   0x00000040   Zero   RW         3982    .bss                nrf_log_backend_rtt.o
    0x20002d7c   0x000000c0   Zero   RW         4139    .bss                nrf_log_frontend.o
    0x20002e3c   0x00000080   Zero   RW         4140    .bss                nrf_log_frontend.o
    0x20002ebc   0x00000018   Zero   RW         4141    .bss                nrf_log_frontend.o
    0x20002ed4   0x00000424   Zero   RW         4142    .bss                nrf_log_frontend.o
    0x200032f8   0x00000288   Zero   RW         4381    .bss                segger_rtt.o
    0x20003580   0x00000800   Zero   RW         4817    HEAP                arm_startup_nrf52810.o
    0x20003d80   0x00000800   Zero   RW         4816    STACK               arm_startup_nrf52810.o


==============================================================================

Image component sizes


      Code (inc. data)   RO Data    RW Data    ZI Data      Debug   Object Name

        22          0          0          0          0       2421   app_error.o
       132         46          0          0          0      28101   app_error_weak.o
       118          0          0          0          0       4822   app_fifo.o
      1506        118          6         20        268      44603   app_timer.o
       388         34         32         20         32      16487   app_uart_fifo.o
       124         14          0          0         12       9494   app_util_platform.o
        36          8        512          0       4096        896   arm_startup_nrf52810.o
      1324          0          0          0          0      52436   ble_advdata.o
       960          6          0          0          0       9688   ble_advertising.o
       636         44          8          8         80       8983   ble_conn_params.o
       360         10          8          0        120       6759   ble_conn_state.o
        72          0          0          0          0       1620   ble_link_ctx_manager.o
       664          6         32          0          0       6768   ble_nus.o
       456          6          0          0          0       3259   ble_srv_common.o
       206         32          8          0          0      36621   boards.o
       804         60         44         16        108      11924   bsp.o
       196          6          8          8          0       3841   bsp_btn_ble.o
      2220        388        116         64       1000     185511   main.o
        64          0          0          0          0       2852   nrf_atflags.o
       306          0          0          0          0       7679   nrf_atomic.o
       164          0          0          0          0       3520   nrf_balloc.o
       634        186         35          0          0       8225   nrf_ble_gatt.o
       254          0          0          0          0       3784   nrf_ble_qwr.o
       276         34         30          0         20      35064   nrf_drv_clock.o
       328         16          6          8          0      20263   nrf_drv_twi.o
       112         14          0          8          0      13468   nrf_drv_uart.o
        50          0          0          0          0       3465   nrf_fprintf.o
       850          4         16          0          0       5326   nrf_fprintf_format.o
       112         18         18          1         64       5441   nrf_log_backend_rtt.o
       200          0          0          0          0      10837   nrf_log_backend_serial.o
        28          4         32          8          0       3305   nrf_log_default_backends.o
      1474        114         44         16       1404      29062   nrf_log_frontend.o
       566        108        102         64          0       5484   nrf_log_str_formatter.o
       346          0          0          0          0       9259   nrf_memobj.o
        60         12         53          8         12       4915   nrf_pwr_mgmt.o
        28          0          0          0          0       2339   nrf_ringbuf.o
       384         46        104          3          0      36486   nrf_sdh.o
       716        232        539          1          0       5777   nrf_sdh_ble.o
        60          4         56          0          0       2444   nrf_sdh_soc.o
        78          0          0          0          0       2672   nrf_section_iter.o
        76         10       1319          0          0       2679   nrf_strerror.o
       226         30         14          8          0      38482   nrfx_clock.o
       518         30         19          0         92      19351   nrfx_gpiote.o
         4          0         12          0          0       2287   nrfx_prs.o
      1396         46         37          0         52      25191   nrfx_twim.o
      1200         38         18          0         36      29540   nrfx_uarte.o
       378         34          0          0        648       8777   segger_rtt.o
       748         72          0          4          0       2743   system_nrf52810.o

    ----------------------------------------------------------------------
     21902       1830       3284        268       8044     784951   Object Totals
         0          0         32          0          0          0   (incl. Generated)
        42          0         24          3          0          0   (incl. Padding)

    ----------------------------------------------------------------------

      Code (inc. data)   RO Data    RW Data    ZI Data      Debug   Library Member Name

         8          4        133          0          0         68   ctype_o.o
         0          0          0          0          0          0   entry.o
         0          0          0          0          0          0   entry10a.o
         0          0          0          0          0          0   entry11a.o
         8          4          0          0          0          0   entry2.o
         4          0          0          0          0          0   entry5.o
         0          0          0          0          0          0   entry7b.o
         0          0          0          0          0          0   entry8b.o
         8          4          0          0          0          0   entry9a.o
        30          0          0          0          0          0   handlers.o
        36          8          0          0          0         68   init.o
         0          0          0          0          0          0   iusefp.o
        30          0          0          0          0         68   llshl.o
        32          0          0          0          0         68   llushr.o
       188         20          0          0          0        160   malloc.o
        36          0          0          0          0         68   memcpya.o
        36          0          0          0          0        108   memseta.o
         0          0          0          8          0          0   mvars.o
        18          0          0          0          0         68   strcpy.o
        14          0          0          0          0         68   strlen.o
        98          0          0          0          0         92   uldiv.o
       176          0          0          0          0        140   fadd.o
       110          0          0          0          0        168   fepilogue.o
        40          0          0          0          0         68   ffixui.o
        10          0          0          0          0         68   ffltui.o
        24          0          0          0          0         68   fscalb.o

    ----------------------------------------------------------------------
       906         40        136          8          0       1348   Library Totals
         0          0          3          0          0          0   (incl. Padding)

    ----------------------------------------------------------------------

      Code (inc. data)   RO Data    RW Data    ZI Data      Debug   Library Name

       546         40        133          8          0        836   mc_w.l
       360          0          0          0          0        512   mf_w.l

    ----------------------------------------------------------------------
       906         40        136          8          0       1348   Library Totals

    ----------------------------------------------------------------------

==============================================================================


      Code (inc. data)   RO Data    RW Data    ZI Data      Debug   

     22808       1870       3420        276       8044     772099   Grand Totals
     22808       1870       3420        276       8044     772099   ELF Image Totals
     22808       1870       3420        276          0          0   ROM Totals

==============================================================================

    Total RO  Size (Code + RO Data)                26228 (  25.61kB)
    Total RW  Size (RW Data + ZI Data)              8320 (   8.13kB)
    Total ROM Size (Code + RO Data + RW Data)      26504 (  25.88kB)

==============================================================================

